:100000000C94051A0C94361A0C94361A0C94361A61
:100010000C94361A0C94361A0C94361A0C94361A20
:100020000C94361A0C94361A0C94361A0C94361A10
:100030000C94361A0C948CCD0C94361A0C94361AF7
:100040000C94361A0C9418BC0C94361A0C94361A6C
:100050000C94361A0C94361A0C944AE30D94DE0E66
:100060000C94361A0C94365F0C94361A0C94361A8B
:100070000C94361A0C94361A0C94361A0C94361AC0
:100080000C94361A0C94361A0C94361A0C94361AB0
:100090000C94361A0C94361A0C94361A0C94361AA0
:1000A0000C94361A0C94361A0C94361A0C94361A90
:1000B0000C94361A0C94361A0C94361A0C94361A80
:1000C0000C94361A0C94361A0C94361A0C94361A70
:1000D0000C94361A0C94361A0C94361A0C94361A60
:1000E0000C94361A0BA2F2A10EA2F5A1F8A104A25B
:1000F000FBA109A2FEA101A2FA00140126012C0114
:10010000D800F200C800EC00EA00220100011E0144
:10011000F400DE00F200D200F600F000E600CC00B1
:100120000C010E01CE00E000F800D400180104011B
:10013000E400DA00D600CA00E0000A01EE00160171
:10014000084AD73B3BCE016E84BCBFFDC12F3D6C3E
:1001500074319ABD56833DDA3D00C77F11BED9E4A4
:10016000BB4C3E916BAAAABE000000803F05A84C84
:10017000CDB2D44EB93836A9020C50B99186880850
:100180003CA6AAAA2ABE000000803F000D94AC1530
:100190000D94620D0D94690E0D94FF0D0D94180EC3
:1001A0000D949D070D94880D0D942A0E0D945F0EED
:1001B0000D94570D0D94500E0D94010A0D94820D5F
:1001C0000D94910E0D94C3140D94460E0D94FA0DDA
:1001D0000D94030A0D946C0D0D94660D0D947D0E17
:1001E0000D94900D0D94950D0D947E0D0D948C0D28
:1001F0000D94220E0D945B0D0D94E4350D94A40F17
:100200000D94740D0D94E83C0D943C0E0D948615E0
:100210000D94E8050D94730E0D94040E0D940E0EBE
:100220000D94020D0D94A0140D945E0D0D94870E87
:100230000D94320E0D94842A0D94FD0C0D947A0DBC
:100240000D9489150D94700D0D94A51F0D944D0DF1
:100250000D94FF0C0D948F170D94510D4E414E4986
:100260004E495459494E46CDCCCC3D0AD7233C1774
:10027000B7D13877CC2B329595E6241FB14F0A00C1
:100280000020410000C84200401C4620BCBE4CCAB1
:100290001B0E5AAEC59D74434F4D4D554E494341BB
:1002A00054494F4E0044525952554E004552524FF8
:1002B000525300494E464F004543484F00536C652A
:1002C00065702E2E2E00205A3A200020593A200028
:1002D00042656420583A2000436C69636B20746F58
:1002E00020726573756D652E2E2E004E6F206D6F1A
:1002F00076652E00456E642066696C65206C6973B6
:10030000740A00426567696E2066696C65206C69D5
:1003100073740A004D31323500286E6F2066696CA7
:100320006529005344207072696E74696E6720629B
:1003300079746520004E6F74205344207072696E8A
:1003400074696E670A0043757272656E742066691F
:100350006C653A200046696C652064656C6574655F
:10036000643A0044656C6574696F6E206661696CFF
:1003700065642C2046696C653A2000256973002568
:10038000696D20256973002569682025696D202520
:10039000697300256964202569682025696D202519
:1003A00069730025697920256964202569682025FD
:1003B000696D20256973005072696E742074696DCF
:1003C000653A2000B802B302AC02A50297026F663C
:1003D000660044454255473A004B494C4C45442E33
:1003E00020004D3131332053006F6B00416E796333
:1003F00075626963204C696E65617220504C55537B
:10040000204F66662E002C20002C200054484552B8
:100410004D414C5F50524F54454354494F4E00415B
:1004200055544F5245504F52545F53445F535441BB
:1004300054555300454D455247454E43595F504131
:100440005253455200434153455F4C494748545F1E
:100450004252494748544E45535300544F47474C26
:10046000455F4C494748545300534F4654574152F7
:10047000455F504F574552004255494C445F5045E7
:100480005243454E54004C4556454C494E475F44F7
:10049000415441005A5F50524F4245004155544F1C
:1004A0004C4556454C005052494E545F4A4F42000D
:1004B00050524F4752455353004155544F524550A7
:1004C0004F52545F54454D5000564F4C554D455476
:1004D00052494300454550524F4D00534552494102
:1004E0004C5F584F4E5F584F4646004649524D5755
:1004F0004152455F4E414D453A4D61726C696E20E7
:100500006275676669782D312E312E78202847690B
:10051000746875622920534F555243455F434F44D9
:10052000455F55524C3A68747470733A2F2F67695F
:10053000746875622E636F6D2F4D61726C696E46C3
:1005400069726D776172652F4D61726C696E2050B2
:10055000524F544F434F4C5F56455253494F4E3ABA
:10056000312E30204D414348494E455F5459504546
:100570003A416E796375626963204C696E65617298
:1005800020504C55532045585452554445525F43D2
:100590004F554E543A3120555549443A6365646588
:1005A000326132662D343161322D343734382D3991
:1005B0006231322D633535633632663336376666DF
:1005C0000A002F2F20004D31343520533C696E64D2
:1005D00065783E206F7574206F662072616E676566
:1005E0002028302D31290A00205400205200416378
:1005F00063656C65726174696F6E3A2050002046C5
:100600006C6F773A20000001363726FF02FFFF3576
:100610003C3D38FF0FFFFF312E303E1213FFFFFF2E
:1006200028FF0C0809FFFF071A1C18FFFF2A0844BF
:100630000A2C4320643A0020693A0020703A0049AD
:100640006E76616C69642065787472756465720A8F
:100650000043290A0061626C656420286D696E2080
:1006600074656D702000436F6C64206578747275DA
:1006700064657320617265200020643A0020693A45
:100680000020703A004E6F2063617365206C6967CB
:1006900068740A00426564204C6576656C696E6713
:1006A00020004661696C656420746F20656E61622C
:1006B0006C6520426564204C6576656C696E670ADE
:1006C00000426564204C6576656C20436F727265EC
:1006D0006374696F6E204D61747269783A004545A4
:1006E00050524F4D204F4B0A003F5A206F757420D7
:1006F0006F662072616E676520282D333020746F1D
:10070000203330290A003A200050726F6265205A67
:10071000204F666673657400416374697665204591
:10072000787472756465723A2000496E76616C69FE
:10073000642065787472756465720A007879007A4D
:100740007800797A00207A00207900207800630010
:100750002E2020202000253033692E7800302E25D1
:10076000303369002073643A0073746420646576E2
:100770003A00737464206465763A004E6F20636FAC
:100780006E76657267656E63650049746572617443
:10079000696F6E203A2025303269005361766520FA
:1007A00077697468204D35303020616E642F6F7228
:1007B00020636F707920746F20436F6E6669677570
:1007C000726174696F6E2E6800253033692E78006F
:1007D000302E253033690043616C6962726174693F
:1007E0006F6E2073643A00726F6C6C696E67206282
:1007F00061636B2E00737464206465763A00436114
:100800006C6962726174696F6E204F4B00456E6453
:10081000204452592D52554E00436F7272656374D5
:100820002064656C74612073657474696E677320ED
:1008300077697468204D36363520616E64204D36F8
:1008400036360A0020284452592D52554E29003F71
:10085000284D3636352042296564207261646975F9
:100860007320697320696D706C61757369626C6562
:100870002E0A00436865636B696E672E2E2E204139
:100880004300473333204175746F2043616C6962C4
:10089000726174650A003F2856296572626F73653C
:1008A000206C6576656C20697320696D706C61756C
:1008B0007369626C652028302D33292E0A003F2889
:1008C00046296F72636520697465726174696F6E21
:1008D00020697320696D706C61757369626C652045
:1008E00028302D3330292E0A003F284329616C69B6
:1008F00062726174696F6E20707265636973696F8B
:100900006E20697320696D706C61757369626C65C6
:1009100020283E3D30292E0A003F2850296F696E5D
:10092000747320697320696D706C61757369626C92
:10093000652028302D3130292E0A0020496E76613D
:100940006C696420657874727564657220000000BB
:10095000E8C20000E8C2000000000000E842000019
:10096000E8420000A043486F6D652025732573257C
:1009700073206669727374002066697273740A006A
:100980005A0059005800486F6D65200050726F6220
:10099000696E67206661696C65640A0050726F62F7
:1009A000696E67206661696C656400205A3A2000B0
:1009B00020593A200042656420583A200047322FDF
:1009C00047332062616420706172616D6574657285
:1009D000730A004B494C4C45442E200053544F5051
:1009E0005045442E20005072696E746572207374F5
:1009F0006F707065642064756520746F2065727215
:100A00006F72732E20466978207468652065727253
:100A10006F7220616E6420757365204D39393920FD
:100A2000746F20726573746172742E202854656D22
:100A30007065726174757265206973207265736583
:100A4000742E205365742069742061667465722069
:100A500072657374617274696E67290A004E6F2043
:100A6000436865636B73756D2077697468206C6982
:100A70006E65206E756D6265722C204C61737420FA
:100A80004C696E653A20004E6F20436865636B7356
:100A9000756D2077697468206C696E65206E756D60
:100AA0006265722C204C617374204C696E653A202B
:100AB00000636865636B73756D206D69736D617438
:100AC00063682C204C617374204C696E653A200079
:100AD0004C696E65204E756D626572206973206E7B
:100AE0006F74204C617374204C696E65204E756D77
:100AF0006265722B312C204C617374204C696E65D9
:100B00003A20004D313130004D33310053442072D2
:100B1000656164206572726F720A00446F6E6520B1
:100B20007072696E74696E672066696C650A00523E
:100B30006573656E643A20006F6B0020746F6F20E0
:100B40006C6F6E6720657874727573696F6E207054
:100B5000726576656E7465640A0020636F6C64204C
:100B6000657874727573696F6E2070726576656EE4
:100B70007465640A00627573793A207061757365F3
:100B80006420666F7220696E7075740A00627573F6
:100B9000793A2070617573656420666F7220757391
:100BA00065720A00627573793A2070726F636573BB
:100BB00073696E670A004B494C4C45442E20004B2C
:100BC000494C4C20636175736564206279204B4900
:100BD0004C4C20627574746F6E2F70696E0A004BF6
:100BE000494C4C45442E20004B494C4C20636175C8
:100BF00073656420627920746F6F206D756368205F
:100C0000696E6163746976652074696D65202D2055
:100C100063757272656E7420636F6D6D616E643A98
:100C20002000506C656173652072657365740050B7
:100C300052494E5445522048414C5445440050724C
:100C4000696E7465722068616C7465642E206B69CE
:100C50006C6C28292063616C6C6564210A00656EE8
:100C60007175657565696E67202200000048420055
:100C700000484200004842000000005761726E695F
:100C80006E673A20486F6D696E672042756D7020FF
:100C900044697669736F72203C20310A000A0A0A9F
:100CA0000000A0400000A0400000A04000006843F9
:100CB000000068430000A043010101000021104230
:100CC0002063308440A550C660E770088129914AAE
:100CD000A16BB18CC1ADD1CEE1EFF1311210027335
:100CE000325222B5529442F772D662399318837BFE
:100CF000B35AA3BDD39CC3FFF3DEE3622443342085
:100D0000040114E664C774A44485546AA54BB5284D
:100D1000850995EEE5CFF5ACC58DD5533672261114
:100D2000163006D776F6669556B4465BB77AA7199D
:100D3000973887DFF7FEE79DD7BCC7C448E55886DC
:100D400068A7784008611802282338CCC9EDD98EED
:100D5000E9AFF9488969990AA92BB9F55AD44AB774
:100D60007A966A711A500A333A122AFDDBDCCBBF3D
:100D7000FB9EEB799B588B3BBB1AABA66C877CE444
:100D80004CC55C222C033C600C411CAEED8FFDEC8D
:100D9000CDCDDD2AAD0BBD688D499D977EB66ED554
:100DA0005EF44E133E322E511E700E9FFFBEEFDDDD
:100DB000DFFCCF1BBF3AAF599F788F8891A981CABA
:100DC000B1EBA10CD12DC14EF16FE18010A100C299
:100DD00030E3200450254046706760B9839893FB48
:100DE000A3DAB33DC31CD37FE35EF3B1029012F3E9
:100DF00022D2323542145277625672EAB5CBA5A898
:100E00009589856EF54FE52CD50DC5E234C324A038
:100E10001481046674476424540544DBA7FAB79927
:100E200087B8975FE77EF71DC73CD7D326F2369188
:100E300006B01657667676154634564CD96DC90EEF
:100E4000F92FE9C899E9898AB9ABA94458654806D8
:100E5000782768C018E1088238A3287DCB5CDB3F87
:100E6000EB1EFBF98BD89BBBAB9ABB754A545A3728
:100E70006A167AF10AD01AB32A923A2EFD0FED6C57
:100E8000DD4DCDAABD8BADE89DC98D267C076C6478
:100E90005C454CA23C832CE01CC10C1FEF3EFF5D67
:100EA000CF7CDF9BAFBABFD98FF89F176E367E55C8
:100EB0004E745E932EB23ED10EF01E7C3C3E5E2BF5
:100EC0003D3F2F5B5D3B2C2A225C00454550524F35
:100ED0004D206461746173697A65206572726F7206
:100EE0002E0A00290A002062797465733B20637220
:100EF00063200053657474696E67732053746F7256
:100F00006564202800290A002062797465733B20FB
:100F100063726320002073746F726564207365745C
:100F200074696E6773207265747269657665642092
:100F30002800202863616C63756C617465642921E5
:100F40000A0020213D2000454550524F4D2043527C
:100F500043206D69736D61746368202D202873745C
:100F60006F7265642920002053697A653A20004930
:100F70006E6465783A2000204D61726C696E3D5652
:100F80003535290A0028454550524F4D3D0045450D
:100F900050524F4D2076657273696F6E206D697384
:100FA0006D617463682000436172642072656D6FC7
:100FB000766564004361726420696E73657274655E
:100FC000640000000000000000000000A0430A0AC6
:100FD000426564204C6576656C20436F7272656370
:100FE00074696F6E204D61747269783A00202B002D
:100FF0000A436F72726563746564204265642048B9
:1010000065696768742076732E2042656420546F8A
:10101000706F6C6F67793A0A00202B000A42656492
:101020002048656967687420546F706F67726170DB
:1010300068793A0A2020202B2D2D2D204241434B48
:10104000202D2D2B0A2020207C2020202020202035
:10105000202020207C0A204C207C20202020282BAF
:1010600029202020207C20520A2045207C2020207E
:1010700020202020202020207C20490A2046207C7F
:1010800020282D29204E20282B29207C20470A208B
:1010900054207C20202020202020202020207C2064
:1010A000480A2020207C20202020282D29202020B4
:1010B000207C20540A2020207C202020202020205A
:1010C000202020207C0A2020204F2D2D2046524F0A
:1010D0004E54202D2D2B0A2028302C30290A004D6B
:1010E00065616E206F662073616D706C6564207041
:1010F0006F696E74733A200020643A200020623ACF
:10110000200045716E20636F656666696369656E70
:1011100074733A20613A2000202844525952554EA7
:101120002900473239204175746F20426564204C94
:101130006576656C696E67003F20284C2C522C4602
:101140002C4229206F7574206F6620626F756E6463
:10115000732E0A003F50726F626520706F696E7463
:10116000732028592920697320696D706C6175732B
:1011700069626C652028322D39292E0A003F507291
:101180006F626520706F696E74732028582920691A
:101190007320696D706C61757369626C65202832AB
:1011A0002D39292E0A003F2856296572626F736512
:1011B000206C6576656C20697320696D706C617553
:1011C0007369626C652028302D34292E0A004C6921
:1011D0006E656172204C6576656C696E6700457856
:1011E000747275646572733A203100687474703A71
:1011F0002F2F6D61726C696E66772E6F726700417A
:101200006E796375626963204C696E656172205006
:101210004C555300323031382D30372D3331006288
:1012200075676669782D312E312E78004D61726CAC
:10123000696E00546865726D6973746F72730042F1
:101240006F61726420496E666F005072696E7465DA
:101250007220496E666F004D61696E004D37303205
:1012600020542564004D363030204230205425640F
:10127000004D373032203B2564004D37303120544B
:10128000256400556E6C6F61642066696C616D65E4
:101290006E7400556E6C6F61642066696C616D657B
:1012A0006E74004D373032004D373031004C6F6175
:1012B000642066696C616D656E74004D3630302057
:1012C0004230004368616E67652066696C616D65D8
:1012D0006E740050726570617265005052494E54D0
:1012E0002050415553454400554E4C4F41442046F3
:1012F000494C414D454E54004C4F41442046494CC9
:10130000414D454E54005075726765206D6F726592
:1013100000436F6E74696E756500524553554D45B7
:10132000204F5054494F4E533A0020204E6F7A7A46
:101330006C653A20006368616E6765006F662074B3
:1013400068652066696C616D656E740057616974CB
:1013500020666F722073746172740020204E6F7A61
:101360007A6C653A200066696C616D656E742075F3
:101370006E6C6F6164005761697420666F72002043
:10138000204E6F7A7A6C653A2000506C6561736507
:1013900020776169742E2E2E0048656174696E672E
:1013A000206E6F7A7A6C650020204E6F7A7A6C65B9
:1013B0003A200068656174206E6F7A7A6C652E0041
:1013C000507265737320627574746F6E20746F0051
:1013D00020204E6F7A7A6C653A2000746F20636F1C
:1013E0006E74696E75652E2E2E00616E64207072AB
:1013F00065737320627574746F6E00496E736572E5
:10140000742066696C616D656E740020204E6F7A81
:101410007A6C653A200066696C616D656E74206C4B
:101420006F6164005761697420666F720020204EFE
:101430006F7A7A6C653A200066696C616D656E74CE
:10144000207075726765005761697420666F72005D
:10145000746F20726573756D6500576169742066DD
:101460006F72207072696E7400205A3A0020593AE7
:101470000020436F756E7420583A0020453A0020D2
:101480005A3A0020593A00583A003A004361703AFB
:1014900000205A00205900580020204D61783A2041
:1014A00000205A00205900580020204D696E3A2033
:1014B000004F6E20004F666600536F667420656EA5
:1014C0006473746F70733A20004B6420002364656A
:1014D00066696E652044454641554C545F004B6932
:1014E000200023646566696E652044454641554C7D
:1014F000545F004B70200023646566696E6520446C
:10150000454641554C545F00504944204175746F25
:1015100074756E652066696E697368656421205014
:10152000757420746865206C617374204B702C2076
:101530004B6920616E64204B6420636F6E7374612D
:101540006E74732066726F6D2062656C6F772069B0
:101550006E746F20436F6E66696775726174696F30
:101560006E2E680A00504944204175746F74756E80
:1015700065206661696C6564212074696D656F75AD
:10158000740A00453120544845524D414C20525573
:101590004E415741590042454420544845524D411F
:1015A0004C2052554E4157415900546865726D6147
:1015B0006C2052756E617761790045312048656114
:1015C00074696E67206661696C65640042656420B9
:1015D00068656174696E67206661696C656400485E
:1015E000656174696E67206661696C656400504965
:1015F00044204175746F74756E65206661696C6511
:1016000064212054656D7065726174757265207413
:101610006F6F20686967680A00204B643A200020D9
:101620004B693A2000204B703A20000A20436C613D
:101630007373696320504944200A002054753A208E
:1016400000204B753A2000206D61783A2000206D13
:10165000696E3A200020643A200020626961733A82
:101660002000504944204175746F74756E65206682
:1016700061696C6564212054656D70657261747573
:10168000726520746F6F20686967680A005049446A
:10169000204175746F74756E652073746172740A7D
:1016A00000504944204175746F74756E6520666101
:1016B000696C656421204261642065787472756488
:1016C0006572206E756D6265720A00496E7365728F
:1016D000742066696C616D656E7420616E64207043
:1016E0007265737320627574746F6E0A0050726550
:1016F000737320627574746F6E20746F20686561F7
:1017000074206E6F7A7A6C650A00496E7365727424
:101710002066696C616D656E7420616E6420707204
:1017200065737320627574746F6E20286F72204D1C
:10173000313038290A0020746F6F206C6F6E67207B
:10174000657874727573696F6E2070726576656EF8
:101750007465640A0020636F6C6420657874727528
:1017600073696F6E2070726576656E7465640A00C9
:1017700024F4D43050C38E20C2A24017828B701143
:10178000127A910D816CD90AA861E108C7586607E1
:10179000615143061E4B5D05C145A7041A41110462
:1017A000093D9803713931034036DB0265339102FC
:1017B000D4305402802E1D02632CEE01752AC5011F
:1017C000B028A001102781018F2564012B244B0133
:1017D000E0223401AC211F018D200D01801FFC008F
:1017E000841EED00971DDF00B81CD200E61BC6006A
:1017F000201BBC00641AB200B219A8000A19A0008C
:101800006A189900D117910040178B00B516840013
:1018100031167E00B31579003A157300C7146F00B6
:1018200058146A00EE1366008813630025135E00E7
:10183000C7125B006C12570015125400C111510001
:1018400070114F0021114B00D61049008D10470038
:101850004610440002104200C00F4000800F3E00BE
:10186000420F3C00060F3B00CB0E3800930E3700B2
:101870005C0E3500270E3400F30D3200C10D31002F
:10188000900D3000600D2E00320D2D00050D2C0046
:10189000D90C2B00AE0C2900850C29005C0C27000C
:1018A000350C27000E0C2600E80B2400C40B240086
:1018B000A00B23007D0B23005A0B2100390B2100C4
:1018C000180B2000F80A1F00D90A1E00BB0A1E00D0
:1018D0009D0A1D00800A1D00630A1C00470A1B00A8
:1018E0002C0A1B00110A1A00F7091A00DD09190059
:1018F000C4091900AB091900920917007B091800E7
:10190000630917004C091600360916002009160055
:101910000A091500F5081500E0081400CC081400A9
:10192000B8081400A4081400900813007D081200E1
:101930006B08130058081200460812003408110002
:10194000230811001208110001081100F00710000F
:10195000E0071000D0071000C0071000B0070F000C
:10196000A107100091070E0083070F0074070F00F6
:1019700065070E0057070E0049070E003B070D00D4
:101980002E070E0020070D0013070D0006070D009F
:10199000F9060C00ED060D00E0060C00D4060C0064
:1019A000C8060C00BC060C00B0060C00A4060B0018
:1019B00099060C008D060B0082060B0077060B00C3
:1019C0006C060B0061060A0057060B004C060A0065
:1019D00042060A0038060A002E060A0024060A00FB
:1019E0001A060A001006090007060A00FD0509008C
:1019F000F4050900EB050900E2050900D905090015
:101A0000D0050900C7050900BE050900B505080095
:101A1000AD050800A50509009C050800940508000F
:101A20008C050800840508007C0508007405080082
:101A30006C050700650508005D05070056050800F0
:101A40004E05070047050700400508003805070058
:101A5000310507002A050700230507001C050600BD
:101A6000160507000F050700080506000205070018
:101A7000FB040600F5040700EE040600E804060077
:101A8000E2040700DB040600D5040600CF040600CC
:101A9000C9040600C3040600BD040600B70406001E
:101AA000B1040500AC040600A6040600A00405006D
:101AB0009B04060095040500900406008A040500B6
:101AC00085040500800406007A04050075040500FD
:101AD000700405006B040500660405006104050040
:101AE0005C04050057040500520405004D04050080
:101AF00048040500430405003E0404003A040500C0
:101B000035040500300404002C04050027040400FB
:101B1000230405001E0404001A0404001604050032
:101B2000110404000D040400090405000404040069
:101B300000040400FC030400F8030400F4030400A0
:101B4000F0030400EC030400E8030400E4030400D1
:101B5000E0030400DC030400D8030400D403040001
:101B6000D0030400CC030400C8030300C503030032
:101B700024F404D9201BC40C5C0E9804C4095F0231
:101B800065077101F405F900FB04B3004804870000
:101B9000C10369005803550003034500BE023A0023
:101BA0008402310053022A00290225000402200089
:101BB000E4011C00C8011900AF01170098011400CE
:101BC00084011300710110006101100051010E0029
:101BD00043010D0036010B002B010B0020010B000F
:101BE000150109000C01090003010800FB000800B1
:101BF000F3000800EB000700E4000600DE0006002A
:101C0000D8000600D2000600CC000500C700050081
:101C1000C2000500BD000400B9000400B5000400C6
:101C2000B1000400AD000400A9000400A5000300F9
:101C3000A20003009F0004009B0003009800030023
:101C40009500020093000300900003008D00020045
:101C50008B0003008800020086000200840003005D
:101C6000810002007F0002007D0002007B00020074
:101C70007900020077000100760002007400020083
:101C800072000100710002006F0002006D0001008F
:101C90006C0002006A000100690002006700010098
:101CA000660001006500010064000200620001009E
:101CB00061000100600001005F0002005D000100A2
:101CC0005C0001005B0001005A00010059000100A6
:101CD00058000100570001005600010055000100A6
:101CE00054000100530000005300010052000100A5
:101CF00051000100500001004F0001004E000000A3
:101D00004E0001004D0001004C0001004B0000009E
:101D10004B0001004A00010049000100480000009A
:101D20004800010047000100460000004600010095
:101D30004500000045000100440001004300000090
:101D40004300010042000000420001004100000089
:101D500041000100400001003F0000003F00010081
:101D60003E0000003E0001003D0000003D0001007B
:101D70003C0000003C0000003C0001003B00000073
:101D80003B0001003A0000003A0001003900000069
:101D90003900010038000000380000003800010060
:101DA0003700000037000100360000003600000058
:101DB000360001003500000035000000350001004C
:101DC0003400000034000000340001003300000043
:101DD0003300000033000100320000003200000038
:101DE000320001003100000031000000310001002C
:101DF0003000000030000000300001002F00000023
:101E00002F0000002F0000002F0001002E00000016
:101E10002E0000002E0001002D0000002D0000000B
:101E20002D0000002D0001002C0000002C000000FF
:101E30002C0000002C0001002B0000002B000000F3
:101E40002B0000002B0001002A0000002A000000E7
:101E50002A0000002A0001002900000029000000DB
:101E600029000000290000002900010028000000CE
:101E700028000000280000002800000028000100C1
:101E800027000000270000002700000027000000B6
:101E900027000100260000002600000026000000A8
:101EA000260000002600010025000000250000009B
:101EB000250000002500000025000000250001008D
:101EC0002400000024000000240000002400000082
:101ED0002400010023000000230000002300000074
:101EE0002300000023000000230000002300010065
:101EF000220000002200000022000000220000005A
:101F0000220000002200010021000000210000004A
:101F1000210000002100000021000000210000003D
:101F2000210001002000000020000000200000002F
:101F30002000000020000000200000002000000021
:101F4000200001001F0000001F0000001F00000013
:101F50001F0000001F0000001F0000001F00010004
:101F60001E0000001E0000001E0000001E000000F9
:101F7000043700001E290000511B0000581000000B
:101F800010090000CC0400007802000041010000AC
:101F90001000C90210012C0140012201700118013A
:101FA000B0010E01F00104015002FA00B002F0008D
:101FB0003003E600D003DC009004D2007005C800B6
:101FC000A006BE000008B400B009AA00D00BA00013
:101FD000600E960060118C000015820020197800B8
:101FE000C01D6E00A0226400B0275A00902C500043
:101FF00000314600E0343C0010383200903A2800AE
:10200000603C1E00A03D1400803E0A00203F0000FE
:10201000202F002042403A0020403A0025753A2502
:1020200030327500253032753A25303275002D2D4D
:102030002D0053440020202020202000202020209C
:102040000000002200250028002B002E0031003463
:102050000002010000050108010B0100002000231F
:1020600000260029002C002F003200000100000390
:10207000010601090105050505070508080808020C
:102080000202020A0A080804040404010101010111
:102090000101010303030303030303040707070C00
:1020A0000C0C0C0C0C0C0C020202020606060606B6
:1020B0000606060B0B0B0B0B0B0B0B010210202063
:1020C000080810204010204080020102010804028C
:1020D0000101020408102040808040201008040202
:1020E000018004020180402010080402010804025B
:1020F0000101020408102040800102040810204061
:102100008000000A0B02090C0D0E080703040100F1
:1021100000000000000000000000000000000000BF
:10212000000000000000000000000000001211107C
:10213000000000000000000000000000000000009F
:102140000000000000000002000000000102040482
:102150000000001C1C0C040404020100000000002C
:1021600004081000000000002D2D2D2D2D2D007CC9
:102170004D61726C696E7C002D2D2D2D2D2D006210
:1021800075676669782D312E312E78006275676625
:1021900069782D312E312E7800002020506C616E30
:1021A0006E657242756666657242797465733A202F
:1021B000002046726565204D656D6F72793A20008A
:1021C000436F6D70696C65643A204A616E203236E7
:1021D00020323031390A00207C20417574686F72DA
:1021E0003A2028416C6C657374657220466F7829BB
:1021F0000A00323031382D30372D333100204C6118
:10220000737420557064617465643A200062756768
:102210006669782D312E312E780A004D61726C6915
:102220006E0020536F667477617265205265736526
:10223000740A00205761746368646F672052657385
:1022400065740A002042726F776E206F7574205299
:10225000657365740A002045787465726E616C2040
:1022600052657365740A00506F77657255700A0085
:1022700073746172740A006175746F25692E67004A
:102280006572726F722077726974696E6720746FFD
:102290002066696C650A00456E6473746F70732004
:1022A000256320256320256320256300205A3A00FA
:1022B00020593A0020583A00656E6473746F707349
:1022C000206869743A2000446F6E652073617669F6
:1022D0006E672066696C652E0A004D3239005072B7
:1022E00065686561742041425320456E64005072F8
:1022F00065686561742041425320426564005072F4
:102300006568656174204142530050726570617266
:1023100065005072656865617420414253005072D7
:10232000656865617420504C4100436F6F6C646F49
:10233000776E004368616E67652066696C616D65E4
:102340006E740044697361626C65207374657070AB
:10235000657273004D3834004F6666004F6E200082
:10236000426564204C6576656C696E670044656CF7
:1023700074612043616C6962726174696F6E004CB4
:102380006576656C20626564004732380A473239E9
:10239000004175746F20686F6D6500473238004DDD
:1023A0006F76652061786973004D61696E00486FD2
:1023B0006D696E672058595A004732380044696188
:1023C0006720526F64004469616720526F64005453
:1023D0007A00547A00547900547900547800547883
:1023E00000526164697573005261646975730045D8
:1023F0007A00457A004579004579004578004578AE
:1024000000486569676874004865696768740044D6
:10241000656C74612043616C6962726174696F6E8E
:10242000004573746570732F6D6D0045737465702E
:10243000732F6D6D004373746570732F6D6D004362
:1024400073746570732F6D6D004273746570732FB4
:102450006D6D004273746570732F6D6D0041737400
:102460006570732F6D6D004173746570732F6D6DA2
:10247000004D6F74696F6E0053746570732F6D6DCE
:10248000004A65726B00416363656C6572617469D3
:102490006F6E0056656C6F636974790050726F627D
:1024A00065205A204F66667365740050726F6265CE
:1024B000205A204F666673657400436F6E74726FA6
:1024C0006C004C6F6164206D6D004C6F6164206D19
:1024D0006D004C6F6164206D6D00556E6C6F6164B2
:1024E000206D6D00556E6C6F6164206D6D00556ED2
:1024F0006C6F6164206D6D0046696C2E20446961CB
:102500002E0046696C2E204469612E004F666600DD
:102510004F6E20004520696E206D6D3300436F6E55
:1025200074726F6C0043616E6E6F7420656E7465BB
:1025300072207375626469723A2000052E2E004D78
:1025400061696E004D61782054656D703A203132BA
:1025500030004D696E2054656D703A20350054424C
:1025600065643A4154432031303447542D32004D94
:1025700061782054656D703A20323735004D696EB0
:102580002054656D703A20350054303A2041544350
:102590002031303447542D32005053553A2047658E
:1025A0006E657269630050726F746F636F6C3A206E
:1025B000312E3000426175643A203235303030308F
:1025C0000052414D505320312E3400496E697469D8
:1025D000616C697A6520454550524F4D00436F6EDE
:1025E00074726F6C00526573746F726520666169F6
:1025F0006C73616665004C6F616420736574746907
:102600006E677300496E697469616C697A6520450B
:102610004550524F4D0053746F726520736574744A
:10262000696E67730046696C616D656E74004D6F0D
:1026300074696F6E0054656D706572617475726552
:10264000004D61696E004D333033205531204525F2
:1026500069205325690050726568656174204142A4
:102660005320636F6E660050726568656174205018
:102670004C4120636F6E6600504944204175746F71
:1026800074756E6500504944204175746F74756EA1
:102690006500504944204175746F74756E65005033
:1026A00049442D44005049442D44005049442D498B
:1026B000005049442D49005049442D500050494490
:1026C0002D500020022046616374002002204661E4
:1026D0006374002002204D6178002002204D617853
:1026E000002002204D6178002002204D696E0020FC
:1026F00002204D696E002002204D696E004F666613
:10270000004F6E20004175746F74656D70004661F6
:102710006E2073706565640046616E207370656538
:10272000640046616E2073706565640042656400F4
:1027300042656400426564004E6F7A7A6C65004EB3
:102740006F7A7A6C65004E6F7A7A6C6500436F6EB3
:1027500074726F6C0053746F726520736574746962
:102760006E67730042656400426564004265640000
:102770004E6F7A7A6C65004E6F7A7A6C65004E6F98
:102780007A7A6C650046616E2073706565640046F8
:10279000616E2073706565640046616E20737065BC
:1027A00065640054656D7065726174757265002CA6
:1027B000FFFFFFFFFF0001010101016265640A00E4
:1027C0002C2073797374656D2073746F70706564F9
:1027D00021204865617465725F49443A2000426572
:1027E000642068656174696E67206661696C656400
:1027F0000048656174696E67206661696C65640094
:1028000045312048656174696E67206661696C6551
:10281000640048656174696E67206661696C65640F
:1028200000453120544845524D414C2052554E41AF
:102830005741590042454420544845524D414C208F
:1028400052554E4157415900546865726D616C2074
:1028500052756E61776179004531204572723A2078
:102860004D415854454D50004572723A204D4158E3
:1028700054454D5020424544004D415854454D501B
:10288000207472696767657265640045312045721E
:10289000723A204D494E54454D50004572723A20CF
:1028A0004D494E54454D5020424544004D494E54EB
:1028B000454D5020747269676765726564004D38D4
:1028C0003420582059205A20450043616C696272B7
:1028D000617465205A0043616C696272617465209D
:1028E000590043616C6962726174652058004175DA
:1028F000746F20686F6D650044656C74612053656A
:102900007474696E6773004C6F61642073657474CE
:10291000696E67730043616C69627261746520431C
:10292000656E7465720053746F726520736574749C
:10293000696E6773004175746F2043616C696272E0
:102940006174696F6E00473333004D61696E004DED
:102950006F76652058004D6F76652059004D6F7673
:1029600065205A004578747275646572004D6F7603
:102970006520302E316D6D004D6F766520316D6DA7
:10298000004D6F76652031306D6D004D6F7665209E
:1029900061786973004578747275646572004D6F73
:1029A0007665205A004D6F76652059004D6F76652B
:1029B0002058004D6F76696E672E2E2E0045787474
:1029C0007275646572004175746F20686F6D650083
:1029D000473238004D6F7665205A00467265652093
:1029E0005859004D6F76652059004D6F7665205817
:1029F000004F6666004F6E2000536F667420456E70
:102A00006473746F70730050726570617265004911
:102A10006E736572742066696C616D656E74206199
:102A20006E6420707265737320627574746F6E20AB
:102A3000286F72204D313038290A005344206361D9
:102A40007264206F6B0A006F70656E526F6F742036
:102A50006661696C65640A00766F6C756D652E69D8
:102A60006E6974206661696C65640A00534420696C
:102A70006E6974206661696C0A0057726974696EC8
:102A80006720746F2066696C653A20006F70656E10
:102A9000206661696C65642C2046696C653A20008B
:102AA0006F70656E206661696C65642C2046696C88
:102AB000653A200046696C652073656C65637465D2
:102AC000640A002053697A653A200046696C6520E3
:102AD0006F70656E65643A20002066696C653A2007
:102AE00000646F696E67006672657368004E6F7789
:102AF0002000454E4420535542524F5554494E45AF
:102B00000A002220706F73002220706172656E745B
:102B10003A2200535542524F5554494E45204341A5
:102B20004C4C207461726765743A22004B494C4CDE
:102B300045442E2000747279696E6720746F20639B
:102B4000616C6C207375622D67636F6465206669C4
:102B50006C6573207769746820746F6F206D616E87
:102B600079206C6576656C732E204D4158206C651C
:102B700076656C2069733A004572726F723A00484C
:102B8000617264636F6465642044656661756C742A
:102B90002053657474696E6773204C6F616465645B
:102BA0000A00E8030000E8030000E8030000E8036F
:102BB0000000000048430000484300004843000074
:102BC00048420000A0420000A0420000A0420000D5
:102BD000C0423A0A0020286D6D290020204D363071
:102BE0003320002055004C0046696C616D656E74A1
:102BF000206C6F61642F756E6C6F6164206C656E04
:102C0000677468733A0A0020204D383531205A0025
:102C10005A2D50726F6265204F666673657400208E
:102C2000440020490020204D3330342050002044FF
:102C30000020490020204D333031205000504944BD
:102C40002073657474696E67733A0A002046002029
:102C5000420020480020204D3134352053004D6182
:102C600074657269616C206865617475702070614B
:102C700072616D65746572733A0A00205A002059BA
:102C8000002058002042002053002048002052001D
:102C900020204D363635204C0044656C746120731D
:102CA000657474696E67733A204C3C646961676F40
:102CB0006E616C5F726F643E20523C726164697534
:102CC000733E20483C6865696768743E20533C73D6
:102CD00065676D656E74735F7065725F733E2042E9
:102CE0003C63616C6962726174696F6E20726164C9
:102CF0006975733E2058595A3C746F77657220612C
:102D00006E676C6520636F7272656374696F6E7352
:102D10003E0A00205A0020590020204D3636362029
:102D20005800456E6473746F702061646A757374C3
:102D30006D656E743A0A0020204D34323020530005
:102D40004175746F20426564204C6576656C696ED0
:102D5000673A0A00204500205A00205900205800F8
:102D600020540020530020204D32303520510020C7
:102D7000453C6D61785F655F6A65726B3E00205807
:102D80003C6D61785F785F6A65726B3E20593C6D7F
:102D900061785F795F6A65726B3E205A3C6D61783D
:102DA0005F7A5F6A65726B3E00416476616E63654F
:102DB000643A20513C6D696E5F7365676D656E7432
:102DC0005F74696D655F75733E20533C6D696E5F1E
:102DD00066656564726174653E20543C6D696E5F22
:102DE00074726176656C5F66656564726174653E78
:102DF0000020540020520020204D3230342050005A
:102E0000416363656C65726174696F6E2028756ECD
:102E10006974732F7332293A20503C7072696E7452
:102E20005F616363656C3E20523C726574726163DE
:102E3000745F616363656C3E20543C7472617665B7
:102E40006C5F616363656C3E0A00204500205A0098
:102E500020590020204D3230312058004D617869D2
:102E60006D756D20416363656C65726174696F6E29
:102E70002028756E6974732F7332293A0A00204531
:102E800000205A0020590020204D323033205800B5
:102E90004D6178696D756D206665656472617465F4
:102EA000732028756E6974732F73293A0A002045C0
:102EB00000205A0020590020204D3932205800535C
:102EC000746570732070657220756E69743A0A00BB
:102ED00020204D3230302044300A0020204D323046
:102EE000302044002044697361626C65640A0046C6
:102EF000696C616D656E742073657474696E677357
:102F00003A0020204D3134392043203B20556E6952
:102F1000747320696E2043656C736975730A0020B1
:102F200020473231202020203B006F70656E2066E4
:102F300061696C65642C2046696C653A20004361C8
:102F40006E6E6F74206F70656E2073756264697247
:102F500020006563686F3A00001C1F11111F0000FC
:102F60000006191803130C00040E1F041C000000B7
:102F7000000E1315110E00001C1018170506050091
:102F8000040A0A0A0A11110E0C12120C00000000A9
:102F9000001F1511151F00005654726176206D69CF
:102FA0006E005654726176206D696E0056547261DF
:102FB00076206D696E00566D696E00566D696E0003
:102FC000566D696E00566D6178204500566D6178CA
:102FD000204500566D6178204500566D617820438C
:102FE00000566D6178204300566D6178204300568D
:102FF0006D6178204200566D6178204200566D6107
:1030000078204200566D6178204100566D6178202D
:103010004100566D61782041004D6F74696F6E00FC
:10302000416D6178204500416D6178204500416D1A
:103030006178204300416D6178204300416D6178E3
:10304000204200416D6178204200416D617820414D
:1030500000416D6178204100412D74726176656C8C
:1030600000412D74726176656C00412D7265747239
:1030700061637400412D7265747261637400416311
:1030800063656C00416363656C004D6F74696F6EBE
:103090000056652D6A65726B0056652D6A65726B08
:1030A0000056652D6A65726B0056632D6A65726BFA
:1030B0000056632D6A65726B0056632D6A65726BEC
:1030C0000056622D6A65726B0056622D6A65726BDE
:1030D0000056622D6A65726B0056612D6A65726BCF
:1030E0000056612D6A65726B0056612D6A65726BC0
:1030F000004D6F74696F6E000000210024002700EE
:103100002A002D00300033000101000004010701F6
:103110000A01416E796375626963204C696E65616D
:103120007220504C55532052656164792E005072C4
:10313000696E74696E672E2E2E005072696E74204F
:10314000706175736564004D313235004D32340065
:103150005072696E742061626F72746564004E6FA4
:103160002053442063617264005072696E7420665B
:10317000726F6D2053440053746F70207072696ECB
:103180007400526573756D65207072696E740041CC
:10319000626F7574205072696E746572005061754B
:1031A0007365207072696E7400436F6E74726F6C19
:1031B00000507265706172650054756E6500496EED
:1031C000666F2073637265656E004368616E676544
:1031D0002066696C616D656E7400466C6F770046A1
:1031E0006C6F7700466C6F770046616E2073706578
:1031F00065640046616E2073706565640046616EAB
:103200002073706565640042656400426564004235
:103210006564004E6F7A7A6C65004E6F7A7A6C65E1
:10322000004E6F7A7A6C6500537065656400537068
:10323000656564005370656564004D61696E00509A
:1032400072656865617420504C4120456E64005081
:1032500072656865617420504C412042656400507D
:1032600072656865617420504C41005072657061F0
:103270007265004572726F722077726974696E6749
:1032800020746F20454550524F4D210A004368611C
:103290006E67652066696C616D656E7400556E6C55
:1032A0006F61642066696C616D656E74004C6F615E
:1032B000642066696C616D656E7400507265686546
:1032C00061742041425300507265686561742050FA
:1032D0004C41004368616E67652066696C616D658D
:1032E0006E74004D3234004D323320257300556E1C
:1032F0006B6E6F776E20636F6D6D616E643A202226
:1033000000486F74656E6420746F6F20636F6C6427
:103310000A004D3630303A20546F6F20636F6C6472
:1033200000486F74656E6420746F6F20636F6C6407
:103330000A0050726F7465637465642050696E0A88
:103340000020573A004520436F6F6C696E672E2E40
:103350002E00452048656174696E672E2E2E002070
:10336000573A0042656420636F6F6C696E672E2E5A
:103370002E004265642068656174696E672E2E2E8A
:1033800000486F6D696E67206661696C6564005402
:103390005249474745524544006F70656E003A20D8
:1033A000007A5F6D6178007A5F6D696E00795F6D9C
:1033B000617800785F6D6178005265706F72746932
:1033C0006E6720656E6473746F70207374617475BA
:1033D000730A0020200020205261646975733A004E
:1033E000547A005479005478002020526164697541
:1033F000733A00457A004579004578002E486569A2
:103400006768743A00000201FC0011241FBECFEF70
:10341000D1E2DEBFCDBF00E00CBF13E0A0E0B2E020
:10342000E0E0FAE902E00BBF02C007900D92AC3475
:10343000B107D9F723E1ACE4B3E001C01D92A33A90
:10344000B207E1F71AE1C4E0DAE100E006C0219733
:103450000109802FFE010F945E4CC330D10780E03C
:103460000807A9F70F9488370D94EF4C0C940000CF
:103470002F923F924F925F926F927F928F929F9284
:10348000AF92BF92CF92DF92EF92FF920F931F9372
:10349000CF93DF93CDB7DEB7A7970FB6F894DEBF13
:1034A0000FBECDBF41E04093EF0C80919C138D3453
:1034B00009F4C6C1843511F40C94212D873411F020
:1034C0000C946D2D20919A1330919B132C31310562
:1034D00009F4C7C09CF4243031053CF42230310596
:1034E0000CF044C037FF28C0A7C12430310509F4CF
:1034F00046C02B31310509F481C09EC1213231050E
:1035000009F41FC14CF42D31310509F4AEC02E3140
:10351000310509F4AEC090C12B35310509F415C150
:103520002C35310509F415C12A35310509F084C15E
:10353000109250030C946F2D80912A02882311F46D
:103540000C946F2D8AE50E942D5B082F89E50E945F
:103550002D5B182F88E50E942D5B402F612F0E9464
:10356000E14981110C946F2D0C94742D81E022306F
:10357000310509F080E00E94934A0C946F2D80E59C
:103580000E94765B882329F00E94BA5A6B017C0165
:1035900003C0C12CD12C760183E50E94765B882381
:1035A00061F00E94FA5A20E030E04AE754E40F94B8
:1035B00034450F94424A6B017C010E9443BB8091C9
:1035C000F20C811105C060E08DEB92E00E949288C0
:1035D0000F94D20EC60ED71EE81EF91E0F94D20EFF
:1035E000DC01CB018C199D09AE09BF09B7FD02C0F2
:1035F0000C946F2D80E00E94D05FF0CF41E061E03D
:1036000081E00E94E14981110C946F2D80E090E0EF
:10361000A4EDB2EC89839A83AB83BC8380E090E015
:10362000A4EDB2E48D839E83AF83B88780E090E001
:10363000A0EFB1E489879A87AB87BC8780E50E94B9
:10364000765B882319F00E94CA5A01C060E068A323
:10365000BE016F5F7F4FCE0180960F948D2E0C942C
:103660006F2D0E9488740C946F2D0E94588C0C94BE
:103670006F2DC090560DD090570DE090580DF090E2
:10368000590D88E50E94765B811108C020E030E08A
:10369000A901C701B6010F94F94802C00E94FA5A65
:1036A00068A379A38AA39BA3C0905A0DD0905B0D09
:1036B000E0905C0DF0905D0D89E50E94765B8111D4
:1036C00008C020E030E0A901C701B6010F94F94815
:1036D00002C00E94FA5A6B017C0169837A838B8352
:1036E0009C8368A179A18AA19BA19B01AC010F9445
:1036F00034454B015C01A7019601C701B6010F9447
:1037000034459B01AC01C501B4010F94F9486B012C
:103710007C0120E030E442E556E40F94CF441816D3
:1037200014F40C946F2D20E030E94FE256E4C70109
:10373000B6010F94CF44181614F40C946F2D0C940A
:10374000792D0E94AF2E0C946F2D409350030C9452
:103750006F2DFBE52F2EF2E03F2EA6EDEA2EACE01A
:10376000FA2EB6E5CB2EBDE0DB2E00E010E0F10135
:1037700081911F010E94765B882309F449C00E9451
:10378000FA5A2B013C01133049F0F70120813181B5
:10379000428153810F94F8482B013C01F6012081AE
:1037A000318142815381C301B2010F94F8484B012A
:1037B0005C012DEB37E346E855EB0F946D4B87FD2D
:1037C0000AC02DEB37E346E855E3C501B4010F9479
:1037D000CF441816ECF4133051F44092620D50921D
:1037E000630D6092640D7092650D01E011C0A5013A
:1037F0009401F70160817181828193810F94F9486E
:10380000F7016083718382839383812F0E94B25476
:103810001F5FF4E0EF0EF11C24E0C20ED11C143047
:1038200009F0A5CF002321F082E69DE00E94DBF89D
:103830000E946DAC0C946F2D0F9487200C946F2D0B
:1038400080919A1390919B138837910511F40C94F1
:1038500099250CF0E3C08D34910509F4ADC50CF049
:1038600058C08931910509F41DC31CF584319105B7
:1038700009F406C27CF48131910509F47CC22CF470
:10388000029708F400C20C941E2D429709F47FC7DA
:103890000C941E2D8631910509F4BEC20CF4B8C2F9
:1038A0008731910509F4BEC2489709F4D1C20C943E
:1038B0001E2D8E31910509F4B3C384F48B3191052B
:1038C00009F40CC30CF4FCC28C31910509F49EC3BD
:1038D0004D9711F40C946F2D0C941E2D8A32910586
:1038E00009F432C54CF48F31910509F477C48097FF
:1038F00009F428C40C941E2D8B34910509F458C585
:103900008C34910511F00C941E2D0E94B1E50C949D
:103910006F2D8C36910509F4E4C50CF047C0853550
:10392000910509F469C74CF58235910509F426C75C
:10393000D4F48135910511F00C941E2D0E94DBE525
:103940000E9481BB109243131092421368EE73E001
:1039500080E090E00E94058860E08CEE93E00E9499
:1039600092880C946F2D8335910509F40BC784352B
:10397000910509F40CC70C941E2D8936910509F4A4
:10398000E1C554F48C35910509F451C78836910589
:1039900009F416C50C941E2D8A36910509F436C615
:1039A0008B36910509F450C60C941E2D8137910574
:1039B00009F49BC59CF48E36910509F42CC50CF4D2
:1039C00003C68F36910509F439C58037910511F08A
:1039D0000C941E2D89ED93E00E94805F8537910540
:1039E00011F40C943C2564F48237910509F4A8C7BE
:1039F0008337910511F00C941E2DEBEEF4E0E0C737
:103A00008637910511F40C944D258737910511F0F7
:103A10000C941E2D0F94972F0C946F2D833631E04C
:103A2000930709F429C10CF088C08C3C910511F46E
:103A30000C949E260CF041C08B39910509F49DC56C
:103A4000DCF48D37910509F411C65CF489379105D2
:103A500011F00C941E2D1092750A1092740A0C9499
:103A60006F2D8C38910509F4B3C58139910511F496
:103A70000C949E250C941E2D883C910511F40C94F9
:103A800016264CF48E3B910511F00C941E2D0F94CC
:103A9000C6230C946F2D893C910511F40C94662675
:103AA0008B3C910511F00C941E2DBBE5EB2EB2E082
:103AB000FB2E06ED12E10C948F26823E910511F447
:103AC0000C94FC27CCF4833D910511F40C947E27D3
:103AD0003CF48D3C910511F40C9413270C941E2D8D
:103AE0008C3D910511F40C9481278D3D910511F4C5
:103AF0000C948E270C941E2D8E32F1E09F0711F44A
:103B00000C94EE286CF48C3231E0930711F40C9491
:103B100025288D32914011F40C944E280C941E2DC2
:103B20008F32F1E09F0711F40C94422980339140C9
:103B300011F40C9445290C941E2D8C3032E093071F
:103B400011F40C94A42A0CF049C0843AF1E09F07C8
:103B500011F40C94E429FCF4813931E0930711F459
:103B60000C94D8294CF48039914011F00C941E2DFE
:103B70000E9443BB0C946F2D823921E0920711F40F
:103B80000C94DE298A39914011F00C941E2D0E946C
:103B9000A5A50C946F2D863FE1E09E0711F40C94CF
:103BA000712A7CF4843F21E0920711F40C946E2A70
:103BB000853F914011F00C941E2D0F947D010C94C3
:103BC0006F2D873FE1E09E0711F40C94742A883F23
:103BD000914011F40C94802A0C941E2D8D3B22E010
:103BE000920711F40C94CE2B3CF58B35E2E09E0746
:103BF00011F40C94AC2A4CF48835924011F00C94DA
:103C00001E2D0E94B4A30C946F2D893932E09307C6
:103C100011F40C94352B8A39924011F00C941E2D1E
:103C20002BE5E22E22E0F22E0AE11CE036E2C32E62
:103C30003CE0D32E0C94C62B8B38F3E09F0711F495
:103C40000C946F2D6CF48E3B32E0930711F40C94BE
:103C5000D12B8335934011F40C94A42C0C941E2D7D
:103C6000803AF3E09F0709F4ACC2873E934011F419
:103C70000C94092D0C941E2DE8E7FBE20C94C52949
:103C8000E3E0F3E087C0A0909813B090991380E52B
:103C90000E94765B882359F00E94BA5A6B017C011E
:103CA00011E0672B682B692B31F410E004C010E0A1
:103CB000C12CD12C760183E50E94765B882311F418
:103CC0000C940A2E0E94FA5A20E030E04AE754E4AD
:103CD0000F9434450F94424A6B017C0111110BC0C3
:103CE000672B682B692B39F4A114B10421F0F5017D
:103CF0008081811102C010E001C011E00E9443BB2D
:103D0000112329F061E0C5010E94CE8805C060E062
:103D100088ED92E00E94928883E08093EF0C81E02E
:103D20008093EE0CC114D104E104F104B1F00F94BE
:103D3000D20EC60ED71EE81EF91E0F94D20EDC015D
:103D4000CB018C199D09AE09BF09B7FF0EC0809148
:103D5000EE0C81110C940F2E08C08091EE0C88237C
:103D600021F080E00E94D05FF8CF0F948B15109265
:103D7000EE0C0C946F2D60E08BEE92E00E94928826
:103D80005F988A988091080181708093060112984B
:103D90000C946F2D84918F010F5F1F4F882321F0AA
:103DA0000E949C5BF801F6CF1092C7128AE790E15F
:103DB0000E94E86F8BE1EAE7F0E1DE0115960190E1
:103DC0000D928A95E1F780917810909179109C83FB
:103DD0008B8385E093E09A83898340E050E0BE01C5
:103DE0006F5F7F4F80E090E00F942503CE01019636
:103DF0000E94605FE4EFF2E084918F010F5F1F4F3C
:103E0000882311F40C946F2D0E949C5BF801F4CF71
:103E10000E941FF70C946F2D109222101092231005
:103E20000C946F2DE0919813F09199138081882361
:103E300029F0803209F410823196F8CF40E061E039
:103E400080919813909199130E943BF50C946F2DDB
:103E500080E090E0A0E2B1E489839A83AB83BC83E5
:103E600018A219A21AA21BA21CA21DA21EA21FA266
:103E700080918C0F882359F020E0AE014F5F5F4F97
:103E8000BE01605E7F4FCE0184960F94B61F809175
:103E90002310882319F081E0809322100E948FE57F
:103EA0000C946F2D109222100E94B1E584E193E0F2
:103EB00090934513809344130E941C5A0C946F2DC9
:103EC00080912310882311F40C946F2D83E50E94B8
:103ED000765B81110C94142E0C946F2D83E40E9458
:103EE0002D5B882309F450C0E6E4F3E084918F0150
:103EF0000F5F1F4F882321F00E949C5BF801F6CFD3
:103F000080911512811103C0E9E1F3E012C0BE01F6
:103F10006F5F7F4F82E192E10E94B06E8E010F5F72
:103F20001F4FF80181918F01882349F10E949C5B0A
:103F3000F8CF84918F010F5F1F4F882301F10E94FA
:103F40009C5BF801F6CF74ECC72E73E0D72EE12C02
:103F5000F12C20E08091F70490E00E2C02C09595A2
:103F600087950A94E2F780FD99C29FEFE91AF90A52
:103F7000E2E0CE0ED11CF5E0EF16F10459F78AE02D
:103F80000E949C5B0C946F2D80912310882339F044
:103F900080912210882319F0E3E2F3E003C0E5E307
:103FA000F3E028C084918F010F5F1F4F882321F019
:103FB0000E949C5BF801F6CF6091C3127091C4120D
:103FC0008091C5129091C6124AE00E94405E8FE235
:103FD0000E949C5B6091BF127091C0128091C112CF
:103FE0009091C2124AE00E94405E8AE00E949C5B6F
:103FF0000C946F2D84918F010F5F1F4F882311F454
:104000000C946F2D0E949C5BF801F4CF40E060E0BF
:1040100080919813909199130E943BF50C946F2D09
:1040200080912310882311F40C946F2D82E192E18A
:104030000F94601D82E192E10E948B6E109221101C
:104040001092201080912310882311F40C946F2D6E
:1040500000919813109199130F941603B801CE0193
:1040600080960F942C058C01892B11F40C946F2DE4
:1040700068A179A16115710511F06C5F7F4F1982FC
:104080001C8222E0A801CE0101960E944D7681118A
:1040900002C0F12C14C0CE0101960F948402882333
:1040A000C1F361E0CE0101960E94946E009789F3FE
:1040B00025EEFC0120831C820F94091BF82ECE01F3
:1040C00001960E94825BF11003C0E3E6F3E022C098
:1040D000E5E5F3E084917F012FEFE21AF20A8823ED
:1040E00021F00E949C5BF701F5CFF80181918F01CF
:1040F000882319F00E949C5BF8CF8AE00E949C5BA9
:104100001092C3121092C4121092C5121092C612CD
:104110000C946F2D84917F012FEFE21AF20A88230D
:1041200021F00E949C5BF701F5CFF80181918F018E
:10413000882319F00E949C5BF8CF8EE20E949C5B62
:104140000C946F2D8091221081110E9443BB8091AD
:104150002310882311F40C946F2D80E50E94765B68
:10416000882319F00E94EB5A03C080E50E942D5B62
:10417000182F482F61E080919813909199130E9415
:104180003BF583E50E94765B882381F00E94CA5A42
:10419000AB01BC014093C3125093C4126093C5128B
:1041A0007093C61282E192E10F94921D80912310C8
:1041B000882319F081E08093221011110C946F2D47
:1041C0006DCE809198139091991321E02093211046
:1041D00040E060E00E943BF50C946F2D0E9440E5AA
:1041E0007B018C0120E831E541E050E00F94BD48AF
:1041F000C9016DE671E00F941B4C4B015C01C801D5
:10420000B70120E13EE040E050E00F94BD48CA0114
:10421000B90128E130E040E050E00F94BD48762E2F
:10422000672EC62ED72EECE32E2E312C412C512C8E
:10423000C801B701A20191010F94BD48F62EE72EE7
:10424000CA01B901A20191010F94BD48CB018E01B1
:104250000F5F1F4F8114910499F0EF92FF927F93AB
:104260006F936F927F92BF92AF929F928F9283EAE9
:1042700093E09F938F931F930F930F94694413C000
:10428000A114B104B1F0EF92FF927F936F936F92FC
:104290007F92BF92AF9283E993E09F938F931F9396
:1042A0000F930F9469440FB6F894DEBF0FBECDBFD5
:1042B00030C0CD2879F0EF92FF927F936F936F9289
:1042C0007F9287E893E09F938F931F930F930F94B0
:1042D0006944E9CF892B69F0EF92FF927F936F9346
:1042E0008FE793E09F938F931F930F930F946944ED
:1042F000DACFEF92FF928BE793E09F938F931F9318
:104300000F930F9469440F900F900F900F900F90A0
:104310000F9060E0C8010E94CE88E2E5FFE2849140
:104320007F013FEFE31AF30A882321F00E949C5B90
:10433000F701F5CFB80187EB93E00E949EC38AE0B6
:104340000E949C5B0C946F2D83E50E94765B882312
:1043500011F40C946F2D0E94DA5AE82E80E50E9429
:10436000765B882339F00E94DA5A182F87FF03C042
:104370000C946F2D1DE089E40E94765B882341F048
:104380000E94EB5A81110C94812EE6E0F6E00BC0FE
:1043900089E40E942D5BF6CF319686E0E333F8077F
:1043A00011F40C94812E84911813F6CF0C94552E91
:1043B0000E948FE50C946F2D0E94C6E50C946F2D22
:1043C00088E690E00E94D75581110C946F2D809162
:1043D000F70483FF02C00C946F2D83E50E94765B87
:1043E0008823A9F00E94FA5A0F943D4ACB010E94FB
:1043F00029880E94FA5A20E030E04AEA52E40F94F9
:10440000CF44181624F00E94C6E50F948B150E9425
:10441000B9C30C946F2D8EE40E94765B882311F44F
:104420000C946F2D0E94CA5A60937F0F7093800F77
:104430008093810F9093820F0C946F2D83E50E94DF
:104440002D5B882359F083E50E94765B882319F061
:104450000E94DA5A01C080E08093F704E2E5FFE2AF
:1044600084918F010F5F1F4F811103C0E2EDF3E0D4
:1044700004C00E949C5BF801F3CF84918F010F5F11
:104480001F4F882321F00E949C5BF801F6CF80919A
:10449000F704811158CDEEECF3E018C0BB24B394BF
:1044A000B20E222319F08CE20E949C5BF6018591EA
:1044B0009491FC0184918F010F5F1F4F882321F09D
:1044C0000E949C5BF801F6CF2B2D4FCD84918F017C
:1044D0000F5F1F4F882309F452CD0E949C5BF801A7
:1044E000F5CF10921B020C946F2D83E50E94765B32
:1044F000811103C0E2E5FFE20DC00E94DA5A8D335C
:1045000020F4809300020C946F2D8CE380930002C2
:104510000C946F2D84918F010F5F1F4F882321F022
:104520000E949C5BF801F6CF4091000250E060E0F1
:1045300070E082EE93E00E944BC38AE00E949C5B95
:104540000C946F2D89E690E00E94D755811111C01F
:10455000E9EEF3E084918F010F5F1F4F882321F074
:104560000E949C5BF801F6CF0E9485CC8AE00E94F5
:104570009C5B1092EF0C0C94962E83E50E94765B68
:10458000882311F40C946F2D0E94DA5A182F8D3362
:1045900008F01CE310936B040F94D20E6B017C01A6
:1045A000212F30E0A8EEB3E00F94E948C60ED71EE5
:1045B000E81EF91EC0926704D0926804E092690474
:1045C000F0926A040C946F2D0F94A0250C946F2D1B
:1045D0008091F70483FF02C00C946F2D83E50E9445
:1045E000765B882311F40C946F2D0E94FA5A0F9475
:1045F0003D4A6936710514F069E670E07093411325
:10460000609340130E9481E30C946F2D80E50E941B
:10461000765B811106C083E50E94765B882361F09A
:1046200006C00E94DA5A81110C946F2DF4CF0E94BB
:10463000CA5A6F3F710510F06FEF70E0709343132B
:10464000609342130C946F2D80E50E94765B81117C
:1046500006C010924313109242130C946F2D0E94C7
:10466000CA5A672B11F00C946F2DF3CF8CE40E9483
:104670002D5B882361F00E94FA5A6B017C0120E0D7
:1046800030E0A9010F946D4B87FF0BC006C0C12C11
:10469000D12C60E8E62E61ECF62EF7FAF094F7F8EC
:1046A000F094F7FAF094F7F8F094CCA2DDA2EEA221
:1046B000FFA280E090E0A4EDB2EC89839A83AB8303
:1046C000BC8380E090E0A4EDB2E48D839E83AF8351
:1046D000B88780E090E0A0EFB1E489879A87AB8744
:1046E000BC8788E50E94765B882379F088E50E9484
:1046F000765B882319F00E94FA5A03C060E070E0EC
:10470000CB0169837A838B839C8389E50E94765BE6
:10471000882379F089E50E94765B882319F00E944E
:10472000FA5A03C060E070E0CB016D837E838F8313
:1047300098878AE50E94765B882379F08AE50E9453
:10474000765B882319F00E94FA5A03C060E070E09B
:10475000CB0169877A878B879C8718A219A21AA236
:104760001BA220E0AE01405E5F4FBE016F5F7F4F36
:10477000CE0184960F94AF290C946F2D10924F03A5
:104780000C946F2D81E080934F030C946F2D83E583
:104790000E94765B8823A1F00E94FA5A20E030E064
:1047A0004AE754E40F9434450F94424A60935B0403
:1047B00070935C0480935D0490935E040C946F2D61
:1047C00088E50E942D5B81110C94252E89E50E94BD
:1047D0002D5B81110C94252E8AE50E942D5B8111A1
:1047E0000C94252E85E40E942D5B81110C94252EBE
:1047F0000E9481BB0C946F2D83E50E942D5B882362
:1048000011F40C946F2D0E94FA5A20E030E04AE730
:1048100054E40F9434450F94424A609363047093B8
:10482000640480936504909366040C946F2D4BE5AB
:10483000C42E42E0D42E56E4E52E5DE0F52E10E0C5
:10484000F60181916F010E942D5B882309F46DC0F0
:10485000133009F063C00E94FA5A4B015C0120E05A
:1048600030E040EA51E40F94CF4487FF4EC0A501E9
:1048700094016091520D7091530D8091540D90915F
:10488000550D0F94D5492B013C019B01AC01609162
:104890000A1370910B1380910C1390910D130F94C8
:1048A000344560930A1370930B1380930C13909309
:1048B0000D13A30192016091E2127091E3128091B5
:1048C000E4129091E5120F9434456093E2127093D4
:1048D000E3128093E4129093E51260910D057091BC
:1048E0000E0580910F05909110050F94D344A301FC
:1048F00092010F9434450F94424A60930D057093D2
:104900000E0580930F05909310058092520D9092A2
:10491000530DA092540DB092550D07C00E94FA5A43
:10492000F70160837183828393831F5FF4E0EF0E4E
:10493000F11C143009F084CF0E9444C40C946F2DF4
:104940000E9443BB83E50E94765B882311F40C949C
:10495000181C0E94CA5A6230710511F00C94181C80
:104960000E9461638BE50E949C5B6091BA04709128
:10497000BB048091BC049091BD0442E00E94C55EDE
:104980004091BE045091BF046091C0047091C10475
:1049900089E094E00E9468C34091C2045091C3042E
:1049A0006091C4047091C50486E094E00E9468C3DD
:1049B0008DE50E949C5B8AE00E949C5B0C946F2DAD
:1049C00084918F010F5F1F4F882321F00E949C5B11
:1049D000F801F6CF60E08BED94E00E9436AC61E028
:1049E00084ED94E00E9436AC61E089EC94E00E9492
:1049F00036AC61E089EB94E00E9436AC60E080EB7D
:104A000094E00E9436AC61E086EA94E00E9436AC05
:104A100061E08CE994E00E9436AC61E084E994E0C6
:104A20000E9436AC61E086E894E00E9436AC60E01B
:104A300088E794E00E9436AC60E089E694E00E944A
:104A400036AC60E08BE594E00E9436AC60E085E433
:104A500094E00E9436AC60E084E394E00E9436ACBF
:104A600060E08FE194E00E9436AC61E08CE094E07D
:104A70000E9436AC0C946F2D8091981390919913ED
:104A8000FC012081222329F060E00E94CE880C9452
:104A90006F2D0F948B150C946F2D0091981310911E
:104AA000991383E0D12C40E08150E1F0F80190812E
:104AB000292F2B7F2134C1F721812133A9F791348C
:104AC00021F0953421F441E002C0DD24D394980113
:104AD0002E5F3F4F89012F5F3F4FF8019081903249
:104AE000C9F3E2CF442369F0E2E5FFE284917F015C
:104AF0002FEFE21AF20A882321F00E949C5BF70153
:104B0000F5CFDD2069F0E2ECF5E084917F013FEF25
:104B1000E31AF30A882321F00E949C5BF701F5CF8A
:104B2000F80181918F01882309F429CA0E949C5BB6
:104B3000F7CF4093750A4093740AD1C783E50E946A
:104B4000765B882319F00E94CA5A02C060E070E0C8
:104B50008B01112702301105D4F0E8E7FBE28491C4
:104B60008F010F5F1F4F811103C0E6ECF5E004C019
:104B70000E949C5BF801F3CF84918F010F5F1F4F60
:104B8000882309F4ACC70E949C5BF801F5CF88E448
:104B90000E94765B8823A9F00E94CA5A6A3A71057E
:104BA0003CF06530F1E07F072CF064E071E002C07A
:104BB0006AEA70E0F801EE0FFF1FE45BF34F7183C8
:104BC000608386E40E94765B8823A9F00E94CA5A1B
:104BD000F801EE0FFF1FE05BF34F718360836F3FBF
:104BE000710519F014F06FEF70E077FF02C060E01C
:104BF00070E07183608382E40E94765B882309F40D
:104C00006EC70E94CA5A6530710534F06A36710564
:104C10002CF069E670E002C065E070E0000F111F43
:104C2000F801E85BF34F7183608359C788EC90E02B
:104C30000E94D755811153C784E40E942D5B8823BD
:104C400009F441C00E94FA5A6B017C0111E020E096
:104C500030E0A9010F94CF44811101C010E01093FE
:104C60003A0C20E030E0A901C701B6010F94CF440F
:104C7000882349F10E94FA5AE0913A0A24E0E29F1F
:104C8000F0011124EA5CF34F608371838283938384
:104C900020E030E0A9016091360C7091370C8091D2
:104CA000380C9091390C0F94CF4481110CC080E0E6
:104CB00090E0A0EEBFE38093360C9093370CA09366
:104CC000380CB093390C0F94842A09C71BE5E12EE8
:104CD00012E0F12E06EE12E186EFC82E82E1D82E08
:104CE000F70181917F010E942D5B882349F00E948A
:104CF000FA5A0F94424AF801608371838283938346
:104D00000C5F1F4FC016D10659F70E94E9C3E7C6D2
:104D10000C5F1F4FF2E1063E1F0709F4E0C6F701E2
:104D200081917F010E942D5B882391F30E94FA5AA2
:104D3000F8016083718382839383EACF83E50E94C5
:104D4000765B8823A1F00E94FA5A6093FA1270935E
:104D5000FB128093FC129093FD126093F6127093F5
:104D6000F7128093F8129093F91210E001C011E04D
:104D700080E50E94765B882359F00E94FA5A60937E
:104D8000FA127093FB128093FC129093FD1210E0C4
:104D900082E50E94765B882359F00E94FA5A60935C
:104DA000EA0C7093EB0C8093EC0C9093ED0C10E0FC
:104DB00084E50E94765B882359F00E94FA5A60933A
:104DC000F6127093F7128093F8129093F91287C637
:104DD000112309F484C64091FA125091FB1260919C
:104DE000FC127091FD128EEE95E00E9468C3409116
:104DF000EA0C5091EB0C6091EC0C7091ED0C8BEE89
:104E000095E00E9468C34091F6125091F7126091AC
:104E1000F8127091F91288EE95E00E9468C38AE05A
:104E20000E949C5B5CC681E50E942D5B882351F04B
:104E30000E94BA5A6093880F7093890F80938A0FEB
:104E400090938B0F83E50E942D5B882351F00E9485
:104E5000FA5A6093D2127093D3128093D412909323
:104E6000D51284E50E942D5B882351F00E94FA5AE6
:104E70006093CE127093CF128093D0129093D11280
:104E800088E50E942D5B882351F00E94FA5A6093B6
:104E9000FE127093FF12809300139093011389E523
:104EA0000E942D5B882351F00E94FA5A60930213EE
:104EB0007093031380930413909305138AE50E9463
:104EC0002D5B882351F00E94FA5A60930613709369
:104ED0000713809308139093091385E40E942D5BB8
:104EE000882309F4FCC50E94FA5A60930A13709350
:104EF0000B1380930C1390930D13F1C50E9458ABC4
:104F0000EEC583E50E94765B882309F4E8C50E941C
:104F1000CA5A7093550260935402E1C58DED90E03A
:104F20000E94D7558111DBC583E50E94765B811114
:104F300003C0E2E5FFE23AC000913A0A10E00E94A5
:104F4000CA5A000F111FF801EE5AFD4F718360839A
:104F500080913A0A90E08C01000F111F000F111F81
:104F60009801225B3D4F7901880F991FFC01EE5A91
:104F7000FD4F60817181072E000C880B990B0F94F7
:104F8000D5442AE037ED43E25CE30F943445F80161
:104F9000E85EFC4E20813181428153810F9434457B
:104FA000F701608371838283938399C584918F0114
:104FB0000F5F1F4F882321F00E949C5BF801F6CF02
:104FC00085E40E949C5B80913A0A805D0E949C5B14
:104FD000E0913A0AF0E0EE0FFF1FEE5AFD4F6081BC
:104FE00071818EEF95E00E9485C385E20E949C5BF3
:104FF0008AE00E949C5B73C580E50E942D5B88233C
:1050000009F46DC50E94CA5A6B017C0183E50E94B8
:10501000765B882321F00E94CA5A8B0102C00FEFF1
:105020001FEFC8010196039708F059C5D7FC57C573
:105030008C2DE6E0F6E09491891709F436C6319696
:1050400026E0E333F207B9F733C683E50E94765BC7
:10505000882319F00E94CA5A02C064E071E079A363
:1050600068A380E50E94765B882339F00E94CA5AC3
:10507000693833E1730730F402C068EE73E07A8375
:10508000698304C088E893E19A838983BE01605EE6
:105090007F4FCE0101960E9462F821C585E40E94EF
:1050A000765B811110C080E50E942D5B882391F012
:1050B0000E94FA5A60933B0C70933C0C80933D0C19
:1050C00090933E0C07C00E94DA5A882361F3E8E708
:1050D000FBE271C089E40E942D5B882381F00E946D
:1050E000FA5A2CEA35EC47E25EE30F9434456093BC
:1050F000430C7093440C8093450C9093460C84E4CD
:105100000E942D5B882381F00E94FA5A2CEA35EC2C
:1051100047E25EE30F94D54960933F0C7093400CD7
:105120008093410C9093420CE2E5FFE284918F0161
:105130000F5F1F4F882321F00E949C5BF801F6CF80
:1051400040913B0C50913C0C60913D0C70913E0C99
:105150008BE396E00E9468C32CEA35EC47E25EE3FD
:105160006091430C7091440C8091450C9091460CD9
:105170000F94D549AB01BC0187E396E00E9468C358
:105180002CEA35EC47E25EE360913F0C7091400CF5
:105190008091410C9091420C0F943445AB01BC01BD
:1051A00083E396E00E9468C38AE00E949C5B97C4F8
:1051B0000E949C5BF80184918F010F5F1F4F81114A
:1051C000F7CFEFE3F6E084918F010F5F1F4F882345
:1051D00009F485C40E949C5BF801F5CF83E50E9429
:1051E0002D5B182F882371F00E94FA5A0F943D4AC4
:1051F00070935A026093590221E0672B09F020E076
:1052000020936D1380E50E942D5B882359F0209137
:10521000590230915A02232B11F00E94EB5A8093CD
:105220006D135DC411115BC4E2E5FFE284918F014F
:105230000F5F1F4F882321F00E949C5BF801F6CF7F
:1052400080916D13882319F069E173E002C06CE16D
:1052500073E086E696E00E949EC3609159027091C9
:105260005A0285E596E00E9485C3E1E5F6E0849167
:105270008F010F5F1F4F882309F431C40E949C5B8C
:10528000F801F5CF0E94DBA52AC480E50E942D5BC2
:10529000882351F00E94FA5A6093730C7093740C37
:1052A0008093750C9093760C89E40E942D5B882383
:1052B00081F00E94FA5A2CEA35EC47E25EE30F9443
:1052C000344560936F0C7093700C8093710C9093C5
:1052D000720C84E40E942D5B882381F00E94FA5AAC
:1052E0002CEA35EC47E25EE30F94D54960936B0CF2
:1052F00070936C0C80936D0C90936E0CE2E5FFE262
:1053000084918F010F5F1F4F882321F00E949C5BC7
:10531000F801F6CF4091730C5091740C6091750CAC
:105320007091760C81E896E00E9468C32CEA35EC17
:1053300047E25EE360916F0C7091700C8091710C8C
:105340009091720C0F94D549AB01BC018DE796E0AA
:105350000E9468C32CEA35EC47E25EE360916B0C77
:1053600070916C0C80916D0C90916E0C0F94344583
:10537000AB01BC0189E796E00E9468C38AE00E9405
:105380009C5BADC30E949C5BF80184918F010F5F11
:105390001F4F8111F7CFE5E8F6E084918F010F5F91
:1053A0001F4F882309F49BC30E949C5BF801F5CF33
:1053B00081E00E947E510E946DAC91C380E00E940A
:1053C0007E510E946DAC8BC383E50E942D5B8823C8
:1053D00049F00E94EB5A182F811106C080E00E940C
:1053E000964902C01091010C8091560D9091570D75
:1053F000A091580DB091590D89839A83AB83BC83DA
:1054000080915A0D90915B0DA0915C0DB0915D0D56
:105410008D839E83AF83B88780915E0D90915F0DE1
:10542000A091600DB091610D89879A87AB87BC8789
:1054300086E50E942D5B882321F081EC96E00F9495
:10544000A23C812F0E949649111103C0E2E5FFE2C0
:105450001DC08091010C8111F9CFE8E7FBE2849136
:105460008F010F5F1F4F811103C0E2EAF6E004C015
:105470000E949C5BF801F3CF84918F010F5F1F4F57
:10548000882321F30E949C5BF801F6CF84918F0161
:105490000F5F1F4F882321F00E949C5BF801F6CF1D
:1054A0008091010C882319F060E273E002C064E28D
:1054B00073E084E996E00E949EC38AE00E949C5BB0
:1054C0004CE050E066E57DE0CE0101960F94784C0B
:1054D000892B09F404C30E946DAC01C30E947F7D37
:1054E000FEC20E94C5FFFBC283E50E942D5B88239C
:1054F00021F00E94EB5A91E089270E946EFAEFC2D8
:1055000081E08093830F0E945D771092830F882340
:1055100009F4E5C2E2E5FFE284918F010F5F1F4FBE
:10552000811103C0EEEDF6E004C00E949C5BF8011F
:10553000F3CF84918F010F5F1F4F882309F4CFC2EF
:105540000E949C5BF801F5CF80912210882309F41A
:10555000C6C240932510C3C28BE592E00E94D75586
:105560008111BDC285E50E942D5B8823D9F1009190
:105570003A0A10E00E94FA5A6B017C0120E030E008
:10558000A9010F946D4B87FF04C0F7FAF094F7F868
:10559000F094000F111F000F111FF801EE5CF34F84
:1055A000C082D182E282F38200913A0A84E0089FAD
:1055B000800111240E5C134F20E030E046E154E4FA
:1055C000F80160817181828193810F946D4B18166F
:1055D0004CF480E090E0A6E1B4E4F801808391838C
:1055E000A283B3838CE40E942D5B882309F477C2E5
:1055F00000913A0A10E00E94FA5A6B017C0120E007
:1056000030E0A9010F946D4B87FF04C0F7FAF094C6
:10561000F7F8F094000F111F000F111FF801E25D61
:10562000F34FC082D182E282F38200913A0AF4E021
:105630000F9F80011124025D134F20E030E046E10E
:1056400054E4F80160817181828193810F946D4BE4
:1056500018160CF044C280E090E0A6E1B4E4F80132
:1056600080839183A283B3833AC288E40E942D5B36
:10567000882351F00E94FA5A6093260C7093270CED
:105680008093280C9093290C8CE40E942D5B882336
:1056900051F00E94FA5A6093060C7093070C8093A5
:1056A000080C9093090C82E50E942D5B882351F031
:1056B0000E94FA5A6093160C7093170C8093180C82
:1056C0009093190C83E50E942D5B882351F00E9472
:1056D000FA5A6093840F7093850F8093860F90938E
:1056E000870F82E40E942D5B882351F00E94FA5AB2
:1056F0006093020C7093030C8093040C9093050C40
:1057000088E50E942D5B882351F00E94FA5A60932D
:105710000A0C70930B0C80930C0C90930D0C89E584
:105720000E942D5B882351F00E94FA5A60930E0C60
:1057300070930F0C8093100C9093110C8AE50E94CB
:105740002D5B882351F00E94FA5A6093120C7093DB
:10575000130C8093140C9093150C0E94016DBFC123
:105760000E94FA5A20E030E0A9010F94CF441816A5
:105770003CF00E94FA5AF80160837183828393831C
:105780000C5F1F4FC016D10609F4A9C1F701819122
:105790007F010E942D5B882399F3E2CF0E9472A2C1
:1057A0009EC141E061E081E00E94E149811107C0B2
:1057B000812C912C90EFA92E91E4B92E03C0812C5D
:1057C000912C54018EEB92E00E94D755811187C134
:1057D0008AE50E94765B882369F08AE50E94765B01
:1057E000882329F00E94FA5A4B015C0103C0812CE6
:1057F000912C540140913A0A62E081E00E94DFA1BD
:1058000020E030E0A901C501B4010F946D4B1816DA
:105810007CF580E090E0A8ECB2E489839A83AB83C6
:10582000BC8320915E0D30915F0D4091600D5091D1
:10583000610DC501B4010F94F9486B017C0120E0B2
:1058400030E040EA53E40F94CF4487FD06C0C12CFA
:10585000D12C80EAE82E83E4F82EC8A2D9A2EAA2CD
:10586000FBA2BE016F5F7F4FCE0180960E945F5109
:1058700085E50E942D5B882329F00E94FA5A6B016E
:105880007C010CC0E0913A0A24E0E29FF00111246F
:10589000EE5CF34FC080D180E280F38020E030E006
:1058A000A901C701B6010F946D4B87FF04C0F7FA39
:1058B000F094F7F8F094F7FAF094F7F8F094C982BE
:1058C000DA82EB82FC8242E061E0CE0101960F9425
:1058D0001E2920E030E0A901C501B4010F946D4BF1
:1058E00018165CF580E090E0A8ECB2E489839A8316
:1058F000AB83BC83A501940160915E0D70915F0D37
:105900008091600D9091610D0F94F8486B017C01BE
:1059100020E030E0A9010F946D4B18161CF0C12C4B
:10592000D12C7601C8A2D9A2EAA2FBA2BE016F5F68
:105930007F4FCE0180960E945F514091F00C60E055
:1059400087E00E94DFA1CBC08AE50E94765B8111CF
:1059500003C0E2E5FFE23BC00E94FA5A6B017C0102
:1059600020E030E040EF51EC0F946D4B87FD0AC012
:1059700020E030E040EF51E4C701B6010F94CF447E
:1059800018161CF4E8E7FBE20CC0C0922A0CD09277
:105990002B0CE0922C0CF0922D0CA1C00E949C5B71
:1059A000F80184918F010F5F1F4F8111F7CFE9EE4E
:1059B000F6E084918F010F5F1F4F882309F48FC099
:1059C0000E949C5BF801F5CF0E949C5BF8018491DA
:1059D0008F010F5F1F4F8111F7CFE9E0F7E084914E
:1059E0008F010F5F1F4F882321F00E949C5BF801FD
:1059F000F6CF40912A0C50912B0C60912C0C709199
:105A00002D0C86E097E00E9468C38AE00E949C5BB0
:105A100066C081E080932A021092350D83E50E94D2
:105A2000765B882339F00E94EB5A811158C00E949E
:105A3000116E55C083E50E942D5BF7CF0F94872030
:105A40004EC0F0909A130E9443BB1091010C80E06D
:105A50000E949649FF2029F1E2E5FFE284918F013F
:105A60000F5F1F4F882321F00E949C5BF801F6CF47
:105A700084E50E949C5B6F2D70E080E090E04AE03E
:105A80000E94405E80E20E949C5BEAE2F7E0849123
:105A90008F010F5F1F4F882311F10E949C5BF8015B
:105AA000F6CF1092F00C812F0E949649E2E5FFE2BA
:105AB00084918F010F5F1F4F882321F00E949C5B10
:105AC000F801F6CF6091F00C70E088E197E00E9459
:105AD00085C38AE00E949C5B02C00F9487201092CD
:105AE000EF0C0E94F46D22C10E9457480E94C567C6
:105AF000F6CF80E00E9496490E941E5185E40E94E4
:105B0000765B882321F00E94EB5A182F04C085E4AD
:105B10000E942D5B11E086E50E94765B882321F0D0
:105B20000E94CA5A262F01C021E001E0412FBE0188
:105B30006F5F7F4FCE0180960E941F526B017C01E8
:105B40009B01AC010F94F34B81115FC088A099A019
:105B5000AAA0BBA020E030E0A901C501B4010F94C8
:105B6000CF4487FF05C027E137EB41E558EB04C080
:105B700027E137EB41E558E3C501B4010F94F9483B
:105B8000AB01BC0180ED92E00E9468C389809A80DD
:105B9000AB80BC8020E030E0A901C501B4010F94C6
:105BA000CF4487FF05C027E137EB41E558EB04C040
:105BB00027E137EB41E558E3C501B4010F94F948FB
:105BC000AB01BC018BEC92E00E9468C320E030E0A6
:105BD000A901C701B6010F94CF4487FF05C027E193
:105BE00037EB41E558EB04C027E137EB41E558E3DB
:105BF000C701B6010F94F948AB01BC0186EC92E0F5
:105C00000E9468C38AE00E949C5B0E9405510E942A
:105C10006DAC65CF11110C947B1E0C94741E80E04A
:105C20000E94D05F0C949D1E0E94CA5AAB01BC0119
:105C30004093C3125093C4126093C5127093C6125E
:105C400082E192E10F94921D4ACF0E9443BB88E506
:105C50000E942D5B882331F05F9A8091760A8E7FB7
:105C60008093760A89E50E942D5B882331F08A9A19
:105C70008091760A8D7F8093760A8AE50E942D5B5B
:105C8000882359F0809108018095817080930601E6
:105C90008091760A8B7F8093760A85E40E942D5B43
:105CA000882309F41CCF129A1ACF0F946D4017CF96
:105CB0000E9443BBBC2C60E08C2D0F94960D0F3FCF
:105CC0003FEF130759F48C2D0E9434CD31E020E0D2
:105CD000892B09F030E0032F122F05C00130110588
:105CE00069F401E010E08B2D0E9434CD80179107FC
:105CF00009F4F5CE80E00E94D05FF5CF00E010E01F
:105D0000F2CF61E0812F0F94960D6E2D812F0E94AE
:105D10005DCDF12CB701812F0F94D20D193009F010
:105D2000DECEF0924313E0924213D9CEA7960FB67F
:105D3000F894DEBF0FBECDBFDF91CF911F910F91C1
:105D4000FF90EF90DF90CF90BF90AF909F908F909B
:105D50007F906F905F904F903F902F9008952F927B
:105D60003F924F925F926F927F928F929F92AF92EB
:105D7000BF92CF92DF92EF92FF920F931F93CF9338
:105D8000DF93CDB7DEB7C350D1400FB6F894DEBF76
:105D90000FBECDBF80E50E94765B882351F00E9444
:105DA000CA5AAE966FAFAE976B30A0F0E9E1F9E05A
:105DB00005C024E0AE962FAFAE970CC084918F0142
:105DC0000F5F1F4F882311F40C94EB450E949C5BDE
:105DD000F801F4CF84E50E942D5BC656DF4F88831F
:105DE000CA59D04083E40E94765B8823F9F00E9470
:105DF000FA5ACC54DF4F688379838A839B83C45BD0
:105E0000D04020E030E0A9010F94CF4487FF16C0B6
:105E1000E9EEF8E084918F010F5F1F4F882311F4A2
:105E20000C94EB450E949C5BF801F4CFCC54DF4FFF
:105E3000188219821A821B82C45BD04086E40E94B9
:105E4000765B882361F00E94CA5AC754DF4F68838B
:105E5000C95BD0406F31A8F0EEEBF8E006C0C75444
:105E6000DF4F1882C95BD0400CC084918F010F5F57
:105E70001F4F882311F40C94EB450E949C5BF801A2
:105E8000F4CF86E50E94765B8823B9F00E94DA5A47
:105E9000CB56DF4F8883C559D0408430A0F0E6E967
:105EA000F8E084918F010F5F1F4F882311F40C9449
:105EB000EB450E949C5BF801F4CF81E0CB56DF4FAD
:105EC0008883C559D04081E0C656DF4F9881CA59B2
:105ED000D0409827CD54DF4F9883C35BD04085E4F2
:105EE0000E942D5B082FAE96AFADAE97A13009F49E
:105EF0005EC0B1E0C655DF4FB883CA5AD040AF3F4D
:105F000011F40C94B945C655DF4F1882CA5AD040D7
:105F1000A230C9F4C656DF4FE881CA59D040E1111A
:105F20000C94C645C855DF4F1882C85AD040CD548E
:105F3000DF4FF881C35BD040C755DF4FF883C95AA4
:105F4000D04010E019C0AE96EFADAE97E33014F438
:105F50000C94B945A1E0C755DF4FA883C95AD0407A
:105F600010E0B1E0C855DF4FB883C85AD040AE96B4
:105F70002FADAE972F3F61F191E0C854DF4F98836A
:105F8000C85BD040AE96AFADAE97AA2309F1AE96EE
:105F9000BFADAE97B3300CF1CD54DF4FE881C35B9A
:105FA000D040C955DF4FE883C75AD0401BC0C85501
:105FB000DF4F1882C85AD040C755DF4F1882C95AE0
:105FC000D04010E021E0C655DF4F2883CA5AD040A8
:105FD000C854DF4F1882C85BD040C955DF4F1882C4
:105FE000C75AD040CB56DF4FF881C559D040C5566F
:105FF000DF4F1882CB59D040FF2399F020ECC456D4
:10600000DF4F2883CC59D04089E7C356DF4F8883C0
:10601000CD59D04094E4C256DF4F9883CE59D0403A
:106020000FC0C456DF4F1882CC59D040C356DF4F43
:106030001882CD59D040C256DF4F1882CE59D04079
:1060400080911A0C90911B0CA0911C0CB0911D0C0E
:10605000C452DF4F88839983AA83BB83CC5DD04031
:1060600080911E0C90911F0CA091200CB091210CDE
:10607000CC52DF4F88839983AA83BB83C45DD04011
:106080008091220C9091230CA091240CB091250CAE
:10609000C453DF4F88839983AA83BB83CC5CD040F1
:1060A0008091160C9091170CA091180CB091190CBE
:1060B000C054DF4F88839983AA83BB83C05CD040E0
:1060C0008091260C9091270CA091280CB091290C5E
:1060D000CC53DF4F88839983AA83BB83C45CD040B1
:1060E00080910A0C90910B0CA0910C0CB0910D0CAE
:1060F000C853DF4F88839983AA83BB83C85CD04091
:1061000080910E0C90910F0CA091100CB091110C7D
:10611000C852DF4F88839983AA83BB83C85DD04070
:106120008091120C9091130CA091140CB091150C4D
:10613000C053DF4F88839983AA83BB83C05DD0405F
:10614000E2E8F8E084917F019FEFE91AF90A8823D9
:1061500021F00E949C5BF701F5CFC655DF4FA88167
:10616000CA5AD040A11173C0AE96BFADAE97BB2343
:1061700009F46DC08090020C9090030CA090040C68
:10618000B090050CA2ED2A2E312CB101032C000C8D
:10619000880B990B0F94D5442BED3FE049E450E474
:1061A0000F94344520E030E044E353E40F94D549A4
:1061B0006B017C010F94A84B9B01AC01C501B4019C
:1061C0000F9434452B013C01C701B6010F94D2490D
:1061D0009B01AC01C501B4010F9434459B01AC0196
:1061E0000F943445E2966CAF7DAF8EAF9FAFE297D0
:1061F000A3019201C301B2010F9434459B01AC018C
:10620000E2966CAD7DAD8EAD9FADE2970F94F948EF
:1062100020E030E442E556E40F94CF44181674F4BD
:10622000EFE4F8E084918F010F5F1F4F882311F492
:106230000C94EB450E949C5BF801F4CFECE32E0E2E
:10624000311CFAE32F16F2E03F0609F09ECFE3E798
:10625000F8E084917F012FEFE21AF20A882321F0FF
:106260000E949C5BF701F5CFCB56DF4F8881C55963
:10627000D04081110DC0E4E4F8E084917F019FEFEC
:10628000E91AF90A882321F00E949C5BF701F5CFF7
:106290008AE00E949C5B60E083E798E00E9492881D
:1062A000C955DF4F6881C75AD040C854DF4F888135
:1062B000C85BD0400F94FD33AE96AFADAE97AA2326
:1062C00041F081E0C655DF4FF880CA5AD040F82629
:1062D00001C0F12C0E9443BB0E941E51F1100E948C
:1062E000B449AE96BFADAE97BB2349F081E0809331
:1062F000750A0E94039B8091740A8093750A00239B
:1063000039F0E1E0C254DF4FE883CE5BD04006C0F5
:10631000F2E0C254DF4FF883CE5BD040AE962FAD93
:10632000AE9728303CF082E0C154DF4F8883CF5BCA
:10633000D04005C0C154DF4F1882CF5BD04011233D
:1063400039F092E0C052DF4F9883C05ED04006C063
:10635000A1E0C052DF4FA883C05ED040AE96BFAD73
:10636000AE97B23039F4E2E0CF51DF4FE883C15E3F
:10637000D04006C0F1E0CF51DF4FF883C15ED0407E
:10638000C556DF4FE880CB59D040C456DF4FF88068
:10639000CC59D040C356DF4F0881CD59D040C256AA
:1063A000DF4F1881CE59D040C156DF4FE882CF5918
:1063B000D040C056DF4FF882C05AD040CF55DF4F93
:1063C0000883C15AD040CE55DF4F1883C25AD040FF
:1063D000CC56DF4F1882C459D040CE014D96AB96B3
:1063E0009FAF8EAFAB97DE01D996AD96BFAFAEAF84
:1063F000AD97C154DF4FE881CF5BD0400E2E000C2B
:10640000FF0BC250DF4FF983E883CE5FD0404C973B
:106410001C01AE968FADAE97082E000C990BAA0BFF
:10642000BB0BC050DF4F88839983AA83BB83C050C6
:10643000D1408CE1AB96AEADBFADAB971D928A95C6
:10644000E9F720E030EC49E754E4B701C8010F94C4
:10645000CF44882399F19701A801C556DF4F688181
:10646000CB59D040C456DF4F7881CC59D040C35669
:10647000DF4F8881CD59D040C256DF4F9881CE5929
:10648000D0400F94F94820E030E040E05FE30F9403
:106490003445CA56DF4F6883C659D040C956DF4FCE
:1064A0007883C759D040C856DF4F8883C859D04039
:1064B000C756DF4F9883C959D04028C0C556DF4F13
:1064C000B881CB59D040CA56DF4FB883C659D040A7
:1064D000C456DF4FE881CC59D040C956DF4FE8831E
:1064E000C759D040C356DF4FF881CD59D040C85668
:1064F000DF4FF883C859D040C256DF4F2881CE59AC
:10650000D040C756DF4F2883C959D040CC56DF4F03
:106510008881C459D0408F5FCC56DF4F8883C459DF
:10652000D040AE969FADAE97913089F0A1E0AF9686
:10653000AFAFAF979F3F79F0AF961FAEAF97923056
:1065400051F4C656DF4F1881CA59D04005C0B1E09A
:10655000AF96BFAFAF9710E0FE017D9611921192FA
:1065600011921192AD968EAD9FADAD97E817F907D8
:10657000A9F7AE969FADAE97911111C0ACEAAF9658
:10658000AFAFAF97B5ECE396BFAFE397E7E2E7961F
:10659000EFAFE797F7E3E896FFAFE89723C4AE962F
:1065A0002FADAE97233099F4AE968FADAE97855050
:1065B000833008F448C0C12CD12CE0EAEE2EE0E490
:1065C000FE2E812C912CA12CF0E4BF2E59C0AE964A
:1065D0008FADAE97863041F3AE96AFADAE97A93092
:1065E00009F43EC019821A821B821C8219AE1AAEAF
:1065F0001BAE1CAE00E020E0C254DF4F4881CE5BF2
:10660000D040B101CE01C9960E941F522D8D3E8D02
:106610004F8D58A10F94F9486D8F7E8F8F8F98A35F
:106620009B01AC010F94F34B81110C94AD45AE96D8
:10663000BFADAE97B3300CF4D0C0AE969FADAE9761
:10664000983074F4B1CFC12CD12C60ECE62E60E40C
:10665000F62E812C912C70E8A72E7FE3B72E10C068
:106660004BEAC42E4AEAD42E4AECE42E40E4F42E3F
:106670005BEA852E5AEA952E5AE2A52E5FE3B52EE7
:1066800022E739EF4FE75FE3C701B6010F946D4B87
:1066900018160CF080C020E030E040E85FE3C7014E
:1066A000B6010F94F84820E030E040E752E40F9440
:1066B000344520E030E042E553E40F94F9482BEDF7
:1066C0003FE049E450E40F94344520E030E044E3F7
:1066D00053E40F94D5492B013C012DEC3CEC4CECE0
:1066E0005DE36091020C7091030C8091040C909119
:1066F000050C0F943445E6966CAF7DAF8EAF9FAF1F
:10670000E697C301B2010F94A84B9B01AC01E6963A
:106710006CAD7DAD8EAD9FADE6970F94344569832A
:106720007A838B839C83C301B2010F94D2499B016E
:10673000AC01E6966CAD7DAD8EAD9FADE6970F9446
:10674000344569AF7AAF8BAF9CAF00E020E0C25414
:10675000DF4F4881CE5BD040B101CE01C9960E9487
:106760001F522D8D3E8D4F8D58A10F94F9486D8F7E
:106770007E8F8F8F98A39B01AC010F94F34B8111F7
:106780000C94AD45A5019401C701B6010F94F848DA
:106790006B017C0175CFCD8CDE8CEF8CF8A0AE96B2
:1067A000EFADAE97E53069F0C050DF4F6881798179
:1067B0008A819B81C050D1400F94D5449B01AC018C
:1067C00004C020E030E040EE50E4C701B6010F9471
:1067D000D5496D8F7E8F8F8F98A3AF96FFADAF9702
:1067E000F11194C2112311F062E001C061E0AE9694
:1067F0002FADAE972A3011F1293071F12830E9F12F
:10680000273009F448C0263009F456C0253009F471
:1068100064C0AF961FAEAF97E3961FAEE3972430E8
:1068200009F46CC0233009F071C080E8E7968FAF9F
:10683000E7979FE3E8969FAFE8976FC0A9E8AF9608
:10684000AFAFAF97B8E8E396BFAFE397E8E8E79656
:10685000EFAFE797FDE356C02BEAAF962FAFAF97A8
:106860008AEAE3968FAFE3979AEAE7969FAFE797B6
:10687000ADE3E896AFAFE89750C0B9E3AF96BFAFCE
:10688000AF97EEE8E396EFAFE397F3EEE796FFAF4F
:10689000E7972DE33FC085E2AF968FAFAF9799E4BE
:1068A000E3969FAFE397A2E1E796AFAFE797BEE32A
:1068B000E896BFAFE89731C0EDECAF96EFAFAF977A
:1068C000FCECE396FFAFE3972CE4E7962FAFE79756
:1068D0008EE3E8968FAFE89720C09BEAAF969FAF14
:1068E000AF97AAEAE396AFAFE397BAEAE796BFAFEE
:1068F000E797EEE3E896EFAFE8970FC0E7961FAE95
:10690000E797FFE3E896FFAFE89707C0E7961FAE6B
:10691000E79720E4E8962FAFE897062E000C770B58
:10692000880B990B0F94D5444B015C0181E0E996EB
:106930008FAFE9972EE23FEF4FED50E4C501B40170
:106940000F94CF4487FF97C120E030E040E85FE339
:10695000C501B4010F94F84820E030E040E752E46C
:106960000F94344520E030E042E553E40F94F948B9
:106970002BED3FE049E450E40F94344520E030E053
:1069800044E353E40F94D5496B017C0120E030E0EF
:1069900040E85FE3C501B4010F94884AC058DF4F57
:1069A000688379838A839B83C058D040C701B6012E
:1069B0000F94A84BC857DF4F688379838A839B83E2
:1069C000C858D040C701B6010F94D249C457DF4F11
:1069D000688379838A839B83CC58D040ED961FAE21
:1069E000ED97E9969FADE997992391F0C250DF4F5B
:1069F00068817981CE5FD040ED96AFADED976A1B8F
:106A00007109A7FD7395072E000C880B990B08C020
:106A1000ED96BFADED976B2FBB0F770B880B990BE6
:106A20000F94D5442DEC3CEC4CEC5DE30F943445D5
:106A30009B01AC0160E070E080E89FE30F94F848B0
:106A40002091020C3091030C4091040C5091050CE4
:106A50000F9434456B017C01C857DF4F2881398181
:106A60004A815B81C858D0400F94344569837A834A
:106A70008B839C83C457DF4F288139814A815B8196
:106A8000CC58D040C701B6010F94344569AF7AAFF6
:106A90008BAF9CAF00E020E0C254DF4F4881CE5B5B
:106AA000D040B101CE01C9960E941F526B017C01FA
:106AB0009B01AC010F94F34B81110C94AD45C05870
:106AC000DF4F288139814A815B81C058D040C501A0
:106AD000B4010F94F8482B013C0120E030E040EC79
:106AE00050E40F94F94820E030E040E85FE30F9471
:106AF000F8480F94784B862F66E00F940F4C0DE109
:106B000010E00C0F1D1FE4E09E9F000D111D1124CD
:106B10000C5F1F4F20E030E044EB52E4C058DF4FE1
:106B2000688179818A819B81C058D0400F94344517
:106B30002BED3FE049E450E40F94344520E030E091
:106B400044E353E40F94D549CC57DF4F68837983EE
:106B50008A839B83C458D0400F94D2499B01AC01D7
:106B60000F943445A70196010F9434459B01AC0165
:106B7000D8016D917D918D919C910F94F948F80108
:106B80006083718382839383C301B2010F94784B36
:106B9000862F66E00F940F4C0DE110E00C0F1D1FC7
:106BA000F4E09F9F000D111D11240C5F1F4FCC5767
:106BB000DF4F688179818A819B81C458D0400F94CE
:106BC000A84B9B01AC010F943445A70196010F948B
:106BD00034459B01AC01D8016D917D918D919C91C3
:106BE0000F94F948F8016083718382839383ED9653
:106BF000FFADED97FF5FED96FFAFED97C154DF4F0F
:106C00002881CF5BD0402F170CF0EBCEE9968FADEB
:106C1000E99791E08927E9968FAFE997AE96AFADF6
:106C2000AE97A8309CF020E030E040E450E4AF960E
:106C30006FADAF97E3967FADE397E7968FADE7979C
:106C4000E8969FADE8970F9434450CC0AF966FADB2
:106C5000AF97E3967FADE397E7968FADE797E8961A
:106C60009FADE8979B01AC01C501B4010F94F948B1
:106C70004B015C015FCEAE96BFADAE97B430C4F4AD
:106C800019821A821B821C8219AE1AAE1BAE1CAE70
:106C900029961CAE1DAE1EAE1FAE2997A101BE01E6
:106CA000675C7F4FCE018B5B9F4F0E943D512EC092
:106CB000AF962FADAF97E3963FADE397E7964FAD15
:106CC000E797E8965FADE89760E070E080E89FE3C3
:106CD0000F94D5496B017C018E010F5D1F4FA701F9
:106CE0009601F80160817181828193810F94D54969
:106CF000D8016D937D938D939D938D01AD96EEADEF
:106D0000FFADAD97EA17FB0751F7BACFC655DF4F76
:106D10008881CA5AD040811131CC6D8D7E8D8F8D86
:106D200098A19B01AC010F9434456B017C01C052CA
:106D3000DF4FB880C05ED04001E010E0EDE1F0E050
:106D4000EC0FFD1F24E0B29EE00DF11D11246081C7
:106D50007181828193819B01AC010F9434459B0129
:106D6000AC01C701B6010F94F9486B017C010F5FBC
:106D70001F4FCF51DF4F8881C15ED040B80E96E0E3
:106D80009B15E0F6B801110F880B990B0F94D544B1
:106D90009B01AC01C701B6010F94D5490F94B24BCA
:106DA00020E030E04AE754E40F9434450F94784BE8
:106DB0000F94D54420E030E04AE754E40F94D549DD
:106DC0002CEA35EC47E257E30F94F948AF966FAFE2
:106DD000AF97E3967FAFE397E7968FAFE797E89695
:106DE0009FAFE897AF962FADAF97E3963FADE39790
:106DF000E7964FADE797E8965FADE897CA56DF4F45
:106E00006881C659D040C956DF4F7881C759D040F4
:106E1000C856DF4F8881C859D040C756DF4F988188
:106E2000C959D0400F946D4B181674F0C754DF4FFA
:106E3000A881C95BD040CC56DF4FB881C459D0403F
:106E4000AB1714F40C94DE40CC54DF4F2881398109
:106E50004A815B81C45BD040AF966FADAF97E3963C
:106E60007FADE397E7968FADE797E8969FADE897FC
:106E70000F946D4B181614F00C94DE40AF962FADA6
:106E8000AF97E3963FADE397E7964FADE797E89668
:106E90005FADE897C156DF4F6881CF59D040C056EB
:106EA000DF4F7881C05AD040CF55DF4F8881C15A1B
:106EB000D040CE55DF4F9881C25AD0400F946D4BD1
:106EC00018160CF080C080911A0C90911B0CA091A8
:106ED0001C0CB0911D0CC452DF4F88839983AA8388
:106EE000BB83CC5DD04080911E0C90911F0CA09173
:106EF000200CB091210CCC52DF4F88839983AA8358
:106F0000BB83C45DD0408091220C9091230CA09152
:106F1000240CB091250CC453DF4F88839983AA8336
:106F2000BB83CC5CD0408091160C9091170CA09143
:106F3000180CB091190CC054DF4F88839983AA8331
:106F4000BB83C05CD0408091260C9091270CA0910F
:106F5000280CB091290CCC53DF4F88839983AA83E6
:106F6000BB83C45CD04080910A0C90910B0CA09123
:106F70000C0CB0910D0CC853DF4F88839983AA8302
:106F8000BB83C85CD04080910E0C90910F0CA091F7
:106F9000100CB091110CC852DF4F88839983AA83DB
:106FA000BB83C85DD0408091120C9091130CA091CE
:106FB000140CB091150CC053DF4F88839983AA83BA
:106FC000BB83C05DD040FE01E35AFF4F8CE0DF0180
:106FD000282F1D922A95E9F73C97DF011D928A958B
:106FE000E9F74090020C5090030C6090040C7090F4
:106FF000050CAE96BFADAE97B83084F026E636E607
:1070000046E65FE3C301B2010F9434456093020C7E
:107010007093030C8093040C9093050C2091160C34
:107020003091170C4091180C5091190C6091020C82
:107030007091030C8091040C9091050C0F94D5492C
:107040002BEA3AEA4AE25FE30F94D5499B01AC018F
:1070500060E070E080E89FE30F94D549C458DF4FAB
:10706000688379838A839B83CC57D0409CE1E92E47
:10707000F1012E2D11922A95E9F75E0185E4A80E03
:10708000B11C2CE0F22ED501EF2D1D92EA95E9F707
:10709000AD96AEADBFADAD97EF2D1D92EA95E9F778
:1070A0008E01075C1F4F2AE037ED43E25CE3B50138
:1070B000C1010F9477302D853E854F8558896D81AC
:1070C0007E818F8198850F94F9482D893E894F895B
:1070D000588D0F94F94829893A894B895C890F9416
:1070E000F948298D3A8D4B8D5C8D0F94F94829858F
:1070F0003A854B855C850F94F948905820E030E044
:1071000040EC50E40F94D5499B01AC016AE077ED67
:1071100083E29CE30F94D54920E030E040E450E462
:107120000F94D549C155DF4F688379838A839B8348
:10713000CF5AD040D1011D92EA94E9F7F5012F2DE5
:1071400011922A95E9F7AD96AEADBFADAD971D9200
:10715000FA94E9F7EA961FAF0EAFEA97610135E0BE
:10716000F32EC555DF4F188219821A821B82CB5A23
:10717000D040C058DF4FA882C058D040EB2C19AE89
:107180001AAE1BAE1CAE21961CAE1DAE1EAE1FAEBF
:10719000219725961CAE1DAE1EAE1FAE2597EA9612
:1071A000EEADFFADEA978AE097EDA3E2BCE38193F1
:1071B0009193A193B193EA96FFAFEEAFEA978E0158
:1071C000075C1F4F20E030E0A901C058DF4F688105
:1071D000C058D0407E2DC1010F9477308F2D66E0CE
:1071E0000F940F4CF10124E0929FE00DF11D11244A
:1071F00020E030E040EC50E4648175818681978125
:107200000F94D549C555DF4F288139814A815B816B
:10721000CB5AD0400F94F9484B015C0120E030E09C
:1072200040EC50E4D60118966D917D918D919C9122
:107230001B970F94D5499B01AC01C501B4010F9474
:10724000F848C555DF4F688379838A839B83CB5A7F
:10725000D040F394F394B8E0CB0ED11CEBE0FE12D7
:107260008ECF4092020C5092030C6092040C7092EC
:10727000050CAE96FFADAE97F13029F0F23031F14A
:10728000F111C5C235C720E030E040E850E46D8D13
:107290007E8D8F8D98A10F94344520E030E040E83A
:1072A0005EE30F943445A1966CAF7DAF8EAF9FAF78
:1072B000A197A5966CAF7DAF8EAF9FAFA597A9960E
:1072C0006CAF7DAF8EAF9FAFA99712C78D8D9E8D8E
:1072D000AF8DB8A1EC968CAF9DAFAEAFBFAFEC97C2
:1072E000CD54DF4F9881C35BD040992309F434C15A
:1072F00089A19AA1ABA1BCA1C058DF4F8883998313
:10730000AA83BB83C058D04020E030E040E850E47E
:10731000BC01CD010F94344520E030E040E85EE34D
:107320000F943445CC57DF4F688379838A839B83DE
:10733000C458D040C9A4DAA4EBA4FCA4A7019601C8
:10734000C701B6010F94F94820E030E040E85EE361
:107350000F943445C857DF4F688379838A839B83B2
:10736000C858D04089A89AA8ABA8BCA8A501940188
:10737000C501B4010F94F94820E030E040E85EE335
:107380000F943445C457DF4F688379838A839B8386
:10739000CC58D04020E030E040E850E4EC966CADB2
:1073A0007DAD8EAD9FADEC970F94344520E030E07D
:1073B00040E85EE30F9434452B013C01C857DF4F92
:1073C000288139814A815B81C858D040CC57DF4F32
:1073D000688179818A819B81C458D0400F94F84894
:1073E000C457DF4F288139814A815B81CC58D04016
:1073F0000F94F848C458DF4F288139814A815B8156
:10740000CC57D0400F943445A30192010F94F94812
:10741000A1966CAF7DAF8EAF9FAFA19720E030E01B
:1074200040E850E4C701B6010F94344520E030E055
:1074300040E85EE30F943445C057DF4F688379839B
:107440008A839B83C059D040C058DF4F288139813F
:107450004A815B81C058D040CA01B9010F94F948F4
:1074600020E030E040E85EE30F9434456B017C019E
:107470009B01AC01C057DF4F688179818A819B8174
:10748000C059D0400F94F848C457DF4F2881398144
:107490004A815B81CC58D0400F94F848C458DF4FE4
:1074A000288139814A815B81CC57D0400F94344583
:1074B000A30192010F94F948A5966CAF7DAF8EAFF2
:1074C0009FAFA59720E030E040E850E4C501B4014B
:1074D0000F94344520E030E040E85EE30F943445FB
:1074E0004B015C01C701B6019058C857DF4F288196
:1074F00039814A815B81C858D0400F94F848A50172
:1075000094010F94F948C458DF4F288139814A818A
:107510005B81CC57D0400F943445A30192010F9466
:10752000F948A9966CAF7DAF8EAF9FAFA997C057B2
:10753000DF4F288139814A815B81C059D040CC57C7
:10754000DF4F688179818A819B81C458D0400F9434
:10755000F948A501940132C18DA99EA9AFA9B8AD82
:10756000C058DF4F88839983AA83BB83C058D0401B
:107570009C01AD01BC01CD010F94F94820E030E041
:1075800040E85EE30F943445CC57DF4F688379833E
:107590008A839B83C458D0408DA49EA4AFA4B8A86E
:1075A00020E030E040E850E4C501B4010F943445D8
:1075B00020E030E040E85EE30F943445C857DF4FE9
:1075C000688379838A839B83C858D040CDA0DEA08E
:1075D000EFA0F8A4A7019601C701B6010F94F948DE
:1075E00020E030E040E85EE30F943445C457DF4FBD
:1075F000688379838A839B83CC58D04020E030E035
:1076000040E850E4EC966CAD7DAD8EAD9FADEC974F
:107610000F94344520E030E040E85EE30F943445B9
:107620002B013C01C857DF4F288139814A815B819A
:10763000C858D040CC57DF4F688179818A819B81BF
:10764000C458D0400F94F848C457DF4F288139817F
:107650004A815B81CC58D0400F94F948C458DF4F21
:10766000288139814A815B81CC57D0400F943445C1
:10767000A30192010F94F948A1966CAF7DAF8EAF34
:107680009FAFA197A5019401C501B4010F94F948DA
:1076900020E030E040E85EE30F943445C057DF4F10
:1076A000688379838A839B83C059D04020E030E08F
:1076B00040E850E4C058DF4F688179818A819B811E
:1076C000C058D0400F94344520E030E040E85EE3FD
:1076D0000F9434454B015C019B01AC01C057DF4F57
:1076E000688179818A819B81C059D0400F94F84884
:1076F000C457DF4F288139814A815B81CC58D04003
:107700000F94F948C458DF4F288139814A815B8141
:10771000CC57D0400F943445A30192010F94F948FF
:10772000A5966CAF7DAF8EAF9FAFA59720E030E000
:1077300040E850E4C701B6010F94344520E030E042
:1077400040E85EE30F9434456B017C01C057DF4F86
:10775000288139814A815B81C059D040CC57DF4FA5
:10776000688179818A819B81C458D0400F94F948FF
:10777000A70196010F94F848C458DF4F288139813A
:107780004A815B81CC57D0400F943445A3019201CC
:107790000F94F948A9966CAF7DAF8EAF9FAFA997B4
:1077A000A5019401C857DF4F688179818A819B8147
:1077B000C858D0400F94F948A70196010F94F94892
:1077C0006B017C0120E030E040E451E4EC966CADCC
:1077D0007DAD8EAD9FADEC970F94344520E030E049
:1077E00040E85EE30F9434459B01AC01C701B6014C
:1077F0000F94F848C155DF4F288139814A815B8158
:10780000CF5AD0400F9434454B015C0188C489A104
:107810009AA1ABA1BCA1EC968CAF9DAFAEAFBFAFB0
:10782000EC979C01AD01BC01CD010F94F94820E01B
:1078300030E040E85EE30F943445C654DF4F688380
:1078400079838A839B83CA5BD04089A59AA5ABA51F
:10785000BCA5C058DF4F88839983AA83BB83C058D7
:10786000D04020E030E040E85EE3BC01CD010F9461
:107870003445CE51DF4F688379838A839B83C25E10
:10788000D04089A99AA9ABA9BCA9CC57DF4F88835E
:107890009983AA83BB83C458D04020E030E040E8FD
:1078A0005EE3BC01CD010F9434454B015C018DA515
:1078B0009EA5AFA5B8A9C857DF4F88839983AA832F
:1078C000BB83C858D0409C01AD01BC01CD010F94D1
:1078D000F94820E030E040E85EE30F943445CA51B7
:1078E000DF4F688379838A839B83C65ED0408DA9EE
:1078F0009EA9AFA9B8ADC457DF4F88839983AA83E7
:10790000BB83CC58D04020E030E040E85EE3BC01CF
:10791000CD010F943445C651DF4F688379838A8344
:107920009B83CA5ED0408DA19EA1AFA1B8A5C057D0
:10793000DF4F88839983AA83BB83C059D04020E05E
:1079400030E040E85EE3BC01CD010F9434456B01AB
:107950007C018D8D9E8DAF8DB8A1CD55DF4F888375
:107960009983AA83BB83C35AD04020E030E040E82B
:1079700050E4BC01CD010F94344520E030E040E8F4
:107980005EE30F9434452B013C01CE51DF4F28813B
:1079900039814A815B81C25ED040C654DF4F688125
:1079A00079818A819B81CA5BD0400F94F848A501F8
:1079B00094010F94F848CA51DF4F288139814A81D8
:1079C0005B81C65ED0400F94F848C651DF4F2881D6
:1079D00039814A815B81CA5ED0400F94F948A70182
:1079E00096010F94F948C458DF4F288139814A81A4
:1079F0005B81CC57D0400F943445A30192010F9482
:107A0000F948A1966CAF7DAF8EAF9FAFA197C058DC
:107A1000DF4F288139814A815B81C058D040CA013B
:107A2000B9010F94F94820E030E040E85EE30F949C
:107A30003445C251DF4F688379838A839B83CE5E4E
:107A4000D04020E030E040E85EE3EC966CAD7DADE8
:107A50008EAD9FADEC970F943445CE50DF4F6883C9
:107A600079838A839B83C25FD04020E030E040E886
:107A70005EE3C857DF4F688179818A819B81C8584E
:107A8000D0400F943445CA50DF4F688379838A838E
:107A90009B83C65FD040C457DF4F288139814A811C
:107AA0005B81CC58D040CA01B9010F94F94820E05D
:107AB00030E040E85EE30F943445C650DF4F688302
:107AC00079838A839B83CA5FD040CE50DF4F288161
:107AD00039814A815B81C25FD040C251DF4F6881EA
:107AE00079818A819B81CE5ED0400F94F848A501B0
:107AF00094010F94F848CA50DF4F288139814A8198
:107B00005B81C65FD0400F94F948C650DF4F288193
:107B100039814A815B81CA5FD0400F94F848A70140
:107B200096010F94F948C458DF4F288139814A8162
:107B30005B81CC57D0400F943445A30192010F9440
:107B4000F948A5966CAF7DAF8EAF9FAFA597CC5788
:107B5000DF4F288139814A815B81C458D040CA01F6
:107B6000B9010F94F94820E030E040E85EE30F945B
:107B700034454B015C01C057DF4F288139814A8170
:107B80005B81C059D040CA01B9010F94F94820E087
:107B900030E040E85EE30F9434456B017C01CE5049
:107BA000DF4F688179818A819B81C25FD040905884
:107BB000CE51DF4F288139814A815B81C25ED0403E
:107BC0000F94F848A50194010F94F948CA50DF4F6B
:107BD000288139814A815B81C65FD0400F94F94882
:107BE000C651DF4F288139814A815B81CA5ED0400E
:107BF0000F94F948A70196010F94F848C458DF4F35
:107C0000288139814A815B81CC57D0400F9434451B
:107C1000A30192010F94F948A9966CAF7DAF8EAF86
:107C20009FAFA997C251DF4F288139814A815B817B
:107C3000CE5ED040C654DF4F688179818A819B81B6
:107C4000CA5BD0400F94F948A50194010F94F948FC
:107C5000CA51DF4F288139814A815B81C65ED0409D
:107C60000F94F948C650DF4F288139814A815B81E2
:107C7000CA5FD0400F94F948A70196010F94F948C4
:107C80006B017C0120E030E040E451E4CD55DF4F52
:107C9000688179818A819B81C35AD0400F94344591
:107CA00020E030E040E85EE30F9434459B01AC01F6
:107CB000C701B6010F94F848C155DF4F28813981BB
:107CC0004A815B81CF5AD0400F9434454B015C010F
:107CD000CD54DF4F9881C35BD040992309F41FC274
:107CE000C555DF4F288139814A815B81CB5AD0400D
:107CF0006AE077ED83E29CE30F94D54920E030E021
:107D000040E450E40F94D549C458DF4F6883798329
:107D10008A839B83CC57D04020E030E040E850E499
:107D2000C058DF4F688179818A819B81C058D040DB
:107D30000F94344520E030E040E85EE30F94344592
:107D4000C555DF4F688379838A839B83CB5AD040A4
:107D500020E030E040E850E4CC57DF4F6881798183
:107D60008A819B81C458D0400F94344520E030E094
:107D700040E85EE30F9434452B013C0120E030E005
:107D800040E850E4C457DF4F688179818A819B8144
:107D9000CC58D0400F94344520E030E040E85EE31A
:107DA0000F943445C155DF4F688379838A839B8361
:107DB000CF5AD04020E030E040E850E4C057DF4FD9
:107DC000688179818A819B81C059D0400F94344564
:107DD00020E030E040E85EE30F943445C654DF4FC6
:107DE000688379838A839B83CA5BD04020E030E03C
:107DF000A901CD55DF4F688179818A819B81C35A62
:107E0000D0400F94344520E030E040E85EE30F942A
:107E10003445CD55DF4F688379838A839B83C35A6A
:107E2000D04020E030E0A901EC966CAD7DAD8EAD88
:107E30009FADEC970F94344520E030E040E85EE3DE
:107E40000F943445C555DF4F288139814A815B81C4
:107E5000CB5AD0400F94F848A30192010F94F948EF
:107E60006B017C0120E030E0A901C857DF4F688139
:107E700079818A819B81C858D0400F94344520E095
:107E800030E040E85EE30F9434459B01AC01C7014C
:107E9000B6010F94F948C155DF4F288139814A81D5
:107EA0005B81CF5AD0400F94F848C654DF4F2881E9
:107EB00039814A815B81CA5BD0400F94F948CD5526
:107EC000DF4F288139814A815B81C35AD0400F94AA
:107ED000F948C458DF4F288139814A815B81CC57EA
:107EE000D0400F94344565966CAF7DAF8EAF9FAF99
:107EF000659720E030E040E850E4EC966CAD7DAD55
:107F00008EAD9FADEC970F94344520E030E040E813
:107F10005EE30F943445EC966CAF7DAF8EAF9FAFB0
:107F2000EC9720E030E040E850E4C857DF4F68812C
:107F300079818A819B81C858D0400F94344520E0D4
:107F400030E040E85EE30F9434456B017C0120E0B3
:107F500030E0A901C058DF4F688179818A819B8117
:107F6000C058D0400F94344520E030E040E85EE354
:107F70000F943445EC962CAD3DAD4EAD5FADEC9716
:107F80000F94F948A30192010F94F848A7019601B4
:107F90000F94F9482B013C0120E030E0A901C457BF
:107FA000DF4F688179818A819B81CC58D0400F94C2
:107FB000344520E030E040E85EE30F9434459B0117
:107FC000AC01C301B2010F94F948C654DF4F2881B8
:107FD00039814A815B81CA5BD0400F94F848CD5506
:107FE000DF4F288139814A815B81C35AD0400F9489
:107FF000F948C458DF4F288139814A815B81CC57C9
:10800000D0400F94344569966CAF7DAF8EAF9FAF73
:10801000699720E030E0A901CC57DF4F6881798172
:108020008A819B81C458D0400F94344520E030E0D1
:1080300040E85EE30F9434452B013C01EC962CADF7
:108040003DAD4EAD5FADEC97C555DF4F6881798191
:108050008A819B81CB5AD0400F94F8489B01AC0198
:10806000C301B2010F94F948A70196010F94F84893
:10807000C155DF4F288139814A815B81CF5AD04079
:108080000F94F9486B017C0120E030E0A901C05752
:10809000DF4F688179818A819B81C059D0400F94DC
:1080A000344520E030E040E85EE30F9434459B0126
:1080B000AC01C701B6010F94F948CD55DF4F2881B7
:1080C00039814A815B81C35AD0400F94F948C45822
:1080D000DF4F288139814A815B81CC57D0400F9492
:1080E00034456D966CAF7DAF8EAF9FAF6D9717C067
:1080F000812C912C5401CA56DF4F1882C659D040AA
:10810000C956DF4F1882C759D040C856DF4F188272
:10811000C859D040C756DF4F1882C959D0407E0198
:10812000ADE5EA0EF11C0AE11CE0F7012191319165
:10813000419151917F01D8016D917D918D919C91DB
:108140000F94F948F80161937193819391938F0192
:10815000FCE006321F0749F7A50194016091160C57
:108160007091170C8091180C9091190C0F94F9488C
:108170006093160C7093170C8093180C9093190C45
:108180007E0121E5E20EF11C0AE01CE0D7012D91F1
:108190003D914D915D917D01F801608171818281F8
:1081A00093810F94F948D8016D937D938D939D939E
:1081B0008D01BCE006311B0749F7A5C0AF962FAD76
:1081C000AF97E3963FADE397E7964FADE797E89615
:1081D0005FADE897CA56DF4F6881C659D040C9568F
:1081E000DF4F7881C759D040C856DF4F8881C859C2
:1081F000D040C756DF4F9881C959D0400F94CF4423
:1082000018160CF480C0C452DF4F88819981AA816E
:10821000BB81CC5DD04080931A0C90931B0CA09333
:108220001C0CB0931D0CCC52DF4F88819981AA8120
:10823000BB81C45DD04080931E0C90931F0CA09313
:10824000200CB093210CC453DF4F88819981AA81FF
:10825000BB81CC5CD0408093220C9093230CA093E4
:10826000240CB093250CC054DF4F88819981AA81DA
:10827000BB81C05CD0408093160C9093170CA093E8
:10828000180CB093190CCC53DF4F88819981AA81C7
:10829000BB81C45CD0408093260C9093270CA093A4
:1082A000280CB093290CC853DF4F88819981AA818B
:1082B000BB81C85CD04080930A0C90930B0CA093B8
:1082C0000C0CB0930D0CC852DF4F88819981AA81A4
:1082D000BB81C85DD04080930E0C90930F0CA0938F
:1082E000100CB093110CC053DF4F88819981AA8183
:1082F000BB81C05DD0408093120C9093130CA0936F
:10830000140CB093150CCB56DF4F9881C559D04053
:10831000911148C00E94016DAF962FADAF97E396C3
:108320003FADE397E7964FADE797E8965FADE897E7
:10833000C156DF4F6881CF59D040C056DF4F78819A
:10834000C05AD040CF55DF4F8881C15AD040CE555A
:10835000DF4F9881C25AD0400F946D4B18160CF025
:10836000C1C0AF96EFADAF97C156DF4FE883CF598D
:10837000D040E396FFADE397C056DF4FF883C05A75
:10838000D040E7962FADE797CF55DF4F2883C15AEE
:10839000D040E8968FADE897CE55DF4F8883C25A1C
:1083A000D040A0C0C955DF4FA881C75AD040A11105
:1083B00023C0C090220CD090230CE090240CF090AD
:1083C000250CA0901E0CB0901F0C0091200C109159
:1083D000210C60901A0C70901B0C80901C0C9090DB
:1083E0001D0C9301A401B501C8010F94CF4487FF70
:1083F00045C05301840142C020E030E0A9016091F2
:108400000A0C70910B0C80910C0C90910D0C0F9438
:10841000F94820910E0C30910F0C4091100C5091A6
:10842000110C0F94F9482091120C3091130C4091CB
:10843000140C5091150C0F94F94820E030E040E402
:1084400050E40F94D5494B015C010AE01CE086E141
:10845000E82E8CE0F82EA5019401F801608171816D
:10846000828193810F94F848D8016D937D938D9309
:108470009D938D01EA16FB0671F79BCF9501A8012C
:10848000B601C7010F94CF4487FF02C06501780190
:108490009601A7016091260C7091270C8091280C01
:1084A0009091290C0F94F8486093260C7093270C38
:1084B0008093280C9093290C0AE11CE09601A701F7
:1084C000F80160817181828193810F94F848D8010D
:1084D0006D937D938D939D938D01BCE006321B07B8
:1084E00069F718CFCB56DF4F9881C559D0409330EC
:1084F00009F060C0E0E5F7E084918F010F5F1F4F46
:10850000882321F00E949C5BF801F6CFBE01635ED8
:108510007F4F8EE497E00F94C033C755DF4FA8819B
:10852000C95AD040AA2331F1BE016F5D7F4F8BE461
:1085300097E00F94C033BE01675D7F4F88E497E0FA
:108540000F94C033BE016F5C7F4F85E497E00F94BA
:10855000C033C855DF4FB881C85AD040BB2331F172
:108560008AE00E949C5B8EE20E949C5B8DE00E94F0
:1085700040C307C0C855DF4FE881C85AD040EE233A
:10858000A9F0BE01635D7F4F82E497E00F94C03392
:10859000BE016B5C7F4F8FE397E00F94C033BE0149
:1085A0006B5D7F4F8CE397E00F94C0338AE00E94AD
:1085B0009C5B0AC0CB56DF4FF881C559D040F11102
:1085C00003C0EDE0F8E0ADC1AF962FADAF97E396F5
:1085D0003FADE397E7964FADE797E8965FADE89735
:1085E000CA56DF4F6881C659D040C956DF4F7881DF
:1085F000C759D040C856DF4F8881C859D040C756A8
:10860000DF4F9881C959D0400F94CF44181664F0B9
:10861000C754DF4F2881C95BD040CC56DF4F8881DB
:10862000C459D0402817CCF0CC54DF4F2881398171
:108630004A815B81C45BD040AF966FADAF97E39644
:108640007FADE397E7968FADE797E8969FADE89704
:108650000F94CF4418160CF4FDC0EEEFF7E08491B0
:108660008F010F5F1F4F882321F00E949C5BF80150
:10867000F6CF80E20E9440C3AF962FADAF97E3964E
:108680003FADE397E7964FADE797E8965FADE89784
:10869000CA56DF4F6881C659D040C956DF4F78812E
:1086A000C759D040C856DF4F8881C859D040C756F7
:1086B000DF4F9881C959D0400F94CF4418167CF0F1
:1086C000C655DF4F9881CA5AD040911108C0AE9666
:1086D000AFADAE97AA2319F0E7EEF7E003C0E5EFE0
:1086E000F7E00AC084918F010F5F1F4F882329F1A3
:1086F0000E949C5BF801F6CF84918F010F5F1F4FA2
:10870000882321F00E949C5BF801F6CF43E0C1561C
:10871000DF4F6881CF59D040C056DF4F7881C05AB3
:10872000D040CF55DF4F8881C15AD040CE55DF4F62
:108730009881C25AD0400E94C55E8AE00E949C5B2C
:1087400067ED77E0C1010F94184420E030E040E885
:108750005FE3C156DF4F6881CF59D040C056DF4F2D
:108760007881C05AD040CF55DF4F8881C15AD04060
:10877000CE55DF4F9881C25AD0400F94CF4487FF27
:1087800021C020E030E04AE754E4C156DF4F688161
:10879000CF59D040C056DF4F7881C05AD040CF5516
:1087A000DF4F8881C15AD040CE55DF4F9881C25AE1
:1087B000D0400F9434450F94784B7F936F9380EDA6
:1087C00097E01AC0C156DF4F6881CF59D040C056DC
:1087D000DF4F7881C05AD040CF55DF4F8881C15AD2
:1087E000D040CE55DF4F9881C25AD0400F94784B7D
:1087F0007F936F9389EC97E09F938F93CE01409680
:108800009F938F930F9469440F900F900F900F9048
:108810000F900F9060E0C1010E94CE88C955DF4FD4
:108820006881C75AD040C854DF4F8881C85BD040A8
:108830000F94FD33EBE9F7E084918F010F5F1F4F39
:10884000882321F00E949C5BF801F6CF8AE00E9409
:108850009C5BEEC0CC56DF4FB881C459D040BF31CD
:10886000C4F48B2F0B2E000C990B9F93BF938AE8B7
:1088700097E09F938F933F922F920F9469440F90AC
:108880000F900F900F900F900F908E010F5F1F4F62
:1088900006C06BE777E0C1010F941844F6CFF801EA
:1088A00081918F01882319F00E949C5BF8CF80E2B0
:1088B0000E9440C3E2E7F7E084918F010F5F1F4FF2
:1088C000882321F00E949C5BF801F6CF43E0AF962D
:1088D0006FADAF97E3967FADE397E7968FADE797E0
:1088E000E8969FADE8970E94C55E8AE00E949C5B77
:1088F00060E0C1010E94CE88CB56DF4FF881C55998
:10890000D040F23008F494C0C955DF4F6881C75A8F
:10891000D040C854DF4F8881C85BD0400F94FD33EE
:1089200087C084918F010F5F1F4F882321F00E9421
:108930009C5BF801F6CF83E20E9440C3E9E6F7E0D2
:1089400084918F010F5F1F4F882321F00E949C5B51
:10895000F801F6CF43E0AF966FADAF97E3967FADEA
:10896000E397E7968FADE797E8969FADE8970E946B
:10897000C55E8AE00E949C5B6DE078E0C1010F94C7
:10898000184464E677E0CE010C960F94184420E07A
:1089900030E040E85FE3AF966FADAF97E3967FAD11
:1089A000E397E7968FADE797E8969FADE8970F942A
:1089B000CF4487FF19C020E030E04AE754E4AF9687
:1089C0006FADAF97E3967FADE397E7968FADE797EF
:1089D000E8969FADE8970F9434450F94784B7F93BA
:1089E0006F938DE597E012C0AF966FADAF97E396AA
:1089F0007FADE397E7968FADE797E8969FADE89751
:108A00000F94784B7F936F9386E597E09F938F93B6
:108A1000CE0140969F938F930F9469440F900F90CF
:108A20000F900F900F900F9060E0C1010E94CE88D0
:108A300081E08093750A0E94039B8091740A809361
:108A4000750AAF962FADAF97E3963FADE397E796E4
:108A50004FADE797E8965FADE897CA56DF4F68815C
:108A6000C659D040C956DF4F7881C759D040C85643
:108A7000DF4F8881C859D040C756DF4F9881C95908
:108A8000D0400F946D4B18163CF4CC56DF4F288124
:108A9000C459D0402F316CF0C754DF4F8881C95B77
:108AA000D040CC56DF4F9881C459D04089170CF480
:108AB0004EC0C556DF4FE880CB59D040C456DF4F7B
:108AC000F880CC59D040C356DF4F0881CD59D040F3
:108AD000C256DF4F1881CE59D040CC54DF4F288189
:108AE00039814A815B81C45BD040AF966FADAF974F
:108AF000E3967FADE397E7968FADE797E8969FAD56
:108B0000E8970F946D4B181614F5AF969FADAF977D
:108B1000C556DF4F9883CB59D040E396AFADE3976E
:108B2000C456DF4FA883CC59D040E796BFADE79736
:108B3000C356DF4FB883CD59D040E896EFADE897E4
:108B4000C256DF4FE883CE59D0400C94193280E0F2
:108B50000E947E510E9405513EC0E9E1F8E08491F7
:108B60008F010F5F1F4F882391F30E949C5BF801D8
:108B7000F6CFC855DF4F1882C85AD040C755DF4FCF
:108B80001882C95AD04010E00C94B72FCD54DF4F53
:108B9000F881C35BD040FF2391F0C656DF4F888138
:108BA000CA59D040C855DF4F8883C85AD040C755EE
:108BB000DF4F8883C95AD040182F0C94BC2FC6565B
:108BC000DF4F1881CA59D040C755DF4F1882C95AA4
:108BD000D0400C94B12FCD5FDE4F0FB6F894DEBFBE
:108BE0000FBECDBFDF91CF911F910F91FF90EF90FE
:108BF000DF90CF90BF90AF909F908F907F906F90BD
:108C00005F904F903F902F9008958F929F92AF92D8
:108C1000BF92CF92DF92EF92FF920F931F93CF9369
:108C2000DF93CDB7DEB764970FB6F894DEBF0FBE03
:108C3000CDBFD62EF72E8C0180904D1390904E1301
:108C4000A0904F13B0905013A50194016091560D60
:108C50007091570D8091580D9091590D0F94CF44FC
:108C600081113DC020915113309152134091531303
:108C70005091541360915A0D70915B0D80915C0D71
:108C800090915D0D0F94CF44811129C0209155130F
:108C900030915613409157135091581360915E0DC7
:108CA00070915F0D8091600D9091610D0F94CF4494
:108CB000811115C02091591330915A1340915B13C3
:108CC00050915C136091620D7091630D8091640D01
:108CD0009091650D0F94CF44882309F46DC0E09006
:108CE000F00C20E030E0A9016D2D7F2DC8010F941C
:108CF000CF44811108C0D0900102F090020200918F
:108D00000302109104026091540270915502072EE3
:108D1000000C880B990B0F94D5442D2D3F2DA801E5
:108D20000F9434452AE037ED43E25CE30F94344579
:108D3000698B7A8B8B8B9C8B1D861E861F86188A6F
:108D400089829A82AB82BC82809151139091521396
:108D5000A0915313B09154138D839E83AF83B88732
:108D60008091551390915613A0915713B0915813B9
:108D700089879A87AB87BC87AE01475F5F4FBE018B
:108D80006B5F7F4FCE0101960F942B2CCE01019685
:108D90000E949E66CE010D966C018E010F5E1F4FE4
:108DA00029E533E14EE65DE06AE67DE086E69DE09A
:108DB0000E9437AD0E94925B64960FB6F894DEBFB6
:108DC0000FBECDBFDF91CF911F910F91FF90EF901C
:108DD000DF90CF90BF90AF909F908F9008952F928B
:108DE0003F924F925F926F927F928F929F92AF923B
:108DF000BF92CF92DF92EF92FF920F931F93CF9388
:108E0000DF93CDB7DEB72C970FB6F894DEBF0FBE59
:108E1000CDBF2B013C0129833A834B835C834701FF
:108E20005801F601108181818C8792819B87038193
:108E300020E030E0A901612F782F892F902F0F9427
:108E4000CF4481110BC0E3E7FCE085919591A5919A
:108E5000B491382E292EAD83BE8305C0312E2C84CB
:108E6000AB85AD830E83A3019201C301B2010F94C0
:108E700034456B017C0129813A814B815C81CA01B7
:108E8000B9010F9434459B01AC01C701B6010F94A1
:108E9000F94820E030E442E556E40F94CF44181638
:108EA0000CF4ECC020E030E0A901612F7C858B85BB
:108EB000902F0F94CF4481110AC010910702B091F6
:108EC0000802BC87809109028B8700910A02809179
:108ED000010290910202A0910302B09104028F83DB
:108EE0009887A987BA87812F9C85AB85B02F8093FF
:108EF000010290930202A0930302B09304020E9425
:108F0000885BC0904802D0904902E0904A02F090FD
:108F10004B02A701960160915E0D70915F0D8091EB
:108F2000600D9091610D0F946D4B18160CF04CC0B4
:108F3000A5019401C701B6010F94CF4487FF38C043
:108F400040924D1350924E1360924F1370925013F3
:108F500089819A81AB81BC81809351139093521384
:108F6000A0935313B09354138092551390925613B9
:108F7000A0925713B092581360E070E0CB012C968A
:108F80000FB6F894DEBF0FBECDBFDF91CF911F911A
:108F90000F91FF90EF90DF90CF90BF90AF909F9098
:108FA0008F907F906F905F904F903F902F902DCE3D
:108FB000C0925513D0925613E0925713F092581363
:108FC00060E070E0CB0121DE20915E0D30915F0DFD
:108FD0004091600D5091610DC501B4010F946D4B2E
:108FE00018166CF48092551390925613A092571352
:108FF000B0925813632D722D8D819E8106DE4092B2
:109000004D1350924E1360924F13709250138981FA
:109010009A81AB81BC818093511390935213A0939A
:109020005313B09354130E94C56720915E0D309185
:109030005F0D4091600D5091610DC501B4010F9419
:10904000CF4487FF0DC08092551390925613A09283
:109050005713B0925813632D722D8D819E81D5DDEB
:109060000E9443BB8F819885A985BA8580930102B0
:1090700090930202A0930302B09304022C960FB6C1
:10908000F894DEBF0FBECDBFDF91CF911F910F913E
:10909000FF90EF90DF90CF90BF90AF909F908F9018
:1090A0007F906F905F904F903F902F9008959F9288
:1090B000AF92BF92CF92DF92EF92FF920F931F93E6
:1090C000CF93DF938BE5A82E82E0B82E0DE413E159
:1090D000C6E5DDE096EDC92E9CE0D92E2CE4E22E0B
:1090E00023E0F22E912CF50181915F010E942D5B0E
:1090F000882309F10E94FA5AF7012081211104C046
:1091000020915003222339F0288139814A815B81E3
:109110000F94F9480AC0F3E09F1639F0F601208158
:109120003181428153810F94F848F8016083718343
:109130008283938309C088819981AA81BB81F801C8
:1091400080839183A283B38393940C5F1F4F2496F3
:10915000F4E0CF0ED11C2FEFE21AF20A84E098124D
:10916000C2CF86E40E94765B8823C9F00E94FA5A37
:1091700020E030E0A9010F946D4B181684F40E9492
:10918000FA5A20E030E040E752E40F94D54960936A
:109190000102709302028093030290930402DF9114
:1091A000CF911F910F91FF90EF90DF90CF90BF90E4
:1091B000AF909F9008952F923F924F925F926F923F
:1091C0007F929F92AF92BF92CF92DF92EF92FF92E7
:1091D0000F931F93CF93DF93CDB7DEB764970FB68E
:1091E000F894DEBF0FBECDBF1A012B01922EF32ED5
:1091F000C82ED12CF601E854F34FE491AA24A3948D
:109200001E160CF4A12CBB24B39420E030E0A9017D
:10921000C201B1010F946D4B18160CF0B12CCC0C9F
:10922000DD1CCC0CDD1CC6018A5A924F3C01FC01AE
:1092300010821182128213820E947D5AF3012082D1
:10924000318242825382E090F00C20E030E0A901AC
:10925000B801892D9F2D0F94CF4481110AC0F601CA
:10926000E559F34F85919591A591B4918C019A2E72
:10927000FB2EC801A92DBF2D898B9A8BAB8BBC8B84
:1092800080915E0D90915F0DA091600DB091610D88
:1092900040915A0D50915B0D60915C0D70915D0D88
:1092A0000091560D1091570D2091580D3091590D88
:1092B00009831A832B833C834D835E836F83788776
:1092C00089879A87AB87BC871D861E861F86188A6A
:1092D000CE010D966C018E010F5E1F4F22E63DE020
:1092E000AE01475F5F4FBE016B5F7F4F0C970E94DF
:1092F00037AD0E9443BBAB100F94C32F64960FB6DB
:10930000F894DEBF0FBECDBFDF91CF911F910F91BB
:10931000FF90EF90DF90CF90BF90AF909F907F90A5
:109320006F905F904F903F902F900895CF939091C2
:10933000010C9817B9F0C82F0E9443BBC093010CD1
:10934000C11109C00E9461638AEB94E00F941C2B49
:109350000E94B27404C086E59DE00F941C2BCF914F
:109360000C947B5ACF91089580E0E0DFEAEAFFE0B9
:1093700080E090E0A0E8BFE380839183A283B38381
:109380001482158216821782108611861286138621
:109390001486158616861786808B918BA28BB38BCD
:1093A000148A158A168A178A108E118E128E138EC1
:1093B000148E158E168E178E80A391A3A2A3B3A32D
:1093C0000895EF92FF921F93CF93DF93882329F0A4
:1093D000D091E60CD095D17001C0D0E0662339F071
:1093E0001091E60C1695117081E0182701C010E06D
:1093F000442341F0C091E60CC2FB882780F9C1E00C
:10940000C82701C0C0E0D11105C0111103C0CC2391
:1094100009F482C0E2E5FFE284917F019FEFE91A3F
:10942000F90A811103C0E6E8F9E004C00E949C5BE0
:10943000F701F2CF84917F019FEFE91AF90A88239F
:1094400021F00E949C5BF701F5CFDD2369F0E4E891
:10945000F9E084917F019FEFE91AF90A882321F04E
:109460000E949C5BF701F5CF112369F0E2E8F9E077
:1094700084917F019FEFE91AF90A882321F00E9465
:109480009C5BF701F5CFCC2319F0E0E8F9E003C0CD
:10949000E8E7F9E00BC084917F019FEFE91AF90A30
:1094A0008823B1F30E949C5BF701F5CF84917F0183
:1094B0009FEFE91AF90A882321F00E949C5BF701CB
:1094C000F5CFCC2319F048E253E002C043E253E069
:1094D000112319F02AE233E002C023E233E0DD2356
:1094E00019F08CE293E002C083E293E05F934F9324
:1094F0003F932F939F938F9386E699E09F938F934B
:109500001F920E943CF98DB79EB709960FB6F8944A
:109510009EBF0FBE8DBFC1E08C2FDF91CF911F91F9
:10952000FF90EF9008952F923F924F925F926F922B
:109530007F928F929F92AF92BF92CF92DF92EF92E3
:10954000FF920F931F93CF93DF93CDB7DEB7C4562F
:10955000D1090FB6F894DEBF0FBECDBF382E41E063
:1095600061E081E02EDF811136C680912A028823D6
:1095700009F431C69CDD82E50E94765B882309F4FC
:109580002CC10E94FA5A4B015C0120E030E0A90195
:109590000F94CF44882309F406C62091560D3091CC
:1095A000570D4091580D5091590D298F3A8F4B8F7F
:1095B0005C8F80915A0D90915B0DA0915C0DB091E4
:1095C0005D0D8D8F9E8FAF8FB8A320914D1330917D
:1095D0004E1340914F13509150132DA73EA74FA704
:1095E00058AB8091511390915213A0915313B091A5
:1095F00054138DA39EA3AFA3B8A7698D7A8D8B8DCD
:109600009C8D0F94CF4481110DC02DA13EA14FA17F
:1096100058A56D8D7E8D8F8D98A10F94CF44882392
:1096200009F4C1C5E32CF12C01E010E020E030E0AA
:10963000A901C501B4010F94CF4487FD02C000E029
:1096400010E0E016F10649F420E030E040E85FE386
:1096500029AB3AAB4BAB5CAB08C080E090E0A0E834
:10966000BFEB89AB9AABABABBCAB298D3A8D4B8DC5
:109670005C8D6DA57EA58FA598A90F94F84869A764
:109680007AA78BA79CA72D8D3E8D4F8D58A16DA1DC
:109690007EA18FA198A50F94F8486B017C0129A5A4
:1096A0003AA54BA55CA5CA01B9010F9434452B011D
:1096B0003C01A7019601C701B6010F9434459B01F7
:1096C000AC01C301B2010F94F9480F94B24B69A3E6
:1096D0007AA38BA39CA320E030E040E05FE30F94EB
:1096E00034452B013C01A5019401C501B4010F943F
:1096F00034454B015C01A3019201C301B2010F94F7
:1097000034459B01AC01C501B4010F94F8480F9496
:10971000B24B9B01AC0169A97AA98BA99CA90F94B2
:1097200034454B015C01C701B601905829A13AA10B
:109730004BA15CA10F94D549A50194010F94344528
:109740006B017C012DA53EA54FA558A9698D7A8D89
:109750008B8D9C8D0F94F94820E030E040E05FE372
:109760000F9434459B01AC01C701B6010F94F94831
:10977000298D3A8D4B8D5C8D0F94F8486B017C01DF
:109780002DA13EA14FA158A56D8D7E8D8F8D98A1E5
:109790000F94F94820E030E040E05FE30F94344557
:1097A0002B013C0129A13AA14BA15CA169A57AA595
:1097B0008BA59CA50F94D549A50194010F94344520
:1097C0009B01AC01C301B2010F94F9482D8D3E8D70
:1097D0004F8D58A10F94F84814C089E40E94765B1D
:1097E000882329F00E94FA5A6B017C0103C0C12C26
:1097F000D12C76018AE40E94765B8823D9F00E94FE
:10980000FA5A6DA77EA78FA798AB20E030E0A90198
:10981000C701B6010F94CF4481111AC020E030E097
:10982000A9016DA57EA58FA598A90F94CF4481119C
:109830000FC0B9C420E030E0A901C701B6010F9400
:10984000CF44882309F4AFC41DA61EA61FA618AADC
:10985000A70196015058298F3A8F4B8F5C8F8DA5A9
:109860009EA5AFA5B8A9B0588D8F9E8FAF8FB8A316
:10987000CA01B9010F9434454B015C012D8D3E8D19
:109880004F8D58A1CA01B9010F9434459B01AC0119
:10989000C501B4010F94F9480F94B24B21966CAFF7
:1098A0007DAF8EAF9FAF21972091560D3091570D10
:1098B0004091580D5091590D2DA33EA34FA358A789
:1098C000C701B6010F94F9482D966CAF7DAF8EAFEE
:1098D0009FAF2D9780915A0D90915B0DA0915C0DDB
:1098E000B0915D0D89A79AA7ABA7BCA79C01AD015C
:1098F0006DA57EA58FA598A90F94F94861966CAFC8
:109900007DAF8EAF9FAF619720914D1330914E1375
:1099100040914F135091501329AB3AAB4BAB5CAB1A
:109920002D962CAD3DAD4EAD5FAD2D9769A97AA9B1
:109930008BA99CA90F94F8486B017C01809151136D
:1099400090915213A0915313B09154138DAB9EABD1
:10995000AFABB8AF61962CAD3DAD4EAD5FAD61978D
:10996000BC01CD010F94F8484B015C0120915E0DC4
:1099700030915F0D4091600D5091610D29AF3AAF6C
:109980004BAF5CAF60915513709156138091571394
:10999000909158130F94F84869A37AA38BA39CA3C2
:1099A000A7019601698D7A8D8B8D9C8D0F9434451E
:1099B0002B013C01A50194016D8D7E8D8F8D98A1A9
:1099C0000F9434459B01AC01C301B2010F94F948D7
:1099D0002B013C01A5019401698D7A8D8B8D9C8DA5
:1099E0000F9434454B015C01A70196016D8D7E8D6E
:1099F0008F8D98A10F9434459B01AC01C501B40132
:109A00000F94F848A30192010F946C496B017C01FB
:109A100020E030E0A9010F94CF4487FF0AC02BED6E
:109A20003FE049EC50E4C701B6010F94F9486B01DF
:109A30007C01332051F02BED3FE049EC50E4C701AD
:109A4000B6010F94F8486B017C0120E030E0A901D9
:109A5000C701B6010F94CF44811120C029A93AA9AA
:109A60004BA95CA96DA17EA18FA198A50F94CF44AD
:109A7000811114C02DA93EA94FA958AD69A57AA599
:109A80008BA59CA50F94CF44811108C08BEDC82EE7
:109A90008FE0D82E89ECE82E80E4F82EA7019601FD
:109AA00021966CAD7DAD8EAD9FAD21970F94344561
:109AB0004B015C0120E030E0A90169A17AA18BA1F2
:109AC0009CA10F94CF448823D9F0A5019401C5012E
:109AD000B4010F9434454B015C0129A13AA14BA17B
:109AE0005CA1CA01B9010F9434459B01AC01C501C9
:109AF000B4010F94F9480F94B24B4B015C010DC0B7
:109B000020E030E0A901C501B4010F946D4B87FF3F
:109B100004C0B7FAB094B7F8B0942FE632E143E846
:109B20005AE3C501B4010F94CF4487FD54C3C50166
:109B3000B4010F946E4A0F94424A7AAB69AB672B1B
:109B400021F481E090E09AAB89AB4090620D509097
:109B5000630D6090640D7090650DA9A9BAA9BD014F
:109B600080E090E00F94D3444B015C019B01AC0179
:109B7000C701B6010F94D5496DA37EA38FA398A703
:109B8000A501940169A17AA18BA19CA10F94D5494B
:109B9000A1966CAF7DAF8EAF9FAFA197A30192014D
:109BA0006091591370915A1380915B1390915C13DB
:109BB0000F94F848A50194010F94D549A5966CAF70
:109BC0007DAF8EAF9FAFA5972DA13EA14FA158A508
:109BD000CA01B9010F94344520E030E040E05FE372
:109BE0000F9434459B01AC0160E070E080E89FE396
:109BF0000F94F84865966CAF7DAF8EAF9FAF6597B9
:109C000029AD3AAD4BAD5CAD29873A874B875C8770
:109C10004D865E866F86788A6091540270915502F7
:109C2000072E000C880B990B0F94D544209101024C
:109C30003091020240910302509104020F94344586
:109C40002AE037ED43E25CE30F94344569966CAF4C
:109C50007DAF8EAF9FAF69970F94D20E9B01AC0181
:109C600028533F4F4F4F5F4F6D962CAF3DAF4EAFD8
:109C70005FAF6D978091E20F9091E30FA091E40F99
:109C8000B091E50F21968CAF9DAFAEAFBFAF2197DE
:109C90002091E60F3091E70F4091E80F5091E90FC6
:109CA00025962CAF3DAF4EAF5FAF25978091EA0F61
:109CB0009091EB0FA091EC0FB091ED0F29968CAF26
:109CC0009DAFAEAFBFAF2997998D99A3AA8DA9A7D4
:109CD0002B8C3C8C21E030E03EAB2DAB39E139AF31
:109CE00049A95AA98DA99EA94817590709F4BFC1C6
:109CF0000E94BEE80F94D20EDC01CB016D962CAD14
:109D00003DAD4EAD5FAD6D97821B930BA40BB50BB4
:109D1000B7FD11C00F94D20E9B01AC0128533F4FE9
:109D20004F4F5F4F6D962CAF3DAF4EAF5FAF6D970E
:109D300080E00E94D05F39AD315039AF332309F450
:109D400044C02D8D3E8D4F8D58A165966CAD7DAD77
:109D50008EAD9FAD65970F9434456B017C0129A1B1
:109D600039A5A1016DA17EA18FA198A50F943445BD
:109D7000A70196010F94F9487B018C0129A139A50F
:109D8000A10165966CAD7DAD8EAD9FAD65970F94CD
:109D900034454B015C012D8D3E8D4F8D58A16DA139
:109DA0007EA18FA198A50F9434459B01AC01C501FC
:109DB000B4010F94F84869A379A71C01C701D80121
:109DC0008D8F9E8FAF8FB8A350C04DA95EA9BA01E9
:109DD00080E090E00F94D3442DA13EA14FA158A55F
:109DE0000F9434454B015C010F94D2496B017C0107
:109DF000C501B4010F94A84B4B015C01A70196016A
:109E0000698D7A8D8B8D9C8D0F9434452B013C018F
:109E1000A50194016DA57EA58FA598A90F94344541
:109E2000A30192010F94F94869A379A71C01A50128
:109E30009401698D7A8D8B8D9C8D0F9434454B01E7
:109E40005C01A70196016DA57EA58FA598A90F9429
:109E500034459B01AC01C501B4010F94F8486D8FE6
:109E60007E8F8F8F98A359E159AF29A139A5A10100
:109E70002D966CAD7DAD8EAD9FAD2D970F94F948AD
:109E800069837A838B839C832D8D3E8D4F8D58A162
:109E900061966CAD7DAD8EAD9FAD61970F94F94825
:109EA0006D837E838F839887A1962CAD3DAD4EAD9B
:109EB0005FADA19769857A858B859C850F94F9485C
:109EC00069877A878B879C87A5962CAD3DAD4EAD73
:109ED0005FADA5976D857E858F8598890F94F9482C
:109EE0006D877E878F87988B80914C02882321F025
:109EF000CE0101960E94BC74CE0101960E949E661E
:109F000080E090E0A0E8BFE38D8B9E8BAF8BB88F95
:109F10001091F00C21962CAD3DAD4EAD5FAD21976B
:109F20006091660D7091670D8091680D9091690D3B
:109F30000F94F8482B013C0125962CAD3DAD4EAD5C
:109F40005FAD259760916A0D70916B0D80916C0DDE
:109F500090916D0D0F94F8484B015C0129962CAD42
:109F60003DAD4EAD5FAD299760916E0D70916F0D57
:109F70008091700D9091710D0F94F8486B017C01E8
:109F8000A3019201C301B2010F9434452B013C019E
:109F9000A5019401C501B4010F9434459B01AC01A6
:109FA000C301B2010F94F9484B015C01A70196016E
:109FB000C701B6010F9434459B01AC01C501B40142
:109FC0000F94F9480F94B24B9B01AC0169966CADAC
:109FD0007DAD8EAD9FAD69970F943445698B7A8BBB
:109FE0008B8B9C8BDE0155966D01E12E8E010F5EF1
:109FF0001F4F9E01235F3F4F4EE65DE06AE67DE026
:10A0000086E69DE00E9437AD882389F12091660D98
:10A010003091670D4091680D5091690D21962CAFDC
:10A020003DAF4EAF5FAF219780916A0D90916B0D60
:10A03000A0916C0DB0916D0D25968CAF9DAFAEAF1C
:10A04000BFAF259720916E0D30916F0D4091700D2F
:10A050005091710D29962CAF3DAF4EAF5FAF299750
:10A060004DA95EA94F5F5F4F5EAB4DAB39CE8DE41E
:10A0700093E10E949E6621962CAD3DAD4EAD5FAD45
:10A0800021976091660D7091670D8091680D909198
:10A09000690D0F94F8482B013C0125962CAD3DAD80
:10A0A0004EAD5FAD259760916A0D70916B0D8091FB
:10A0B0006C0D90916D0D0F94F8484B015C01299641
:10A0C0002CAD3DAD4EAD5FAD299760916E0D709199
:10A0D0006F0D8091700D9091710D0F94F8486B0188
:10A0E0007C01A3019201C301B2010F9434452B01FD
:10A0F0003C01A5019401C501B4010F9434459B01B5
:10A10000AC01C301B2010F94F9484B015C01A701F6
:10A110009601C701B6010F9434459B01AC01C501FE
:10A12000B4010F94F9486B017C0120E030E0A901F3
:10A130000F94CF44882369F180E090E0A0E8BFE36A
:10A140008D8B9E8BAF8BB88F1091F00CC701B60131
:10A150000F94B24B9B01AC0169966CAD7DAD8EAD99
:10A160009FAD69970F943445698B7A8B8B8B9C8B51
:10A17000CE0145966C01E12E8E010F5E1F4F29E541
:10A1800033E14EE65DE06AE67DE086E69DE00E9412
:10A1900037AD80E1EDE4F3E1A6E5BDE001900D927D
:10A1A0008A95E1F718C0E8E7FBE284918F010F5F21
:10A1B0001F4F882321F00E949C5BF801F6CFEDEB46
:10A1C000F9E084918F010F5F1F4F882321F00E94D7
:10A1D0009C5BF801F6CFCC59DF4F0FB6F894DEBF89
:10A1E0000FBECDBFDF91CF911F910F91FF90EF90E8
:10A1F000DF90CF90BF90AF909F908F907F906F90A7
:10A200005F904F903F902F900895809153039091CD
:10A210005403A0915503B09156038093010290938B
:10A220000202A0930302B093040280915103909123
:10A230005203909355028093540208958091010235
:10A2400090910202A0910302B09104028093530303
:10A2500090935403A0935503B093560380915402F6
:10A2600090915502909352038093510384E690E0BD
:10A2700090935502809354020895CF92DF92EF920B
:10A28000FF920F931F936A01E0905E0DF0905F0DB7
:10A290000091600D1091610DFB012081318142819F
:10A2A0005381FC0160817181828193810E94EF461C
:10A2B0001F910F91FF90EF90DF90CF900895CF9274
:10A2C000DF92EF92FF920F931F936B01FC01E080EE
:10A2D000F18002811381E6E5FDE02481358146812C
:10A2E000578160817181828193810E94EF461F9125
:10A2F0000F91FF90EF90DF90CF900895BF92CF9293
:10A30000DF92EF92FF920F931F93CF93DF93CDB71E
:10A31000DEB728970FB6F894DEBF0FBECDBF909181
:10A32000770A981709F47AC0B82E882309F453C025
:10A3300080E090E0A0E2B1E48D839E83AF83B88794
:10A34000C0902A0CD0902B0CE0902C0CF0902D0C8F
:10A3500020E030E0A901C701B6010F94CF4487FF88
:10A360000CC0A701960160E070E080E291E40F94D8
:10A37000F8486D837E838F83988720E030E040EA41
:10A3800053E46D817E818F8198850F946D4B1816F3
:10A3900044F480E090E0A0EAB3E48D839E83AF8331
:10A3A000B8872D813E814F81588560915E0D7091F7
:10A3B0005F0D8091600D9091610D0F94CF4487FFE8
:10A3C0000AC019821A821B821C82BE016F5F7F4FF6
:10A3D000CE01059674DF6091560D7091570D8091F6
:10A3E000580D9091590D20915A0D30915B0D40916F
:10A3F0005C0D50915D0D19821A821B821C82E090C7
:10A400005E0DF0905F0D0091600D1091610DFE01E9
:10A4100031966F010E94EF46B092770A80E028964D
:10A420000FB6F894DEBF0FBECDBFDF91CF911F9165
:10A430000F91FF90EF90DF90CF90BF9008952F92F3
:10A440003F924F925F926F927F928F929F92AF92C4
:10A45000BF92CF92DF92EF92FF920F931F93CF9311
:10A46000DF93CDB7DEB7A4970FB6F894DEBF0FBE6B
:10A47000CDBF1C017BA36AA3498F2CA3DC018D9067
:10A480009D90AD90BC90FB014080518062807380B4
:10A49000A5019401C501B401002311F10F943445C5
:10A4A0006B017C01A3019201C301B2010F943445F9
:10A4B0009B01AC01C701B6010F94F9486B017C0107
:10A4C00020E030E442E556E40F94CF4418160CF433
:10A4D00018C220E030E94FE256E4C701B60114C0CB
:10A4E0000F9434456B017C01A3019201C301B201B9
:10A4F0000F9434459B01AC01C701B6010F94F94894
:10A5000020E030E442E556E40F94CF4418160CF4F2
:10A51000F8C1D0904802E0904902C0904A021091E0
:10A520004B02F0915E0DFA8F80915F0D8B8F9091B1
:10A53000600D9C8FA091610DAD8F2F2F382F492F6B
:10A540005A2F6D2D7E2D8C2D912F0F946D4B18163B
:10A5500024F0DA8EEB8ECC8E1D8F809101029091CB
:10A560000202A0910302B09104028E8F9F8FA8A3D4
:10A57000B9A38091070290910802A0910902B091BD
:10A580000A028093010290930202A0930302B09307
:10A59000040219821A821B821C82DE0111966D014F
:10A5A000EA8CFB8C0C8D1D8DA3019201C501B401B9
:10A5B0000E94EF4681E0A2DE81111AC18091760AE5
:10A5C00082FF11C020912A0C30912B0C40912C0C51
:10A5D00050912D0C60E070E080E090EC0F94F84812
:10A5E0002B013C0106C0412C512C20E2622E21ECB3
:10A5F000722E80902A0C90902B0CA0902C0CB09076
:10A600002D0C20E030E0A901C501B4010F94CF4426
:10A6100087FF0BC0A501940160E070E080E791E442
:10A620000F94F8484B015C0106C0812C912C90E7F7
:10A63000A92E91E4B92EA501940160915E0D70914F
:10A640005F0D8091600D9091610D0F946D4B181608
:10A650000CF04DC08D869E86AF86B88A812C912CD9
:10A6600088E4A82E82E4B82E89869A86AB86BC86BA
:10A67000BE01675F7F4FCE010D9621DE10917D0AEE
:10A6800010927D0A0E9461638AEB94E00F941C2B68
:10A690008091C2049091C304A091C404B091C504F8
:10A6A00080935E0D90935F0DA093600DB093610D4C
:10A6B00022D712FF1CC089829A82AB82BC8220E022
:10A6C00030E040EA50E460915E0D70915F0D809142
:10A6D000600D9091610D0F94F9486D837E838F8397
:10A6E0009887BE016F5F7F4FCE010596E8DD4D82F2
:10A6F0005E826F82788685E595E5A5E0B1E4898381
:10A700009A83AB83BC83BE016F5F7F4FCE010596FA
:10A71000D6DD10917D0A10927D0A0E9461638AEB5A
:10A7200094E00F941C2B8091C2049091C304A091DB
:10A73000C404B091C50480935E0D90935F0DA09307
:10A74000600DB093610DD7D612FF09C060915E0D08
:10A7500070915F0D8091600D9091610D04C060E07B
:10A7600070E080EC9FE720912A0C30912B0C4091F7
:10A770002C0C50912D0C0F94F9484B018C01898DB4
:10A780008250823048F580E090E0A8E4B2E48D8BFE
:10A790009E8BAF8BB88F20915E0D30915F0D4091F5
:10A7A000600D5091610DB98DB33029F060E070E01B
:10A7B00080EA90E404C060E070E088EC91E40F94DB
:10A7C000F948698B7A8B8B8B9C8BBE016B5E7F4FBC
:10A7D000CE01419674DD07C0E98DE13021F480E0BF
:10A7E0008DDD811105C0FCA1F33008F459C008C00B
:10A7F0009CA1933008F48AC0812C912C00EC1FE7B7
:10A80000E5EBF9E084915F019FEFA91AB90A88236B
:10A8100019F092D7F501F6CF2091D60C3091D70CD4
:10A820004091D80C5091D90CD1016D917D918D91B1
:10A830009C910F94F94843E00E94C55EE0EBF9E07B
:10A8400084915F01BFEFAB1ABB0A882319F074D75C
:10A85000F501F6CF2091DA0C3091DB0C4091DC0C45
:10A860005091DD0CEAA1FBA160817181828193810D
:10A870000F94F94843E00E94C55EEBEAF9E0849149
:10A880005F019FEFA91AB90A882319F055D7F5017E
:10A89000F6CF43E0B401C8010E94C55E8AE04CD700
:10A8A0008E8D9F8DA8A1B9A1809301029093020281
:10A8B000A0930302B09304029401A801B401C8015B
:10A8C0000F94F34B882399F160E08CE999E00E94A2
:10A8D0009288E8E7FBE284917F019FEFE91AF90A89
:10A8E000882319F029D7F701F6CFECE8F9E0849135
:10A8F0007F01AFEFEA1AFA0A8823C9F01DD7F701E2
:10A90000F6CF812C912C00EC1FE711C08E8D9F8D0E
:10A91000A8A1B9A18093010290930202A09303021F
:10A92000B0930402812C912C00EC1FE7CDCFB40131
:10A93000C801A4960FB6F894DEBF0FBECDBFDF915D
:10A94000CF911F910F91FF90EF90DF90CF90BF902C
:10A95000AF909F908F907F906F905F904F903F90BF
:10A960002F9008952F923F924F925F926F927F9215
:10A970008F929F92AF92BF92CF92DF92EF92FF920F
:10A980000F931F93CF93DF93CDB7DEB72C970FB6FE
:10A99000F894DEBF0FBECDBFB82E84E0B89E800114
:10A9A0001124F801E25BF64F85919591A591B49140
:10A9B000F801E65CFD4F80839183A283B38382E03C
:10A9C000B81215C020912A0C30912B0C40912C0C00
:10A9D00050912D0C6091260C7091270C8091280CC1
:10A9E0009091290C0F94F8486B017C0109C0F80183
:10A9F000E65AF64F85919591A591B4916C017D0130
:10AA0000F801E25DFD4FC601D70180839183A283E7
:10AA1000B38381E08B1528F482E0B81609F463C093
:10AA2000ADC0A0903202B090330200913402109178
:10AA3000350260902E0270902F028090300290902C
:10AA4000310220903E0230903F02409040025090F0
:10AA50004102C0903A02D0903B02E0903C02F0905C
:10AA60003D02A7019601B101C2010F94CF4487FDB9
:10AA700002C06101720120E030E0A901C701B60106
:10AA80000F946D4B87FF04C0F7FAF094F7F8F09439
:10AA9000A7019601B301C4010F946D4B181614F071
:10AAA00063017401A7019601B501C8010F946D4BB4
:10AAB000181614F065017801C092B204D092B30464
:10AAC000E092B404F092B504A7019601C701B60163
:10AAD0000F9434456093B6047093B7048093B80420
:10AAE0009093B9044BC019821A821B821C821D826A
:10AAF0001E821F82188619861A861B861C86CE0126
:10AB000001960E949E668090660D9090670DA090C1
:10AB1000680DB090690D80E090E0A8EEB2E48D83FE
:10AB20009E83AF83B887CE0101960E949E662091D6
:10AB3000660D3091670D4091680D5091690DC5010A
:10AB4000B4010F94F8484B015C0120E030E0A9010A
:10AB50000F946D4B87FF04C0B7FAB094B7F8B09468
:10AB6000A5019401B601C7010F94F848609348020B
:10AB70007093490280934A0290934B022C960FB631
:10AB8000F894DEBF0FBECDBFDF91CF911F910F9123
:10AB9000FF90EF90DF90CF90BF90AF909F908F90FD
:10ABA0007F906F905F904F903F902F900895EF921D
:10ABB000FF920F931F93CF93DF937C0184E596D58B
:10ABC000D82F882329F1F6D4C82F1816ECF4E2E523
:10ABD000FFE284918F010F5F1F4F882319F0ACD5DE
:10ABE000F801F7CF8DE4A8D5B70180E090E04AE006
:10ABF0000E94405E6C2FCC0F770B8BE399E00E9494
:10AC000085C38AE099D508C080933A0AD0E004C091
:10AC10008091F00C80933A0A8D2FDF91CF911F9194
:10AC20000F91FF90EF90089590917C0AE92FF0E04A
:10AC3000E858F54F80839F5F943018F490937C0A16
:10AC400002C010927C0A8091FF0B8F5F8093FF0BF4
:10AC50000895089580E090E00895809159049091BE
:10AC60005A04981759F0E92FF0E0E752FC4F808121
:10AC70009F5F9F7790935A0490E008958FEF9FEF26
:10AC80000895CF93FC0120812B33A1F02091FF0B7D
:10AC9000243080F4C62FBC0180917C0AF0E68F9F9F
:10ACA000C00111248258954F0F94C04C8C2FBCDFEB
:10ACB00081E001C080E0CF9108952F923F924F92A2
:10ACC0005F926F927F928F929F92AF92BF92CF923C
:10ACD000DF92EF92FF920F931F93CF93DF9300D0F9
:10ACE00000D0CDB7DEB79A8389830F94D20EE98165
:10ACF000FA81C680D780E084F184C114D104E104D4
:10AD0000F10409F0ACC22485222309F469C3328519
:10AD10002150248721E0230F22874585241301C079
:10AD20001286E981FA8124E0329FE00DF11D1124A1
:10AD3000C684D784E088F188E981FA81C282D3820F
:10AD4000E482F582DC01CB018C0D9D1DA11DB11D9E
:10AD500086839783A087B18784819581892B09F4A5
:10AD60003FC3FFB7FD83F894E981FA8122803380E5
:10AD70002101612C712C048115818091140285328E
:10AD800021F08F3F09F068C205C0E7E4F1E22491A9
:10AD90002E83DAC085E280931402E7E4F1E2849125
:10ADA0008E838F3F09F458C2823009F469C030F5B0
:10ADB000882309F44CC0813009F0C6C0109280008D
:10ADC0001092810080918100886080938100809141
:10ADD0008100816080938100EAE9F0E2E491F0E093
:10ADE000EE0FFF1FEF5BFF4D85919491E0EEF0E2D7
:10ADF000E491E0935C03E1E0EE8330C19E81943006
:10AE000009F482C008F460C0953009F09DC010922A
:10AE100020011092210180912101886080932101FD
:10AE200080912101816080932101EAE9F0E2E491BF
:10AE3000F0E0EE0FFF1FEF5BFF4D85919491E0EE88
:10AE4000F0E2E491E093590395E09E8307C114BCBE
:10AE500015BC84B5826084BD85B5816085BDEAE995
:10AE6000F0E2E491F0E0EE0FFF1FEF5BFF4D859104
:10AE70009491E0EEF0E2E491E0935D031E82ABC2B8
:10AE80001092B0001092B1008091B0008260809367
:10AE9000B0008091B10081608093B100EAE9F0E2F6
:10AEA000E491F0E0EE0FFF1FEF5BFF4D8591949171
:10AEB0009093670A8093660AE0EEF0E2E491E093F3
:10AEC000680AF2E0FE8387C210929000109291000F
:10AED00080919100886080939100809191008160C1
:10AEE00080939100EAE9F0E2E491F0E0EE0FFF1FB9
:10AEF000EF5BFF4D85919491E0EEF0E2E491E093F9
:10AF00005B0323E02E83AAC01092A0001092A10040
:10AF10008091A10088608093A1008091A100816050
:10AF20008093A100EAE9F0E2E491F0E0EE0FFF1F68
:10AF3000EF5BFF4D85919491E0EEF0E2E491E093B8
:10AF40005A0384E08E838AC0EE81E7FD85C161E00B
:10AF500085E20F94960D8E818D7F09F083C04801A4
:10AF6000A12CB12C60E072E18AE790E0A501940188
:10AF70000F94424C29833A834B835C8369017A01A5
:10AF8000F1E0CF1AD108E108F1082FEFC216D10481
:10AF9000E104F10409F008F44EC060E472E48FE0CB
:10AFA00090E0A50194010F94424C69017A0181E07F
:10AFB000C81AD108E108F1089E81923009F5EFEF37
:10AFC000CE16D104E104F10409F008F4CBC160E924
:10AFD00070ED83E090E0A50194010F94424C69016B
:10AFE0007A01F1E0CF1AD108E108F1082FEFC2167B
:10AFF000D104E104F10411F008F041C183E027C05D
:10B000008FEFC816D104E104F104B9F0B0F068E4A0
:10B0100078EE81E090E0A50194010F94424C690123
:10B020007A0191E0C91AD108E108F108EE81EE2316
:10B0300009F49AC163C181E001C082E09E8191114F
:10B0400006C095B5987F892B85BD7AC085E0909123
:10B05000B100987F892B8093B10072C061E085E2D6
:10B060000F94960D4801A12CB12C60E072E18AE7A3
:10B0700090E0A50194010F94424C69017A01E1E04E
:10B08000CE1AD108E108F108C114D104F1E0EF06AD
:10B09000F10488F068E478EE81E090E0A501940185
:10B0A0000F94424C69017A0181E0C81AD108E10885
:10B0B000F10883E001C081E09E81913071F49091AC
:10B0C0008100987F892B8093810045284628472856
:10B0D000D9F52FEF3FEFA90168C0EE81E33071F49D
:10B0E00090919100987F892B809391004528462864
:10B0F000472851F52FEF3FEFA90179C0FE81F430C9
:10B1000071F49091A100987F892B8093A10045282C
:10B1100046284728C9F42FEF3FEFA9017AC02E81B6
:10B12000253071F490912101987F892B8093210122
:10B1300045284628472841F42FEF3FEFA9017BC05F
:10B1400045284628472869F0D801AA0FBB1F91015E
:10B150000F94E94828EE33E040E050E00F94BD48FA
:10B1600003C02FEF3FEFA9018E81823081F12CF4D3
:10B17000882361F08130C9F06FC09E81943009F45A
:10B1800048C0ACF1953009F456C066C0C7BC2093E6
:10B190006E0330936F03409370035093710380915B
:10B1A0006E00826080936E0057C0D0928900C0927A
:10B1B000880020936A0330936B0340936C03509391
:10B1C0006D0380916F00826080936F0045C0C092D4
:10B1D000B3002093690A30936A0A40936B0A509334
:10B1E0006C0A8091700082608093700035C0D092AC
:10B1F0009900C092980020936603309367034093B0
:10B20000680350936903809171008260809371009C
:10B2100023C0D092A900C092A8002093620330936B
:10B2200063034093640350936503809172008260CE
:10B230008093720011C0D0922901C09228012093FE
:10B240005E0330935F0340936003509361038091EA
:10B250007300826080937300ED81EFBFC1C0DC0199
:10B26000CB018C199D09AE09BF09B7FDB9C0409843
:10B27000E981FA811682178210861186B1C068E4CE
:10B2800078EE81E090E0A50194010F94424C6901B1
:10B290007A01F1E0CF1AD108E108F1082FEFC216C8
:10B2A000D104E104F10441F138F164E274EF80E08B
:10B2B00090E0A50194010F94424C69017A01F1E0FC
:10B2C000CF1AD108E108F1082FEFC216D104E1042A
:10B2D000F10409F008F4BACE62E17AE780E090E088
:10B2E000A50194010F94424C69017A0181E0C81ACA
:10B2F000D108E108F10819C084E0A9CE2FEFC216E9
:10B30000D104E104F10409F008F463C062E17AE7D2
:10B3100080E090E0A50194010F94424C69017A010C
:10B32000F1E0CF1AD108E108F1082FEFC216D104DD
:10B33000E104F104A9F0A0F089819A81AB81BC817C
:10B340002AE0B595A795979587952A95D1F76C0131
:10B350007D01F1E0CF1AD108E108F10887E077CE4E
:10B3600086E075CE82E073CEEFEFCE16D104E10415
:10B37000F10469F160F162E17AE780E090E0A50113
:10B3800094010F94424C69017A0181E0C81AD108F6
:10B39000E108F1089FEFC916D104E104F104A9F016
:10B3A000A0F089819A81AB81BC813AE0B595A795DF
:10B3B000979587953A95D1F76C017D01E1E0CE1A1A
:10B3C000D108E108F10885E03CCE84E03ACE83E084
:10B3D00038CE84E033CE61E085E20F94960DBFCD88
:10B3E00026960FB6F894DEBF0FBECDBFDF91CF918A
:10B3F0001F910F91FF90EF90DF90CF90BF90AF9093
:10B400009F908F907F906F905F904F903F902F9084
:10B410000895CF93DF93EC0160E0CE0132DC81111F
:10B4200003C080E0BDD5F8CFCE010E942C768823E2
:10B43000C1F3DF91CF910895DF92EF92FF920F93C6
:10B440001F93CF93DF93CDB7DEB76E970FB6F89407
:10B45000DEBF0FBECDBF60914413709145136115DF
:10B46000710501F14DE150E0CE0101967C010F9490
:10B4700040441E8EF7018F010E191F09D190DD2067
:10B4800019F09AE0D912F7CFF701E00FF11F1082FF
:10B4900060E0C701F6DB882329F0C7010E942C7603
:10B4A000811109C081E02091441330914513232B71
:10B4B000A1F480E012C0DD2049F00F5F1F4F8091A2
:10B4C000441390914513080F191F02C000E010E0CB
:10B4D0001093451300934413E5CF6E960FB6F8947E
:10B4E000DEBF0FBECDBFDF91CF911F910F91FF90B7
:10B4F000EF90DF9008950C9496F80F931F93CF93DD
:10B50000DF93CDB7DEB72C970FB6F894DEBF0FBE32
:10B51000CDBFE6E5FDE080859185A285B3854481B8
:10B520005581668177810081118122813381098370
:10B530001A832B833C834D835E836F83788789874F
:10B540009A87AB87BC8722E63DE0AE01475F5F4F3D
:10B55000BE016B5F7F4FCE0101960E9467C42C969F
:10B560000FB6F894DEBF0FBECDBFDF91CF911F9114
:10B570000F9108958091570390915803009731F0EF
:10B580004AE050E060E070E00D94064360E070E057
:10B59000CB0108958091570390915803009731F0A3
:10B5A0004AE050E060E070E00D94DB4160E070E064
:10B5B000CB010895EFDF97FD0AC0ECDF6F3F710507
:10B5C0008105910509F02CF4E5DF862F089580E0D0
:10B5D00008958FEF08958091570390915803892B18
:10B5E00031F0E8DF91E0811103C090E001C091E00B
:10B5F000892F08950F931F93CF93809157039091B4
:10B6000058030097F1F0FC018F01C1912C2F2F7D81
:10B6100089F0C53411F0C536B9F7F801108260E041
:10B6200070E00F948840F801C083562F472F382FC1
:10B63000292F0BC060E070E0CF911F910F910D9406
:10B64000884050E040E030E020E0652F742F832FE9
:10B65000922FCF911F910F91089581548A3108F054
:10B6600042C0E82FF0E040919413509195136091FF
:10B6700096137091971304C07695679557954795E3
:10B680008A95D2F7842F817040FF2FC0E658FC4E78
:10B690009081992309F1E0914713F0914813E90F44
:10B6A000F11D908120ED290F2A3098F09E3211F47F
:10B6B00091810CC09D3211F09B3271F4918120ED8B
:10B6C000290F2A3030F09E3239F4928190539A300B
:10B6D00018F42E2F9F2F02C020E090E020935703F4
:10B6E00090935803089580E008950895B6DF882365
:10B6F00041F081E02091570330915803232B09F446
:10B7000080E00895FC01238121110C948B6E089533
:10B7100080E1E6E5FDE0ADE4B3E101900D928A95AC
:10B72000E1F7089580E1EDE4F3E1A6E5BDE00190E5
:10B730000D928A95E1F708959091C00095FFFCCF96
:10B740008093C60008953F924F925F926F927F92CE
:10B750008F929F92AF92BF92CF92DF92EF92FF9221
:10B760000F931F93CF93DF931F92CDB7DEB764DEA5
:10B77000811173C28091FF0B843008F047C06DDAED
:10B78000AC0197FF7CC142C08E3409F0D9C10115CC
:10B79000110509F4D5C163E07BE0C8010F944F4463
:10B7A0007C01892B09F48EC16EE470E0C801049617
:10B7B0000F94AC4C009709F485C14AE050E060E07A
:10B7C00070E001960F94DB416093720370937303F2
:10B7D000809374039093750380907F0F9090800FF7
:10B7E000A090810FB090820F2FEF821A920AA20AC6
:10B7F000B20A681579058A059B0509F465C1EF2829
:10B8000009F062C180ED9AE00E94EDF6809122106D
:10B81000882309F422C28091FF0B811102C010928B
:10B82000D803EE24E3944091C3125091C412609166
:10B83000C5127091C6128091BF129091C012A09152
:10B84000C112B091C212481759076A077B0708F462
:10B85000E12C00E010E09924939480E6882E98E093
:10B86000A92E9BE0B92E2DE8322E8091FF0B84305B
:10B8700008F0F3C1E110F1C18091D8038111EDC14D
:10B8800080911A1290911B12A0911C12B0911D125E
:10B890008093C3129093C412A093C512B093C612A2
:10B8A00041E050E0BE016F5F7F4F82E192E10E9474
:10B8B0007B71019719F4898190E002C08FEF9FEFAF
:10B8C000F82E4090C3125090C4126090C512709030
:10B8D000C6124091BF125091C0126091C112709176
:10B8E000C212EE24E394441655066606770608F461
:10B8F000E12C4416550666067706B0F4019609F465
:10B900006AC08AE0F81609F489C09DE0F91609F4C6
:10B9100085C023E2F21619F08AE3F81296C08091EE
:10B92000D703811192C06FC00E9443BB82E192E1B4
:10B930000E948B6E80912D12882359F18150809343
:10B940002D12389EC001112441E061E08E5C9D4EB5
:10B950000E943BF5E0912D1294E0E99FF001112443
:10B96000E25DFD4E40815181628173814093C3123B
:10B970005093C4126093C5127093C61282E192E193
:10B980000F94921D809123108823A9F09092221089
:10B9900012C0109222100E9481BB0E94C6E50E9434
:10B9A00040E56D3371058105910528F0B09245138E
:10B9B000A092441341DD80912210811128C0EBE157
:10B9C000FBE084916F012FEFC21AD20A8823D9F0CD
:10B9D000B3DEF601F6CFE8E7FBE284916F019FEF5B
:10B9E000C91AD90A882319F0A7DEF601F6CFECE0D0
:10B9F000FBE084916F012FEFC21AD20A882319F05D
:10BA00009BDEF601F6CF83E2F81208C005C023E200
:10BA1000F21220C100E010E09092D8031092D703F8
:10BA20000115110519F40E94BEE80CC080917C0A32
:10BA3000889E000D111D1124F801E258F54F108267
:10BA400080E0F2D800E010E010CF0F35110508F0CB
:10BA50000CCF9BE3F91202C09092D7038091D703D9
:10BA6000811103CF80917C0AF801889EE00DF11DC1
:10BA70001124E258F54FF0820F5F1F4FF6CE982F3A
:10BA800020917D0F30917E0F8A3019F09D3009F0A2
:10BA9000B0C01092D6032115310519F40E94BEE8FA
:10BAA00069CEF901EA58FC4F108210927E0F109275
:10BAB0007D0F06E713E0F8018191803209F064CE32
:10BAC0008F01F9CFC80179CE6AE270E0C8010F9406
:10BAD000E44C9C01009701F1982F901BF12C9923C5
:10BAE00039F09150F801E90FF11D8081F826F7CF68
:10BAF0004AE050E060E070E0C90101960F94DB413C
:10BB0000CF2CD12CE12CF12C6C157D058E059F05D9
:10BB100031F081EB9AE078CE87E89AE075CE80919B
:10BB2000720390917303A0917403B0917503809395
:10BB30007F0F9093800FA093810FB093820F0EC060
:10BB400080912010882351F06EE273E0C8010F94B9
:10BB5000B74C892B19F08DE59AE056CE80912A02D8
:10BB6000811124C067E470E0C8010F94AC4C0097C9
:10BB7000E9F04AE050E060E070E001960F94DB41AC
:10BB8000643071058105910588F4E6EEF9E0849151
:10BB90007F019FEFE91AF90A882319F0CDDDF7013B
:10BBA000F6CF60E08CED99E00E94928862E373E04A
:10BBB000C8010F94B74C892B21F410921B021092EC
:10BBC000EE0C67E373E0C8010F94B74C892B19F4AE
:10BBD00083ED99E095D16CE373E0C8010F94B74C05
:10BBE000892B11F40E94A5A561E086E793E049D86E
:10BBF000C1CD2F3531050CF0BDCD9C35B9F42DD814
:10BC000097FDB8CD2091D6032111B4CD20917D0FA1
:10BC100030917E0FA9014F5F5F4F50937E0F40938D
:10BC20007D0FF901EA58FC4F8083A4CD9B3319F4B2
:10BC300081E08093D6038091D60381119BCDC90109
:10BC4000019690937E0F80937D0FF901EA58FC4F87
:10BC5000408390CD1092D703E6CE0F90DF91CF9125
:10BC60001F910F91FF90EF90DF90CF90BF90AF901A
:10BC70009F908F907F906F905F904F903F9008952E
:10BC80008F929F92AF92BF92EF92FF920F931F936A
:10BC9000CF93DF93CDB7DEB7A0970FB6F894DEBF92
:10BCA0000FBECDBF611571058105910589F100E0D9
:10BCB000842E912CA12CB12C102FEE24E394F12C86
:10BCC000EC0EFD1EE00EF11C07FDFA94A501940197
:10BCD0000F94BD48F7016083B901CA010F5F611578
:10BCE00071058105910541F71F3F21F1E1E0F0E089
:10BCF000EC0FFD1FE10FF11D17FDFA9580818A30D1
:10BD000010F097E301C090E3890F16DD1150ECCFDE
:10BD100080E3A0960FB6F894DEBF0FBECDBFDF91D3
:10BD2000CF911F910F91FF90EF90BF90AF909F9098
:10BD30008F9002CDA0960FB6F894DEBF0FBECDBF98
:10BD4000DF91CF911F910F91FF90EF90BF90AF9037
:10BD50009F908F900895CF92DF92EF92FF926B01A8
:10BD60007C0197FF0AC08DE2E7DCF094E094D09468
:10BD7000C094C11CD11CE11CF11C4AE0C701B601F2
:10BD8000FF90EF90DF90CF907BCF8F929F92AF92FA
:10BD9000BF92CF92DF92EF92FF92CF936B017C0123
:10BDA000B42E20E030E0A9010F94CF4487FF06C0F5
:10BDB0008DE2C2DCF7FAF094F7F8F094C0E060E0AE
:10BDC00070E080E09FE3CB1541F02DEC3CEC4CECB7
:10BDD0005DE30F943445CF5FF6CF9B01AC01C70103
:10BDE000B6010F94F9486B017C010F94424A4B0154
:10BDF0005C014AE045DFCC2379F1C501B4010F9421
:10BE0000D3449B01AC01C701B6010F94F8486B0104
:10BE10007C018EE291DC20E030E040E251E4C70199
:10BE2000B6010F9434454B015C010F943D4A6B0100
:10BE3000770FEE08FF08C701B6018DDFC701B60115
:10BE40000F94D5449B01AC01C501B4010F94F8488F
:10BE50006B017C01C150F9F6CF91FF90EF90DF901C
:10BE6000CF90BF90AF909F908F9008951F920F92A8
:10BE70000FB60F9211240BB60F922F938F939F93AF
:10BE8000EF93FF9320915A04E091590481E08E0FC3
:10BE90008F779091C600281729F0F0E0E752FC4F09
:10BEA0009083E82FE0935904FF91EF919F918F9138
:10BEB0002F910F900BBE0F900FBE0F901F901895F3
:10BEC00025E033E0FC013183208304961BCC5F9A8C
:10BED0008091760A8E7F8093760A8A9A8091760A7C
:10BEE0008D7F8093760A8091080180958170809380
:10BEF00006018091760A8B7F8093760A129A0895C4
:10BF00008C01E8E7FBE28491EF012196882319F088
:10BF100013DCFE01F8CFEEE3FCE08491EF01219603
:10BF2000882319F009DCFE01F8CF0E94DBE5CFDFA2
:10BF30000E94318C61E0C8010E9492880E944EC626
:10BF400060E080E00F94A90164E182EF9CE00E9430
:10BF500001C762E080E00F94A9018FE29CE00F949A
:10BF60008A0163E080E00F94A90182E29CE00F94D3
:10BF70008A012FEF8BE49DE1215080409040E1F752
:10BF800000C00000F8942FEF84E39CE02150804033
:10BF90009040E1F700C000000E94DBE5A895FECFCD
:10BFA0002F923F924F925F926F927F928F929F92C9
:10BFB000AF92BF92CF92DF92EF92FF920F931F93B7
:10BFC000CF93DF9300D01F92CDB7DEB7182F0E941A
:10BFD000F6880F94D20E6B017C01009100020023C1
:10BFE00009F475C08091EF0C882309F470C040916A
:10BFF0009C0450919D0460919E0470919F044601A1
:10C000005701841A950AA60AB70AB7FC72C0833092
:10C0100041F134F481300CF45AC0E2E5FFE206C08D
:10C02000843009F054C0E2E5FFE237C084919F01FB
:10C030002F5F3F4F3B832A83882321F07DDBEA81FA
:10C04000FB81F4CFE4EAFBE08491AF014F5F5F4FE7
:10C050005B834A83882309F43AC06EDBEA81FB8163
:10C06000F3CFE2E5FFE284919F012F5F3F4F3B83D7
:10C070002A83882321F060DBEA81FB81F4CFEDE89D
:10C08000FBE08491AF014F5F5F4F5B834A8388235E
:10C09000F1F052DBEA81FB81F4CF84919F012F5FA5
:10C0A0003F4F3B832A83882321F046DBEA81FB81D3
:10C0B000F4CFE5E7FBE08491AF014F5F5F4F5B8317
:10C0C0004A83882321F038DBEA81FB81F4CF202FDB
:10C0D00030E0A8EEB3E00F94E948C60ED71EE81E84
:10C0E000F91EC0929C04D0929D04E0929E04F092AE
:10C0F0009F048091FF0B843008F425DB0F94D20E4F
:10C100008090630490906404A0906504B0906604ED
:10C1100081149104A104B10479F1C0905F04D0901E
:10C120006004E0906104F0906204C80CD91CEA1C21
:10C13000FB1C4B015C018C189D08AE08BF08B7FCC6
:10C140001BC0E8E7FBE284919F012F5F3F4F3B83D9
:10C150002A83882321F0F0DAEA81FB81F4CF609111
:10C1600047137091481388EE9BE00E949EC38AE0BB
:10C17000E3DA8FED9BE084C0C0905B04D0905C0458
:10C18000E0905D04F0905E04C114D104E104F10478
:10C1900009F441C03091A80F2091A90F321749F03E
:10C1A00060935F04709360048093610490936204D1
:10C1B00032C020918C0F21112EC011112CC0009182
:10C1C0005F041091600420916104309162040C0DB1
:10C1D0001D1D2E1D3F1DDC01CB01801B910BA20BF1
:10C1E000B30BB7FD18C05F9A8091760A8E7F80935B
:10C1F000760A8A9A8091760A8D7F8093760A80915A
:10C20000080180958170809306018091760A8B7F6A
:10C210008093760A129A8091B0049091B10490991B
:10C2200002C0019604C0181619062CF401979093C9
:10C23000B1048093B0048091B0049091B1048E3E1B
:10C240009240FCF0E8E7FBE28491AF014F5F5F4F63
:10C250005B834A83882321F06FDAEA81FB81F4CF84
:10C26000EFEBFBE084919F012F5F3F4F3B832A83DD
:10C27000882321F061DAEA81FB81F4CF86EB9BE031
:10C280003FDE0F94D20E0091A4041091A5042091DA
:10C29000A6043091A7044B015C01801A910AA20AFE
:10C2A000B30AB7FC4AC08B019C010C53164F2F4FA9
:10C2B0003F4F0093A4041093A5042093A604309349
:10C2C000A7044F9BDEC17A9BDCC12091060120FFB1
:10C2D000D8C12091390A2111D4C1029BD2C1009149
:10C2E000A0041091A1042091A2043091A30401158F
:10C2F00011052105310599F0DC01CB01801B910B63
:10C30000A20BB30B80569A4EA109B1098827B7FD3D
:10C3100083959927AA27BB27682F619501C060E004
:10C32000262F30E080910201611180958071809309
:10C330000001B90187E00F94D20D9091A80F809170
:10C34000A90F9817A1F0E091A90F2DE4E29FF00149
:10C350001124E859FA4F60818091A90F9091A80F9C
:10C36000981302C0698306C08F5F8F70F7CF8090EB
:10C37000421389829980992049F10F94D20E00913D
:10C38000AC041091AD042091AE043091AF04DC01F7
:10C39000CB01011511052105310579F48C599F4F09
:10C3A000AF4FBF4F8093AC049093AD04A093AE0405
:10C3B000B093AF042FEF298311C0801B910BA20B08
:10C3C000B30BB7FF0BC03FEF398308C01092AC042A
:10C3D0001092AD041092AE041092AF048980682DC3
:10C3E00070E089E00F94D20D8091470C882309F406
:10C3F000F9C00091260210912702909028029C8299
:10C40000A0902902AA826091DB047091DC046E5F27
:10C410007F4F072E000C880B990B0F94D544980181
:10C42000492D5A2D0F94CF4487FDDCC0F090A90F01
:10C43000212C312CE12C19828091A80F8F1509F441
:10C4400062C08F2D90E03DE4B32EB89EF001B99EFE
:10C45000F00D1124EF5DFA4F458956896789708D7B
:10C46000452B462B472B81F4418D528D638D748D66
:10C47000452B462B472B41F4458D568D678D70A17A
:10C48000452B462B472BD1F12DE4C22EC89E90019F
:10C49000C99E300D1124A9014F5D5A4F6A01FA015E
:10C4A00061817281838194810F94B24B4B015C0155
:10C4B000F60161A172A183A194A10F94D3442B0131
:10C4C0003C01F60165A176A187A190A50F94D34404
:10C4D0009B01AC01C301B2010F94D549A5019401A0
:10C4E0000F9434455B016C0191014E2D59810F94DD
:10C4F0006D4B18161CF41501EC2CD98281E08F0DC0
:10C500008F70F82E99CF20911E0230911F0240911A
:10C51000200250912102B1018E2D99810F94344552
:10C5200098014C815A810F94F9486B017C019B0161
:10C53000AC01B8018C819A810F946D4B1816ACF048
:10C540000091220210912302809024028C8290900C
:10C5500025029A829801A401B601C7010F946D4B80
:10C5600018161CF08601EC82FA82C090A804D090C4
:10C57000A904E090AA04F090AB0498014C815A8180
:10C58000C701B6010F946D4B1816D4F420E037EDB7
:10C5900043EA5CE3B8018C819A810F9434454B01E6
:10C5A0005C0128E431EE4AE75FE3C701B6010F946E
:10C5B0003445A50194010F94F9488B018C839A832B
:10C5C000C801AC81BA818093A8049093A904A09378
:10C5D000AA04B093AB04B801CD010F943D4ACB013E
:10C5E0000E9429880E94BEE882E090E10E945D5688
:10C5F000A0906B04A982AA2009F44CC00F94D20E1B
:10C6000000916704109168042091690430916A04D4
:10C61000DC01CB01801B910BA20BB30BB7FD3AC021
:10C620000F94D20E6B017C01B9802B2D30E0A8EE67
:10C63000B3E00F94E948C60ED71EE81EF91EC0925B
:10C640006704D0926804E0926904F0926A040E9440
:10C6500085CC8AE00F900F900F900F90DF91CF91D3
:10C660001F910F91FF90EF90DF90CF90BF90AF9010
:10C670009F908F907F906F905F904F903F902F9002
:10C680005BC86093A0047093A1048093A20490936C
:10C69000A30425CE0F900F900F900F90DF91CF91B4
:10C6A0001F910F91FF90EF90DF90CF90BF90AF90D0
:10C6B0009F908F907F906F905F904F903F902F90C2
:10C6C00008954F925F926F927F928F929F92AF9256
:10C6D000BF92CF92DF92EF92FF92CF93DF93CDB7CD
:10C6E000DEB7E4970FB6F894DEBF0FBECDBF82E091
:10C6F0000E9454BB69877A878B879C8781E00E9460
:10C7000054BB2B013C0180E00E9454BB6D8F7E8F97
:10C710008F8F98A3ACE6B4E08D919D910D90BC9164
:10C72000A02D89A39AA3ABA3BCA39C01AD016091EA
:10C7300074047091750480917604909177040F943D
:10C74000F8484B015C018091700490917104A091B4
:10C750007204B09173048DA39EA3AFA3B8A79C01EC
:10C76000AD01609178047091790480917A04909180
:10C770007B040F94F8486B017C012D8D3E8D4F8D0D
:10C7800058A1C301B2010F94F84869837A838B835F
:10C790009C83A5019401C501B4010F9434452B017C
:10C7A0003C01A7019601C701B6010F9434459B01D6
:10C7B000AC01C301B2010F94F9482B013C0129815E
:10C7C0003A814B815C81CA01B9010F9434459B01C8
:10C7D000AC01C301B2010F94F9486DA77EA78FA7E2
:10C7E00098AB0F94B24B9B01AC0160E070E080E825
:10C7F0009FE30F94D5496D837E838F8398879B0138
:10C80000AC01C501B4010F943445698B7A8B8B8BD5
:10C810009C8B2D813E814F815885C701B6010F94B5
:10C8200034456D8B7E8B8F8B988F2D813E814F8110
:10C83000588569817A818B819C810F943445698FF9
:10C840007A8F8B8F9C8F29A13AA14BA15CA160911B
:10C850007C0470917D0480917E0490917F040F94FC
:10C86000F8484B015C012DA13EA14FA158A5609154
:10C8700080047091810480918204909183040F94CC
:10C88000F8486B017C012D8D3E8D4F8D58A1698537
:10C890007A858B859C850F94F8486D877E878F8776
:10C8A000988BA501940169897A898B899C890F9459
:10C8B00034452B013C01A70196016D897E898F8942
:10C8C000988D0F9434459B01AC01C301B2010F94C4
:10C8D000F9482B013C012D853E854F855889698D8E
:10C8E0007A8D8B8D9C8D0F9434459B01AC01C301D7
:10C8F000B2010F94F94869837A838B839C839B01EF
:10C90000AC0169897A898B899C890F9434459B0194
:10C91000AC01C501B4010F94F84869877A878B8709
:10C920009C8729813A814B815C816D897E898F89C1
:10C93000988D0F9434459B01AC01C701B6010F944B
:10C94000F8484B015C0129813A814B815C81698DFA
:10C950007A8D8B8D9C8D0F9434459B01AC016D8538
:10C960007E858F8598890F94F8486B017C01298515
:10C970003A854B855C85CA01B9010F9434452B017A
:10C980003C01A5019401C501B4010F9434459B01FC
:10C99000AC01C301B2010F94F9482B013C01A7017E
:10C9A0009601C701B6010F9434459B01AC01C30148
:10C9B000B2010F94F94869AB7AAB8BAB9CAB0F9487
:10C9C000B24B9B01AC0160E070E080E89FE30F9404
:10C9D000D5492B013C019B01AC0169857A858B858A
:10C9E0009C850F94344569877A878B879C87A30140
:10C9F0009201C501B4010F9434456D877E878F87FE
:10CA0000988BA3019201C701B6010F94344569A721
:10CA10007AA78BA79CA7A4E8B4E0CD90DD90ED9019
:10CA2000FC90209188043091890440918A045091AF
:10CA30008B04C701B6010F94F8482DA53EA54FA55C
:10CA400058A90F94F9482D813E814F8158850F9444
:10CA5000344520E030E040E05FE30F9434456D83DF
:10CA60007E838F83988720918C0430918D04409130
:10CA70008E0450918F04C701B6010F94F8484B0102
:10CA80005C0129813A814B815C81CA01B9010F9413
:10CA900034459B01AC01C501B4010F94F94829A9A3
:10CAA0003AA94BA95CA90F94F94820E030E040E096
:10CAB0005FE30F9434454B015C012D813E814F8132
:10CAC000588569817A818B819C810F9434459B01C3
:10CAD000AC01C501B4010F94F848A30192010F9471
:10CAE00034454B015C012D813E814F815885CA013F
:10CAF000B9010F9434452B013C01A5019401C501F6
:10CB0000B4010F9434459B01AC01C301B2010F94F1
:10CB1000F9489B01AC01C701B6010F94F8480F9486
:10CB2000B24B69837A838B839C832D813E814F81B5
:10CB3000588569897A898B899C890F94344529A104
:10CB40003AA14BA15CA10F94F9486B017C01A501AE
:10CB5000940169857A858B859C850F9434459B016A
:10CB6000AC01C701B6010F94F9486B017C0129A5FE
:10CB70003AA54BA55CA56D897E898F89988D0F9408
:10CB800034452B013C012D853E854F855889698DA3
:10CB90007A8D8B8D9C8D0F9434459B01AC01C30124
:10CBA000B2010F94F84829813A814B815C810F943E
:10CBB00034459B01AC01C701B6010F94F848EAEB7C
:10CBC000F4E060837183828393832D813E814F8162
:10CBD00058856D897E898F89988D0F9434452DA154
:10CBE0003EA14FA158A50F94F9486B017C01A50106
:10CBF00094016D857E858F8598890F9434459B01BE
:10CC0000AC01C701B6010F94F9486B017C0129857D
:10CC10003A854B855C85698D7A8D8B8D9C8D0F94C3
:10CC200034452B013C0129A53AA54BA55CA5698992
:10CC30007A898B899C890F9434459B01AC01C3018F
:10CC4000B2010F94F84829813A814B815C810F949D
:10CC500034459B01AC01C701B6010F94F8486093BD
:10CC6000BE047093BF048093C0049093C1042D81CF
:10CC70003E814F815885698D7A8D8B8D9C8D0F9467
:10CC800034452D8D3E8D4F8D58A10F94F9486B0181
:10CC90007C01A501940169A57AA58BA59CA50F949B
:10CCA00034459B01AC01C701B6010F94F9486B01F3
:10CCB0007C012D853E854F85588969897A898B89C4
:10CCC0009C890F9434454B015C0129853A854B853D
:10CCD0005C856D897E898F89988D0F9434459B0181
:10CCE000AC01C501B4010F94F84829813A814B8108
:10CCF0005C810F9434459B01AC01C701B6010F94D0
:10CD0000F8486093C2047093C3048093C404909362
:10CD1000C504E4960FB6F894DEBF0FBECDBFDF9119
:10CD2000CF91FF90EF90DF90CF90BF90AF909F900A
:10CD30008F907F906F905F904F9008952F923F92C9
:10CD40004F925F926F927F928F929F92AF92BF921B
:10CD5000CF92DF92EF92FF920F931F93CF93DF93C7
:10CD600000D000D0CDB7DEB79E838D83DC0118964E
:10CD7000CD90DD90ED90FC901B970CE614E02D918A
:10CD80003D914D915C91F801608171818281938127
:10CD90000F94F8482B013C01AD81BE8114968D9112
:10CDA0009D910D90BC91A02D89839A83AB83BC8308
:10CDB0009C01AD01F80164817581868197810F9492
:10CDC000F8484B015C0184E8282E84E0382EA3014A
:10CDD0009201C301B2010F9434452B013C01A5011E
:10CDE0009401C501B4010F9434459B01AC01C3010A
:10CDF000B2010F94F9489B01AC01D1016D917D9175
:10CE00008D919C910F94F8480F94B24B9B01AC010B
:10CE1000C701B6010F94F948E6E6FDE0608371832F
:10CE200082839383AD81BE812D913D914D915C9123
:10CE3000F80160857185828593850F94F8484B01D0
:10CE40005C0129813A814B815C81D8011C966D91EE
:10CE50007D918D919C911F970F94F8482B013C0177
:10CE6000A5019401C501B4010F9434454B015C0147
:10CE7000A3019201C301B2010F9434459B01AC019F
:10CE8000C501B4010F94F9489B01AC01F101648123
:10CE90007581868197810F94F8480F94B24B9B015E
:10CEA000AC01C701B6010F94F94860936A0D709305
:10CEB0006B0D80936C0D90936D0DAD81BE812D91A6
:10CEC0003D914D915C91F8016089718982899389C6
:10CED0000F94F8484B015C01AD81BE8114962D91F1
:10CEE0003D914D915C911797F80164897589868908
:10CEF00097890F94F8482B013C01A5019401C501C5
:10CF0000B4010F9434454B015C01A3019201C301AC
:10CF1000B2010F9434459B01AC01C501B4010F94DB
:10CF2000F9489B01AC01D10118966D917D918D91CD
:10CF30009C911B970F94F8480F94B24B9B01AC0146
:10CF4000C701B6010F94F94860936E0D70936F0D91
:10CF50008093700D9093710D26960FB6F894DEBFF6
:10CF60000FBECDBFDF91CF911F910F91FF90EF903A
:10CF7000DF90CF90BF90AF909F908F907F906F90F9
:10CF80005F904F903F902F9008952F923F924F9235
:10CF90005F926F927F928F929F92AF92BF92CF9249
:10CFA000DF92EF92FF920F931F93CF93DF93CDB752
:10CFB000DEB7C854D1090FB6F894DEBF0FBECDBF9F
:10CFC00080914C02882321F08DE493E10E94BC748F
:10CFD0008091F70483FDA5C0C0905913D0905A13D7
:10CFE000E0905B13F0905C132091620D3091630D23
:10CFF0004091640D5091650DC701B6010F94CF4467
:10D00000882309F48EC080916D13811131C0609125
:10D010006E1370916F1380917013909171130F9430
:10D020003D4A2091590230915A026217730704F564
:10D03000C092620DD092630DE092640DF092650D86
:10D04000E2E5FFE284918F010F5F1F4F882321F0FB
:10D050000E949C5BF801F6CFEAE5FBE084918F012A
:10D060000F5F1F4F882321F00E949C5BF801F6CFD1
:10D070008090591390905A13A0905B13B0905C135A
:10D080002091620D3091630D4091640D5091650DBA
:10D09000C501B4010F94F8486B017C0120E030E039
:10D0A000A9010F946D4B87FF04C0F7FAF094F7F8CD
:10D0B000F094E091F00C84E0E89FF0011124E25B31
:10D0C000FD4F2081318142815381C701B6010F9408
:10D0D000344520E030E046E154E40F946D4B1816DF
:10D0E00004F58092620D9092630DA092640DB0924F
:10D0F000650DE2E5FFE284918F010F5F1F4F8823EA
:10D1000021F00E949C5BF801F6CFEBE3FBE08491F9
:10D110008F010F5F1F4F882321F00E949C5BF80155
:10D12000F6CF6091540270915502072E000C880BC7
:10D13000990B0F94D5442091010230910202409145
:10D140000302509104020F9434452AE037ED43E284
:10D150005CE30F94344569AF7AAF8BAF9CAF69A79E
:10D160007AA78BA79CA780904D1390904E13A09008
:10D170004F13B09050132091560D3091570D4091A0
:10D18000580D5091590DC501B4010F94F8482B0169
:10D190003C01C0905113D0905213E0905313F09083
:10D1A000541320915A0D30915B0D40915C0D5091BC
:10D1B0005D0DC701B6010F94F84869AB7AAB8BAB34
:10D1C0009CAB20E030E0A901C301B2010F94CF4431
:10D1D00081113AC020E030E0A90169A97AA98BA9A0
:10D1E0009CA90F94CF4481112FC01091F00C198A83
:10D1F0001A8A1B8A1C8A89829A82AB82BC82CD825F
:10D20000DE82EF82F8868091551390915613A0919B
:10D210005713B091581389879A87AB87BC87AE01A3
:10D22000475F5F4FBE016B5F7F4FCE0101960F944A
:10D230002B2CCE01019682DDDE0151966D01E12E8F
:10D240008E01075D1F4FB7C3A5019401C501B4014D
:10D250000F9434454B015C01A7019601C701B6014B
:10D260000F9434459B01AC01C501B4010F94F948FA
:10D2700020E030E442E556E40F94CF4418160CF455
:10D28000A6C320915E0D30915F0D4091600D5091CD
:10D29000610D6091551370915613809157139091C1
:10D2A00058130F94F8486DAB7EAB8FAB98AF2091BD
:10D2B000620D3091630D4091640D5091650D609148
:10D2C000591370915A1380915B1390915C130F94D2
:10D2D000F8486DA77EA78FA798ABA3019201C30161
:10D2E000B2010F9434456B017C0129A93AA94BA9DD
:10D2F0005CA9CA01B9010F9434459B01AC01C70177
:10D30000B6010F94F9486B017C012DA93EA94FA9E4
:10D3100058ADCA01B9010F9434459B01AC01C70156
:10D32000B6010F94F9480F94B24B6B017C012DEBC1
:10D3300037E346E855E30F94CF4487FF13C020E05E
:10D3400030E0A9016DA57EA58FA598A90F946D4B1E
:10D35000CDA4DEA4EFA4F8A887FF04C0F7FAF094E8
:10D36000F7F8F0942DEB37E346E855E3C701B60133
:10D370000F94CF4487FD2BC329AD3AAD4BAD5CADC7
:10D38000C701B6010F94D5492091840F3091850FC4
:10D390004091860F5091870F0F9434450F94424A65
:10D3A0001B01672B19F422242394312CB10180E056
:10D3B00090E00F94D3449B01AC0160E070E080E802
:10D3C0009FE30F94D5494B015C019B01AC01C30164
:10D3D000B2010F943445698B7A8B8B8B9C8BA501A2
:10D3E000940169A97AA98BA99CA90F9434456D8BE6
:10D3F0007E8B8F8B988FA50194016DA97EA98FA933
:10D4000098AD0F943445698F7A8F8B8F9C8FA501CF
:10D4100094016DA57EA58FA598A90F9434456D8FB5
:10D420007E8F8F8F98A3A5019401C701B6010F9439
:10D4300034459B01AC016DA37EA38FA398A760E048
:10D4400070E080E89FE30F94D54929AD3AAD4BAD2C
:10D450005CAD0F94344525966CAF7DAF8EAF9FAF1A
:10D4600025978091E20F9091E30FA091E40FB09186
:10D47000E50F8DAB9EABAFABB8AF8091E60F90914F
:10D48000E70FA091E80FB091E90F89AF9AAFABAF6A
:10D49000BCAF8091EA0F9091EB0FA091EC0FB0918F
:10D4A000ED0F21968CAF9DAFAEAFBFAF219780E15E
:10D4B000E6E5FDE0DE01119601900D928A95E1F717
:10D4C00091E0291A310809F4FBC18091940481117B
:10D4D00013C00F94D20EDC01CB0188539F4FAF4F86
:10D4E000BF4F8093900490939104A0939204B093C3
:10D4F0009304A1E0A09394040E94BEE80F94D20E7E
:10D500000091900410919104209192043091930421
:10D51000DC01CB01801B910BA20BB30BB7FD13C039
:10D520000F94D20EDC01CB0188539F4FAF4FBF4FFA
:10D530008093900490939104A0939204B0939304E9
:10D5400080E00E94D05F7E01B1E1EB0EF11C8E0104
:10D550000F5F1F4F6701F701219131914191519167
:10D560007F01D8016D917D918D919C910F94F94827
:10D57000F80161937193819391938F01CE16DF0629
:10D5800051F789859A85AB85BC858DA79EA7AFA7E6
:10D59000B8ABC980DA80EB80FC80A701960160916E
:10D5A0006C0470916D0480916E0490916F040F94DF
:10D5B000F8482B013C018D819E81AF81B88589ABF4
:10D5C0009AABABABBCAB9C01AD01609170047091A8
:10D5D000710480917204909173040F94F8484B0188
:10D5E0005C01A3019201C301B2010F9434452B01E8
:10D5F0003C01A5019401C501B4010F9434459B0180
:10D60000AC01C301B2010F94F9489B01AC016091D8
:10D6100084047091850480918604909187040F940E
:10D62000F8480F94B24B9B01AC016DA57EA58FA568
:10D6300098A90F94F94829966CAF7DAF8EAF9FAF34
:10D6400029976093660D7093670D8093680D909392
:10D65000690DA70196016091740470917504809121
:10D660007604909177040F94F8482B013C0129A986
:10D670003AA94BA95CA960917804709179048091D2
:10D680007A0490917B040F94F8484B015C01A3014C
:10D690009201C301B2010F9434452B013C01A50155
:10D6A0009401C501B4010F9434459B01AC01C30141
:10D6B000B2010F94F9489B01AC016091880470910C
:10D6C000890480918A0490918B040F94F8480F94F8
:10D6D000B24B9B01AC016DA57EA58FA598A90F94B7
:10D6E000F9484B015C0160936A0D70936B0D809358
:10D6F0006C0D90936D0DA701960160917C04709163
:10D700007D0480917E0490917F040F94F8486B0112
:10D710007C0129A93AA94BA95CA960918004709168
:10D72000810480918204909183040F94F8482B0126
:10D730003C01A7019601C701B6010F9434456B0166
:10D740007C01A3019201C301B2010F9434459B01F6
:10D75000AC01C701B6010F94F9489B01AC0160917F
:10D760008C0470918D0480918E0490918F040F949D
:10D77000F8480F94B24B9B01AC016DA57EA58FA517
:10D7800098A90F94F9486B017C0160936E0D70931A
:10D790006F0D8093700D9093710D1091F00C2DA969
:10D7A0003EA94FA958AD29966CAD7DAD8EAD9FAD0C
:10D7B00029970F94F8482B013C0129AD3AAD4BADA8
:10D7C0005CADC501B4010F94F8484B015C01219692
:10D7D0002CAD3DAD4EAD5FAD2197C701B6010F94A5
:10D7E000F8486B017C01A3019201C301B2010F94BF
:10D7F00034452B013C01A5019401C501B4010F94EE
:10D8000034459B01AC01C301B2010F94F9484B01AF
:10D810005C01A7019601C701B6010F9434459B0135
:10D82000AC01C501B4010F94F9480F94B24B9B01B0
:10D83000AC0125966CAD7DAD8EAD9FAD25970F9457
:10D84000344569A37AA38BA39CA3DE0195966D0151
:10D85000E12E8E010F5D1F4F9E01235F3F4F4EE66D
:10D860005DE06AE67DE086E69DE00E9437AD8823B4
:10D8700039F18091660D9091670DA091680DB0917E
:10D88000690D8DAB9EABAFABB8AF80916A0D909137
:10D890006B0DA0916C0DB0916D0D89AF9AAFABAFD0
:10D8A000BCAF80916E0D90916F0DA091700DB091F5
:10D8B000710D21968CAF9DAFAEAFBFAF219700CE5B
:10D8C0008DE493E13BDA2DA93EA94FA958AD6091B3
:10D8D000660D7091670D8091680D9091690D0F94A0
:10D8E000F8482B013C0129AD3AAD4BAD5CAD6091E0
:10D8F0006A0D70916B0D80916C0D90916D0D0F9470
:10D90000F8484B015C0121962CAD3DAD4EAD5FADAD
:10D91000219760916E0D70916F0D8091700D9091B7
:10D92000710D0F94F8486B017C01A3019201C301B2
:10D93000B2010F9434452B013C01A5019401C501AE
:10D94000B4010F9434459B01AC01C301B2010F94A3
:10D95000F9484B015C01A7019601C701B6010F947C
:10D9600034459B01AC01C501B4010F94F9486B012A
:10D970007C0120E030E0A9010F94CF44882329F1F5
:10D980001091F00CC701B6010F94B24B9B01AC0192
:10D9900025966CAD7DAD8EAD9FAD25970F9434452A
:10D9A00069A37AA38BA39CA3DE0195966D01E12E5A
:10D9B0008E010F5D1F4F29E533E14EE65DE06AE61B
:10D9C0007DE086E69DE00E9437AD0E94925BC85BD9
:10D9D000DF4F0FB6F894DEBF0FBECDBFDF91CF9102
:10D9E0001F910F91FF90EF90DF90CF90BF90AF907D
:10D9F0009F908F907F906F905F904F903F902F906F
:10DA000008954F925F926F927F928F929F92AF9202
:10DA1000BF92CF92DF92EF92FF920F931F93CF931B
:10DA2000DF930AE01CE020E030E042E553E4F80137
:10DA300060817181828193810F94F9482BED3FE0E1
:10DA400049E450E40F94344520E030E044E353E4EB
:10DA50000F94D5494B015C010F94D2492B013C0135
:10DA600020E030E0A9016091160C7091170C8091B4
:10DA7000180C9091190C0F94F9486B017C01CCE6BD
:10DA8000D4E09B01AC01C301B2010F94344568831B
:10DA900079838A839B83C501B4010F94A84B9B01B2
:10DAA000AC01C701B6010F9434456C837D838E832E
:10DAB0009F8320E030E045EA53E4F80164817581FA
:10DAC000868197810F94F9482BED3FE049E450E4BB
:10DAD0000F94344520E030E044E353E40F94D549FB
:10DAE0004B015C010F94D2499B01AC01C701B60107
:10DAF0000F943445688779878A879B87C501B4016D
:10DB00000F94A84B9B01AC01C701B6010F9434459B
:10DB10006C877D878E879F8720E030E044EB52E45E
:10DB2000F80160857185828593850F94F9482BED06
:10DB30003FE049E450E40F94344520E030E044E312
:10DB400053E40F94D5494B015C010F94D2499B01DA
:10DB5000AC01C701B6010F943445688B798B8A8B71
:10DB60009B8BC501B4010F94A84B9B01AC01C7016D
:10DB7000B6010F9434456C8B7D8B8E8B9F8B20E090
:10DB800030E0A9016091060C7091070C8091080C9F
:10DB90009091090C0F94F9489B01AC010F94344506
:10DBA000E4E8F4E060837183828393836483758304
:10DBB00086839783608771878287938782E00E943C
:10DBC000B2541092E60CDF91CF911F910F91FF900C
:10DBD000EF90DF90CF90BF90AF909F908F907F900D
:10DBE0006F905F904F900895CF93DF93E091FE0B7D
:10DBF000F0E0E858F54F8081882381F0E8E3FBE00E
:10DC00008491EF012196882321F00E949C5BFE0104
:10DC1000F7CF8AE0DF91CF910C949C5BDF91CF919D
:10DC20000895CF93DF938091590480935A04EFE2D3
:10DC3000FBE08491EF012196882321F00E949C5BF8
:10DC4000FE01F7CF80917F0F9091800FA091810FFF
:10DC5000B091820FBC01CD016F5F7F4F8F4F9F4FFF
:10DC60000E94AB5E8AE00E949C5BDF91CF91BCCFAB
:10DC70000F931F93CF93DF93FC012381222311F095
:10DC800080E044C08B01EC01FB018789803139F1D0
:10DC90008032B1F783E08B83F801428D538D648D20
:10DCA000758D4D8B5E8B6F8B788F9E012F5E3F4FF6
:10DCB000C8010F94921C882319F31A8F098F81E0F1
:10DCC0008983188619861A861B861C821D821E82ED
:10DCD0001F82188A1C861D861E861F8617C082E03A
:10DCE0008B831D8A1E8A1F8A188EFB01808D918D61
:10DCF000A0E0B0E025E0880F991FAA1FBB1F2A955E
:10DD0000D1F7898B9A8BAB8BBC8BD7CFDF91CF911F
:10DD10001F910F910895CF93DF93EC010F94601D35
:10DD20001B82DF91CF910895CF93DF93EC0141E007
:10DD3000611101C040E06C857D858E859F850F94C3
:10DD4000491B882341F0888920E2829FC001112469
:10DD50008E58924F02C080E090E0DF91CF910895FD
:10DD6000CF93DF93EB01FC012381211102C080E0FE
:10DD700027C02250223020F48FE2888319821FC0EE
:10DD800060E0D2DF009799F3FC0190E080E02EE2A2
:10DD90003081303269F0883029F4DE01A90FB11DDD
:10DDA0002C939F5FDE01A90FB11D30813C939F5FD3
:10DDB0008F5F31968B3061F7C90FD11D188281E0DA
:10DDC000DF91CF9108953F924F925F926F927F9231
:10DDD0008F929F92AF92BF92CF92DF92EF92FF927B
:10DDE0000F931F93CF93DF93CDB7DEB72C970FB66A
:10DDF000F894DEBF0FBECDBF5C01DC0159968D905B
:10DE00009C905A97F40181859285A385B4859C01E5
:10DE1000AD012F5F3F4F4F4F5F4F29873A874B87A9
:10DE20005C87D5011496CD90DD90ED90FC9017970E
:10DE3000C114D104E104F10439F0BFEFCB1ADB0ABD
:10DE4000EB0AFB0A312C07C0F401C080D180E280CC
:10DE5000F38033243394260137011D821E821F82F2
:10DE60001886F40181859285A385B4852D813E8134
:10DE70004F815885281739074A075B0708F064C0A7
:10DE800089859A85AB85BC858C159D05AE05BF053A
:10DE900050F482E0C82ED12CE12CF12C92E0492ED6
:10DEA000512C612C712C9E012F5F3F4FB701A601B1
:10DEB000C4010F94121C882309F446C089819A81F9
:10DEC000AB81BC81892B8A2B8B2B41F0260137013A
:10DED0009FEF491A590A690A790A05C0C414D50482
:10DEE000E604F70491F02D813E814F8158852F5F24
:10DEF0003F4F4F4F5F4F2D833E834F8358873FEFF8
:10DF0000C31AD30AE30AF30AACCF0FEF1FEF2FEFC8
:10DF10003FE0B301A201C4010F94811BF82E8823B6
:10DF200099F0D50114964D915D916D917C91179763
:10DF3000411551056105710549F093018201C40144
:10DF40000F94811B811102C0F12C29C0D5011496B8
:10DF50004D925D926D927C921797332051F0D301D0
:10DF6000C2010196A11DB11DF40180839183A2839A
:10DF7000B383F50185899689A789B08D892B8A2B72
:10DF80008B2B69F4D50155964D925D926D927C92E2
:10DF9000589711968C911197806811968C938F2DBC
:10DFA0002C960FB6F894DEBF0FBECDBFDF91CF9198
:10DFB0001F910F91FF90EF90DF90CF90BF90AF90A7
:10DFC0009F908F907F906F905F904F903F900895BB
:10DFD00040E050E0BA010D94921D61E0FC018081A7
:10DFE0000C945DCD8EBD0DB407FEFDCF08958FEF6F
:10DFF0008EBD0DB407FEFDCF8EB508950F931F9310
:10E00000CF93DF93EB010F94D20E8B01F0DF8F3FA4
:10E0100049F00F94D20E601B710B6C177D07B0F3A3
:10E0200080E001C081E0DF91CF911F910F910895B1
:10E030008F929F92AF92BF92EF92FF921F93CF93D6
:10E04000DF93EC01162F49015A019A81892F806ACA
:10E0500086958CBD90FD03C081E0963009F480E088
:10E060008DBD60E088810E945DCD6CE271E0CE01E3
:10E07000C5DF812F8064B6DF88E1E82EF12CD50161
:10E08000C4010E2C04C0B695A795979587950A9460
:10E09000D2F7A8DF88E0E81AF10888EFE8168FEFDA
:10E0A000F80669F7112391F0183011F487E801C0E0
:10E0B0008FEF98DF1C3009F49ADF10E098DF8B8334
:10E0C00087FF07C01F3F29F01F5FF8CF85E98ADF70
:10E0D000F4CFDF91CF911F91FF90EF90BF90AF9061
:10E0E0009F908F9008950F931F93CF93DF93EC0130
:10E0F00089018C81833039F089E0440F551F661FF8
:10E10000771F8A95D1F79A01AB0168E1CE0190DFC4
:10E11000882311F086E02CC08EEF8EBDF801C80177
:10E120009E5F0DB407FEFDCF20812EBD0DB407FE0E
:10E13000FDCF21812EBD32968E179F0791F70DB42A
:10E1400007FEFDCF8FEF4EDF8FEF4CDF50DF8B836D
:10E150008F71853029F083E18983CE013EDF09C0CC
:10E1600068E572E0CE014ADF182F811106C087E111
:10E170008983CE0132DF10E00FC020E030E0A9013A
:10E180006DE0CE0155DF811103C031DF882311F02E
:10E1900086E1EECFCE0121DF812FDF91CF911F915C
:10E1A0000F9108952F923F924F925F926F927F92BC
:10E1B0008F929F92AF92BF92CF92DF92EF92FF9297
:10E1C0000F931F93CF93DF93EC012A013B01690169
:10E1D0008C81833039F059E0440C551C661C771C47
:10E1E0005A95D1F743E0342E22242A94560181E037
:10E1F000A81A8EEFB80A4601EEEF9E1AA30192010B
:10E2000061E1CE0115DF882319F0F4E0F98352C0F3
:10E210000F94D20E8B01EBDE8B838F3F51F40F9462
:10E22000D20E601B710B6D327140A8F381E18983BE
:10E230003DC08E3F19F0EFE0E98338C02EBCD60117
:10E24000F6010DB407FEFDCF8EB581932EBCAE1640
:10E25000BF06B9F70DB407FEFDCF8EB5F50180837B
:10E26000E12CF12C8D91EF2DFF27E827EE0FFF1FFA
:10E27000E554F34F85919491FE2CEE24E826F9267F
:10E28000A815B90579F7B3DE082F10E0102F002785
:10E29000AEDE082B0E151F0519F0F0E2F98306C05B
:10E2A000CE019BDE8FEF9EDE81E012C0CE0195DEB7
:10E2B0008FEF98DECE0191DE3A94332041F020E0DA
:10E2C00030E0A9016CE0CE01B3DE198297CF80E087
:10E2D000DF91CF911F910F91FF90EF90DF90CF9042
:10E2E000BF90AF909F908F907F906F905F904F9076
:10E2F0003F902F9008952F923F924F925F926F928E
:10E300007F928F929F92AF92BF92CF92DF92EF92C5
:10E31000FF920F931F93CF93DF9300D01F92CDB73F
:10E32000DEB79C838B834B015A01DC0113968C91E1
:10E33000811103C08FEF9FEFEAC0EB81FC818181E7
:10E3400080FFF8CFAB81BC8151960D911D912D912D
:10E350003C91549718964D915D916D917C911B97CE
:10E36000C501A0E0B0E068017901C41AD50AE60A47
:10E37000F70AC816D906EA06FB0618F45801A41ACB
:10E38000B50A75018B819C8104969A838983612CDF
:10E3900042E0742EE114F10409F48BC0AB81BC811E
:10E3A00018964D915D916D917C911B976A01B1E03A
:10E3B000DB22EB81FC812381818D928D1A012B015F
:10E3C00039E056944794379427943A95D1F7223000
:10E3D00061F4FC01828D938DA48DB58DBC01CD01BE
:10E3E000620D731D841D951D4AC0DC0114961C919D
:10E3F00011501221C114D10401F511111EC0452B79
:10E40000462B472B59F4EB81FC8185899689A78996
:10E41000B08D84839583A683B7830FC0AB81BC8105
:10E4200014964D915D916D917C91179729813A8158
:10E430000F94121C882309F47DCFEB81FC81218D80
:10E44000328D84819581A681B7810297A109B10996
:10E45000F901058404C0880F991FAA1FBB1F0A94E5
:10E46000D2F74685578560897189840F951FA61F4D
:10E47000B71FBC01CD01610F711D811D911D93015D
:10E480002C193D0987012E153F0508F48901011556
:10E49000F2E01F0771F52091720F3091730F4091D8
:10E4A000740F5091750F621773078407950719F45D
:10E4B00020C0C5012CC09401AB01BC0180917B0F31
:10E4C00090917C0F6FDE882309F434CF800E911E6B
:10E4D000EB81FC8180859185A285B385800F911F9A
:10E4E000A11DB11D80879187A287B387E01AF10A29
:10E4F00051CF40E00F94491B882309F41BCFB6018C
:10E500006E58724FA801C4010F94854CDFCF0F9055
:10E510000F900F900F90DF91CF911F910F91FF906F
:10E52000EF90DF90CF90BF90AF909F908F907F90B3
:10E530006F905F904F903F902F9008954F925F9211
:10E540006F927F929F92AF92BF92CF92DF92EF92A3
:10E55000FF920F931F93CF93DF931F92CDB7DEB738
:10E560008C017B015A01C22EDB0159968D919C9141
:10E570005A97F801928F818FCB012ADD912CF701F8
:10E5800080859185A285B385418952896389748983
:10E5900084179507A607B70708F05FC025E0B69572
:10E5A000A795979587952A95D1F7F82FFF70DF2EBD
:10E5B000D70113968C91823008F45EC041E050E0A0
:10E5C000BE016F5F7F4FC70196DE019719F4898105
:10E5D00090E002C08FEF9FEF019609F44DC0F70164
:10E5E00080859185A285B3854F96A11DB11D808739
:10E5F0009187A287B387F0E2DF9EB00111246E58A5
:10E60000724F61157105C1F1DB018C91882319F0FE
:10E61000853EC1F469C191100EC08091720F909136
:10E62000730FA091740FB091750FF80184879587CF
:10E63000A687B787D08ADB018C91882361F0992463
:10E6400093949DCF4BE050E0C5010F94784C892BFB
:10E6500009F095CF13C0992493948C2D8274823441
:10E6600059F4992009F48AC0F801D08861E0C80102
:10E670005BDB009709F00BC180E039C1C7FCFCCF20
:10E68000F0E2DF9EA00111249A012E58324FD901E9
:10E690001B968C91817121F08C2D827109F06AC0DA
:10E6A0008091720F9091730FA091740FB091750FBC
:10E6B000F80184879587A687B787D08ACA018E58C4
:10E6C000924F7C01DC0154964D915C91559760E02E
:10E6D00070E0DA0199278827858B968BA78BB08FFE
:10E6E000F701428D538D60E070E0482B592B6A2B67
:10E6F0007B2BD80155964D935D936D937C935897E2
:10E70000F9018385887161F4F701848D958DA68D5B
:10E71000B78DF801818B928BA38BB48B81E010C0F5
:10E72000803141F598012F5E3F4FD80159968D9168
:10E730009C915A970F94921C8823E1F084E0F80191
:10E7400083838C2D8F70D80111968C931197F801CB
:10E75000148215821682178218961D921D921D92A0
:10E760001C921B97C4FEB3C0C8010F948402811190
:10E77000AEC082CFD80113961C927ECFD7011396DC
:10E780008C911397823009F477CF51968D919D919A
:10E790000D90BC91A02D803E9F4FAF41B10508F078
:10E7A0006BCFC70110DB882309F466CF0F94091BD8
:10E7B000882309F461CFD70159962D913C915A973E
:10E7C00014968D919D910D90BC91A02D0297A10959
:10E7D000B109F901058404C0880F991FAA1FBB1F46
:10E7E0000A94D2F74684578460887188480E591E6F
:10E7F0006A1E7B1E81E080937A0F4092720F5092C6
:10E80000730F6092740F7092750F80E092E0E2E7F0
:10E81000FDE0DF019C011D9221503040E1F7DD2435
:10E82000D394D7015996ED91FC915A978481D816CB
:10E8300090F422E73DE0B301A2014D0D511D611D91
:10E84000711D80917B0F90917C0F4DDC882309F422
:10E8500013CFD394E6CF80E092E0A0E0B0E005844F
:10E8600004C0880F991FAA1FBB1F0A94D2F7F70193
:10E870004189528963897489840F951FA61FB71F28
:10E88000818B928BA38BB48B82E79DE0D12C20E20D
:10E89000DC011D922A95E9F72BE0F501DC010190DE
:10E8A0000D922A95E1F721E238E2FC01318B208BB1
:10E8B00040E058E057874687338B228B318F208F7B
:10E8C000578B468B0F94091B8111DACED5CEC5FE2E
:10E8D00009C0F8014189528963897489C8010F947C
:10E8E000921D05C081E003C09110A9CE96CE0F9075
:10E8F000DF91CF911F910F91FF90EF90DF90CF901C
:10E90000BF90AF909F907F906F905F904F900895D1
:10E910008091760A8770873069F48FE40E94765B75
:10E92000882319F00E94EB5A03C08FE40E942D5BEC
:10E93000811117C00E9443BB80E00E9496490E944B
:10E940001E5181E08093750A0E94039B8091740A96
:10E950008093750A0E94055183E080934D020C94C8
:10E960006DAC08958CE0EAEBF4E0A6E5BDE0019023
:10E970000D928A95E1F708954F925F926F927F9280
:10E980008F929F92AF92BF92CF92DF92EF92FF92BF
:10E99000CF93DF93EC0188809980AA80BB80CC80E4
:10E9A000DD80EE80FF80A5019401C501B4010F94C4
:10E9B00034452B013C01A7019601C701B6010F9414
:10E9C00034459B01AC01C301B2010F94F9482B01FE
:10E9D0003C012091B6043091B7044091B8045091A5
:10E9E000B9040F946D4B181634F5C301B2010F949E
:10E9F000B24B9B01AC016091B2047091B304809161
:10EA0000B4049091B5040F94D5492B013C019B01AE
:10EA1000AC01C501B4010F943445688379838A83BE
:10EA20009B83A3019201C701B6010F9434456C8307
:10EA30007D838E839F83C0904202D0904302E090FA
:10EA40004402F0904502A7019601688579858A8580
:10EA50009B850F94CF4487FF04C0C886D986EA8679
:10EA6000FB86C0903602D0903702E0903802F090DA
:10EA70003902A7019601688579858A859B850F945F
:10EA80006D4B181624F4C886D986EA86FB86DF917A
:10EA9000CF91FF90EF90DF90CF90BF90AF909F907D
:10EAA0008F907F906F905F904F9008954F925F92FC
:10EAB0006F927F928F929F92AF92BF92DF92EF926E
:10EAC000FF920F931F93CF93DF93D82EC82FD0E0E0
:10EAD000FE01E854F34F64917E01EE0CFF1CEE0C36
:10EAE000FF1CF701E455F34F4590559065907490E5
:10EAF000062E000C770B880B990B0F94D5444B0115
:10EB00005C0120E030E040EC5FE3C301B2010F9410
:10EB10003445A50194010F943445AB01BC0100E0DC
:10EB200010E098018D2D0E94DB48F701E056F34F6D
:10EB30002591359145915491C501B4010F94344507
:10EB40004B015C0120E030E0A9010F94CF44882301
:10EB500009F447C000E010E09801B501A401705825
:10EB60008D2D0E94DB48FE01E356F34F6491611145
:10EB700017C0E2E5FFE28491EF012196882321F09E
:10EB80000E949C5BFE01F7CFEBE7FCE08491EF0174
:10EB90002196882321F00E949C5BFE01F7CF6AE05A
:10EBA000F701E559F34F459055906590749070E0EA
:10EBB00080E090E00F94D5449B01AC01C301B20109
:10EBC0000F94D5492B013C01A5019401C501B40165
:10EBD0000F94F948AB01BC01930182018D2D0E9475
:10EBE000DB48F701E65EF34F80809180A280B3801E
:10EBF00020E030E0A901C501B4010F94CF441816FC
:10EC0000DCF0F701EF5EFA4F20E030E040EE50E438
:10EC100060817181828193810F9434459B01AC01A5
:10EC2000C501B4010F94F848AB01BC0100E010E04D
:10EC300098018D2D0E94DB48DF91CF911F910F919C
:10EC4000FF90EF90DF90BF90AF909F908F907F905C
:10EC50006F905F904F9008950F931F93CF93DF9322
:10EC60008C01E2E5FFE28491EF012196882321F0F7
:10EC70000E949C5BFE01F7CFB8018EE59CE00E94EC
:10EC80009EC382E20E949C5B8AE00E949C5B81E0C2
:10EC9000DF91CF911F910F9108952F923F924F9244
:10ECA0005F926F927F928F929F92AF92BF92CF921C
:10ECB000DF92EF92FF920F931F93CF93DF93CDB725
:10ECC000DEB7C254D1090FB6F894DEBF0FBECDBF78
:10ECD0004C015B016A01322E19821C821C8E1F8E30
:10ECE0006115710511F410E0A4C0FC01838181114C
:10ECF000FACFFA0180818F3209F099C0F501838142
:10ED00008250823010F485010CC0F501618D728D46
:10ED1000CE014C960E94386E882329F38E01045E42
:10ED20001F4FC6016C010196F60120812F32D1F3ED
:10ED3000CE0101967C013C012E019CE1490E511C43
:10ED40002396EFAE23972F2C9BE09150E7E3F0E062
:10ED5000EC0FFD1FE90FF11D80E280839111F5CFCB
:10ED6000960147E0D9018D91882369F18F3259F1DD
:10ED70008E3239F44A3009F4B6CF98E04AE09D016A
:10ED8000F1CFEBEBFEE02491222321F031968213A8
:10ED9000FACFA9CF491708F4A6CF813208F4A3CF40
:10EDA0008F3709F4A0CF21E0290FE7E3F0E0EC0F63
:10EDB000FD1FE90FF11D9FE9980F9A3108F4805269
:10EDC0008083922FDCCF8FA9803209F48CCF690128
:10EDD000F90180812F5F3F4F8F32C9F38823F1F013
:10EDE00021E0AE01495C5F4FB801C701A7DB882372
:10EDF00009F479CF0A151B0519F0C8010E948B6E22
:10EE00006E147F0441F023969FAD2397822D8701D6
:10EE1000E92EF82E99CF942D852DF9CF232DAE0113
:10EE2000495C5F4FB801C40189DB182F02C08B0118
:10EE30007FCFCE014C960E94825BCE0101960E944C
:10EE4000825B812FCE5BDF4F0FB6F894DEBF0FBE23
:10EE5000CDBFDF91CF911F910F91FF90EF90DF9089
:10EE6000CF90BF90AF909F908F907F906F905F906A
:10EE70004F903F902F900895CF93DF938B3B92401C
:10EE8000B1F0E8E7FBE28491EF012196882321F0BD
:10EE90000E949C5BFE01F7CFEBECFEE08491EF015A
:10EEA0002196882331F00E949C5BFE01F7CF80E021
:10EEB00001C081E0DF91CF9108952F923F924F9250
:10EEC0005F926F927F928F929F92AF92BF92CF92FA
:10EED000DF92EF92FF920F931F93CF93DF93CDB703
:10EEE000DEB7C157D1090FB6F894DEBF0FBECDBF54
:10EEF0008DB69EB6A3961FAE1EAEA39784E690E095
:10EF0000A5969FAF8EAFA59701E09E012F593F4F69
:10EF100044E050E0BE01695A7F4FCE018D599F4FAA
:10EF20000F94B0199E012F593F4F42E050E0BE01AF
:10EF30006B597F4FCE018D599F4F0F94B01943E00D
:10EF400050E0BE01695A7F4F8BED92E00F94C74CA1
:10EF5000892B09F43CC06B968FAD6B97882339F0F1
:10EF60008FE368968FAF689769961FAE6997E2E561
:10EF7000FFE284918F010F5F1F4F811103C0EEE804
:10EF8000FFE004C00E949C5BF801F3CF84918F01E5
:10EF90000F5F1F4F882321F00E949C5BF801F6CF82
:10EFA000BE01695A7F4F85E89FE00E949EC3E7E754
:10EFB000FFE084918F010F5F1F4F882321F00E9493
:10EFC0009C5BF801F6CF81E08093C6046FC52DB637
:10EFD0003EB667961CAE1DAE1EAE1FAE6797A396DB
:10EFE0001FAE1EAEA39701E09E012F593F4F41E097
:10EFF00050E0BE0164597F4FCE018D599F4F0F9451
:10F00000B01980E1EFE5F2E0DE01919601900D92FA
:10F010008A95E1F780E1EFE6F2E0DE01519601909A
:10F020000D928A95E1F780E1EFE7F2E0DE011196BB
:10F0300001900D928A95E1F7AD964FADAD9750E0F6
:10F040004D5F5F4F440F551F440F551F2DB73EB7FF
:10F05000241B350B0FB6F8943EBF0FBE2DBF8DB7E6
:10F060009EB701963C0100E09E012F593F4FBC0125
:10F07000CE018D599F4F0F94B0199E012F593F4FCC
:10F0800044E050E068E87FE0CE018D599F4F0F9437
:10F09000B019AD96AFACAD97B12C93E0A90EB11CF1
:10F0A000AA0CBB1CAA0CBB1CEDB7FEB7EA19FB09E6
:10F0B0000FB6F894FEBF0FBEEDBF2DB73EB72F5F62
:10F0C0003F4F79018DB79EB78A199B090FB6F89407
:10F0D0009EBF0FBE8DBFEDB7FEB731966F019E018B
:10F0E0002F593F4FA501B701CE018D599F4F0F9466
:10F0F000B0199E012F593F4FA501B601CE018D5980
:10F100009F4F0F94B0198091830F882309F4A4C0F6
:10F1100000E09E012F593F4F44E050E06AEF72E15A
:10F12000CE018D599F4F0F94B0199E012F593F4F1B
:10F1300044E050E06AEE7CE0CE018D599F4F0F9481
:10F14000B0199E012F593F4F44E050E066EF72E145
:10F15000CE018D599F4F0F94B0199E012F593F4FEB
:10F1600044E050E062ED72E1CE018D599F4F0F9463
:10F17000B0199E012F593F4F44E050E06EEC72E110
:10F18000CE018D599F4F0F94B0199E012F593F4FBB
:10F1900040E150E06EEF72E1CE018D599F4F0F9428
:10F1A000B0199E012F593F4F44E050E0BE016D5A07
:10F1B0007F4FCE018D599F4F0F94B0199E012F594B
:10F1C0003F4F4CE050E0BE01635C7F4FCE018D5954
:10F1D0009F4F0F94B0199E012F593F4F44E050E0CC
:10F1E000BE016D5A7F4FCE018D599F4F0F94B019BC
:10F1F0009E012F593F4F44E050E0BE016D5A7F4FB2
:10F20000CE018D599F4F0F94B01901E09E012F59E7
:10F210003F4F41E050E0BE0165597F4FCE018D590F
:10F220009F4F0F94B0199E012F593F4F41E050E07E
:10F23000BE0166597F4FCE018D599F4F0F94B01973
:10F24000AC968FADAC97AB96CFACAB978C9D600175
:10F250001124E12CF12C7CC0AD968FADAD9790E0E0
:10F26000029626ED32E1E0963FAF2EAFE097B60171
:10F27000AE014F5F5F4F26E4A22E2DE0B22ED701E4
:10F280007E0131E1E30EF11C36EEC32E32E1D32EC6
:10F29000E2967FAE6EAEE2978E010F5D1F4F20E0CB
:10F2A00030E0821793072CF0E296EEADFFADE297C7
:10F2B00001C0F8014080518062807380F601419264
:10F2C0005192619271926F018217930734F04D90C1
:10F2D0005D906D907C90139705C0F7014080518040
:10F2E00062807380F50141925192619271925F0147
:10F2F0008217930714F0FB0101C0FA01408051808E
:10F3000062807380E096EEADFFADE097419251923E
:10F3100061927192E096FFAFEEAFE0972F5F3F4FA3
:10F320006C5F7F4F4C5F5F4F1496F4E0EF0EF11C63
:10F33000E296EEADFFADE2973496E296FFAFEEAF08
:10F34000E2970C5F1F4F2430310509F0AACFE0CEC1
:10F3500000E09E012F593F4F44E050E0EC14FD04C3
:10F3600061F0BE016D5A7F4FCE018D599F4F0F94B2
:10F37000B019FFEFEF1AFF0AEBCF6AE27CE0CE0193
:10F380008D599F4F0F94B0199E012F593F4F44E262
:10F3900050E06AEA7FE0CE018D599F4F0F94B0197B
:10F3A00001E09E012F593F4F41E050E0BE016759F7
:10F3B0007F4FCE018D599F4F0F94B0199E012F5949
:10F3C0003F4F41E050E0BE0168597F4FCE018D595B
:10F3D0009F4F0F94B01900E09E012F593F4F44E01A
:10F3E00050E0BE01675B7F4FCE018D599F4F0F9458
:10F3F000B0199E012F593F4F44E050E0BE016F5CB1
:10F400007F4FCE018D599F4F0F94B019AA968FADA3
:10F41000AA97A996CFACA9978C9D60011124E12CE5
:10F42000F12C00E09E012F593F4FEC14FD0471F0C8
:10F4300044E050E0BE016D5A7F4FCE018D599F4F81
:10F440000F94B0192FEFE21AF20AEBCF41E050E02F
:10F45000BE0163597F4FCE018D599F4F0F94B01954
:10F460009E012F593F4F41E050E0BE0169597F4F47
:10F47000CE018D599F4F0F94B0199E012F593F4FC8
:10F4800044E050E066E27CE0CE018D599F4F0F943E
:10F49000B0199E012F593F4F4CE050E06AE17CE0EB
:10F4A000CE018D599F4F0F94B0199E012F593F4F98
:10F4B00044E050E066E17CE0CE018D599F4F0F940F
:10F4C000B0199E012F593F4F44E050E066E07CE0C8
:10F4D000CE018D599F4F0F94B0199E012F593F4F68
:10F4E00044E050E064E87FE0CE018D599F4F0F94D7
:10F4F000B0199E012F593F4F44E050E062E07CE09C
:10F50000CE018D599F4F0F94B0199E012F593F4F37
:10F510004CE050E06AE07CE0CE018D599F4F0F94A3
:10F52000B0199E012F593F4F44E050E06CE47CE05D
:10F53000CE018D599F4F0F94B0199E012F593F4F07
:10F5400044E050E068E47CE0CE018D599F4F0F9479
:10F55000B0199E012F593F4F44E050E060E57CE038
:10F56000CE018D599F4F0F94B01910E000E09E011D
:10F570002F593F4F44E050E0BE016D5A7F4FCE01FE
:10F580008D599F4F0F94B019111110C06796CCACD4
:10F59000DDACEEACFFAC679720E030E84BE355E420
:10F5A000C701B6010F94CF44811103C084E0F82E47
:10F5B00033C08091830F811108C0C0923B0CD09260
:10F5C0003C0CE0923D0CF0923E0C00E09E012F5965
:10F5D0003F4F44E050E063E47CE0CE018D599F4F03
:10F5E0000F94B0199E012F593F4F44E050E06FE354
:10F5F0007CE0CE018D599F4F0F94B0199E012F5979
:10F600003F4F44E050E0BE016D5A7F4FCE018D590F
:10F610009F4F0F94B01912C0FA94FF2079F000E0C8
:10F620009E012F593F4F44E050E0BE016D5A7F4F7D
:10F63000CE018D599F4F0F94B019EECF1F5F15303B
:10F6400009F094CF00E09E012F593F4F42E050E077
:10F65000BE01615A7F4FCE018D599F4F0F94B01953
:10F660009E012F593F4F44E050E0BE016D5A7F4F3D
:10F67000CE018D599F4F0F94B0196796CCACDDAC7D
:10F68000EEACFFAC679720E030E84BE355E4C701F0
:10F69000B6010F94CF44882329F18091830F811103
:10F6A00008C0C092730CD092740CE092750CF0926A
:10F6B000760C00E09E012F593F4F44E050E06FE68A
:10F6C0007CE0CE018D599F4F0F94B0199E012F59A8
:10F6D0003F4F44E050E06BE67CE0CE018D599F4FF8
:10F6E0000F94B01900E09E012F593F4F42E050E0C7
:10F6F000BE01635A7F4FCE018D599F4F0F94B019B1
:10F700009E012F593F4F41E050E0BE0163597F4FAA
:10F71000CE018D599F4F0F94B01919E0115000E0A0
:10F720009E012F593F4F112359F044E050E0BE0194
:10F730006D5A7F4FCE018D599F4F0F94B019EECF68
:10F7400041E050E06AE37CE0CE018D599F4F0F9479
:10F75000B01910E000E09E012F593F4F44E050E007
:10F76000BE016D5A7F4FCE018D599F4F0F94B01936
:10F770008091830F811110C011110EC067964CAD9E
:10F780005DAD6EAD7FAD67974093360C5093370CEF
:10F790006093380C7093390C1F5F1530D9F68111C6
:10F7A00002C00E9457BC1CE0115011F41CE00FC0B5
:10F7B00000E09E012F593F4F42E050E0BE01655AE4
:10F7C0007F4FCE018D599F4F0F94B019EDCF11503F
:10F7D00000E09E012F593F4F112359F044E050E0C3
:10F7E000BE01615B7F4FCE018D599F4F0F94B019C1
:10F7F000EECF46E050E0BE01675B7F4FCE018D59F2
:10F800009F4F0F94B0199E012F593F4F44E050E095
:10F81000BE016D5A7F4FCE018D599F4F0F94B01985
:10F820009E012F593F4F4CE050E0BE016F5C7F4F6F
:10F83000CE018D599F4F0F94B0191CE1115011F456
:10F8400014E00FC000E09E012F593F4F44E050E00C
:10F85000BE016D5A7F4FCE018D599F4F0F94B01945
:10F86000EDCF115079F000E09E012F593F4F44E059
:10F8700050E0BE016D5A7F4FCE018D599F4F0F94BE
:10F88000B019EFCF10E000E09E012F593F4F44E048
:10F8900050E0BE016D5A7F4FCE018D599F4F0F949E
:10F8A000B0198091830F811110C011110EC067969D
:10F8B0008CAD9DADAEADBFAD67978093320C90938C
:10F8C000330CA093340CB093350C1F5F1530D9F670
:10F8D00010E000E09E012F593F4F44E050E0BE0190
:10F8E0006D5A7F4FCE018D599F4F0F94B019809163
:10F8F000830F811110C011110EC067968CAD9DADA4
:10F90000AEADBFAD679780932E0C90932F0CA09354
:10F91000300CB093310C1F5F1530D9F6A5968EAD23
:10F920009FADA59784569109A7DA8093C6048823D2
:10F9300001F1E2E5FFE284918F010F5F1F4F882301
:10F9400021F00E949C5BF801F6CFA5966EAD7FADCD
:10F95000A597645671098FE69FE00E9485C36BEB03
:10F9600072E087E69FE00E9485C38AE00E949C5B6C
:10F970008EC0A3962EAD3FADA397A7968EAD9FAD3B
:10F98000A7972817390709F447C081E08093C60478
:10F99000E8E7FBE284918F010F5F1F4F811103C0E5
:10F9A000E7E4FFE004C00E949C5BF801F3CF849180
:10F9B0008F010F5F1F4F882321F00E949C5BF8018D
:10F9C000F6CFA7966EAD7FADA79780E090E04AE0B6
:10F9D0000E94405EE2E4FFE084918F010F5F1F4FC1
:10F9E000882321F00E949C5BF801F6CFA3966EADB0
:10F9F0007FADA39780E090E04AE00E94405EE2E3A2
:10FA0000FFE084918F010F5F1F4F882309F43FC0EF
:10FA10000E949C5BF801F5CF8091830F811141C05A
:10FA2000E2E5FFE284918F010F5F1F4F811103C058
:10FA30000BED12E004C00E949C5BF801F3CFF801CB
:10FA400081918F01882319F00E949C5BF8CFA596C5
:10FA50006EAD7FADA5976456710985E19FE00E9468
:10FA600085C3A3964EAD5FADA39760E070E088E0DC
:10FA70009FE00E944BC3E5E0FFE084918F010F5FA0
:10FA80001F4F882321F00E949C5BF801F6CF8091E4
:10FA9000830F811106C08091C604811102C00F94AA
:10FAA000711A0FB6F8943EBE0FBE2DBE8091830F23
:10FAB000811102C00E946EFA9091C60481E08927EC
:10FAC0000FB6F8949EBE0FBE8DBECF58DF4F0FB657
:10FAD000F894DEBF0FBECDBFDF91CF911F910F9184
:10FAE000FF90EF90DF90CF90BF90AF909F908F905E
:10FAF0007F906F905F904F903F902F9008958F92DE
:10FB00009F92AF92BF92CF92DF92EF92FF920F93AC
:10FB10001F93CF93DF93CDB7DEB7C65AD1090FB687
:10FB2000F894DEBF0FBECDBFCF57DF4F18821982CA
:10FB30001A821B82C158D0408091410390914203A8
:10FB4000A0914303B0914403CB57DF4F888399833F
:10FB5000AA83BB83C558D040C956DF4F198218828B
:10FB6000C759D04084E690E0C756DF4F9983888319
:10FB7000C959D0401092C6049E0129563F4F44E017
:10FB800050E0BE016B577F4FCE0187569F4F0F94B9
:10FB9000FD19C756DF4F88819981C959D040029617
:10FBA000C756DF4F99838883C959D040C956DF4F64
:10FBB00019821882C759D04081E0C156DF4F88832F
:10FBC000CF59D0409E0129563F4F41E050E0BE0141
:10FBD00061567F4FCE0187569F4F0F94FD199E01AE
:10FBE00029563F4F40E150E066EE72E1CE01875664
:10FBF0009F4F0F94FD199E0129563F4F44E050E05E
:10FC000068E87FE0CE0187569F4F0F94FD199E0153
:10FC100029563F4F40E150E066E47DE0CE01875633
:10FC20009F4F0F94FD199E0129563F4F40E150E030
:10FC300066ED72E1CE0187569F4F0F94FD199E012C
:10FC400029563F4F44E050E06AEF72E1CE018756FB
:10FC50009F4F0F94FD199E0129563F4F44E050E0FD
:10FC60006AEE7CE0CE0187569F4F0F94FD199E01EE
:10FC700029563F4F44E050E066EF72E1CE018756CF
:10FC80009F4F0F94FD199E0129563F4F44E050E0CD
:10FC900062ED72E1CE0187569F4F0F94FD199E01D0
:10FCA00029563F4F44E050E06EEC72E1CE0187569A
:10FCB0009F4F0F94FD199E0129563F4F40E150E0A0
:10FCC0006EEF72E1CE0187569F4F0F94FD198AE0C7
:10FCD00097EDA3EABCE3CF57DF4F88839983AA83CC
:10FCE000BB83C158D0409E0129563F4F44E050E0AD
:10FCF000BE016F577F4FCE0187569F4F0F94FD195E
:10FD0000BE016D597F4F8CE0FB0111928A95E9F796
:10FD10009E0129563F4F4CE050E0CE0187569F4F41
:10FD20000F94FD1980E090E0A0E2B1E4C757DF4FE7
:10FD300088839983AA83BB83C958D0409E012956E2
:10FD40003F4F44E050E0BE0167577F4FCE018756DA
:10FD50009F4F0F94FD19CF57DF4F188219821A82D7
:10FD60001B82C158D04083E0C056DF4F8883C05A01
:10FD7000D040CF55DF4F8883C15AD0409E012956CD
:10FD80003F4F44E050E0BE016F577F4FCE01875692
:10FD90009F4F0F94FD199E0129563F4F41E050E0BF
:10FDA000BE0160567F4FCE0187569F4F0F94FD19BD
:10FDB0009E0129563F4F41E050E0BE016F557F4FF5
:10FDC000CE0187569F4F0F94FD191AE011509E01E6
:10FDD00029563F4F44E050E0112349F0BE016F57D0
:10FDE0007F4FCE0187569F4F0F94FD19EFCF6AE2E8
:10FDF0007CE0CE0187569F4F0F94FD199E01295636
:10FE00003F4F44E250E06AEA7FE0CE0187569F4FC1
:10FE10000F94FD1983E0CE55DF4F8883C25AD0403E
:10FE2000CD55DF4F8883C35AD040C357DF4F188268
:10FE300019821A821B82CD58D040CF56DF4F1882CC
:10FE400019821A821B82C159D040CF57DF4F1882C6
:10FE500019821A821B82C158D0409E0129563F4FF9
:10FE600041E050E0BE016E557F4FCE0187569F4F57
:10FE70000F94FD199E0129563F4F41E050E0BE010D
:10FE80006D557F4FCE0187569F4F0F94FD199E01F0
:10FE900029563F4F44E050E0BE016F567F4FCE01E0
:10FEA00087569F4F0F94FD199E0129563F4F44E0FE
:10FEB00050E0BE0163577F4FCE0187569F4F0F948E
:10FEC000FD190AE010E00150110971F09E01295658
:10FED0003F4F44E050E0BE016F577F4FCE01875641
:10FEE0009F4F0F94FD19EFCFCC55DF4F1882C45AA6
:10FEF000D0408FEFCB55DF4F8883C55AD0409E014D
:10FF000029563F4F41E050E0BE016C557F4FCE0176
:10FF100087569F4F0F94FD199E0129563F4F41E090
:10FF200050E0BE016B557F4FCE0187569F4F0F9417
:10FF3000FD199E0129563F4F44E050E066E27CE007
:10FF4000CE0187569F4F0F94FD199E0129563F4FB2
:10FF50004CE050E06AE17CE0CE0187569F4F0F9461
:10FF6000FD199E0129563F4F44E050E066E17CE0D8
:10FF7000CE0187569F4F0F94FD199E0129563F4F82
:10FF800044E050E066E07CE0CE0187569F4F0F943E
:10FF9000FD199E0129563F4F44E050E064E87FE0A0
:10FFA000CE0187569F4F0F94FD199E0129563F4F52
:10FFB00044E050E062E07CE0CE0187569F4F0F9412
:10FFC000FD199E0129563F4F4CE050E06AE07CE06D
:10FFD000CE0187569F4F0F94FD199E0129563F4F22
:10FFE00044E050E06CE47CE0CE0187569F4F0F94D4
:10FFF000FD199E0129563F4F44E050E068E47CE043
:020000021000EC
:10000000CE0187569F4F0F94FD199E0129563F4FF1
:1000100044E050E060E57CE0CE0187569F4F0F94AE
:10002000FD1910E0C12C80E8D82E8BE3E82E85E482
:10003000F82E812C912C90E8A92E9FE3B92E111156
:100040003AC09E0129563F4F44E050E06BE37CE00C
:10005000CE0187569F4F0F94FD199E0129563F4FA1
:1000600044E050E063E47CE0CE0187569F4F0F945C
:10007000FD199E0129563F4F44E050E06FE37CE0BC
:10008000CE0187569F4F0F94FD19CF57DF4F8882BF
:100090009982AA82BB82C158D0409E0129563F4F07
:1000A00044E050E0BE016F577F4FCE0187569F4F0F
:1000B0000F94FD192EC0CF57DF4FC882D982EA8234
:1000C000FB82C158D0409E0129563F4F44E050E08A
:1000D000BE016F577F4FCE0187569F4F0F94FD197A
:1000E000CF57DF4F188219821A821B82C158D04025
:1000F00004E0015071F09E0129563F4F44E050E06A
:10010000BE016F577F4FCE0187569F4F0F94FD1949
:10011000F0CF1F5F153009F092CF84E190E0C55613
:10012000DF4F99838883CB59D0409E0129563F4F9A
:1001300042E050E0BE0165567F4FCE0187569F4F8B
:100140000F94FD199E0129563F4F44E050E063E7AC
:100150007CE0CE0187569F4F0F94FD199E012956D2
:100160003F4F44E050E06FE67CE0CE0187569F4F62
:100170000F94FD199E0129563F4F44E050E06BE675
:100180007CE0CE0187569F4F0F94FD1980E290E0EE
:10019000C356DF4F99838883CD59D0409E0129569D
:1001A0003F4F42E050E0BE0163567F4FCE0187567D
:1001B0009F4F0F94FD19CA55DF4F1882C65AD04081
:1001C00080E2EFE8F2E0DE019D9601900D928A95C3
:1001D000E1F79E0129563F4F41E050E0BE016A55CC
:1001E0007F4FCE0187569F4F0F94FD199E012956D0
:1001F0003F4F40E250E0BE01635D7F4FCE01875626
:100200009F4F0F94FD199E0129563F4F41E050E04A
:100210006AE37CE0CE0187569F4F0F94FD1910E0F2
:10022000111110C08091360C9091370CA091380CB0
:10023000B091390CCF57DF4F88839983AA83BB8352
:10024000C158D0409E0129563F4F44E050E0BE01C6
:100250006F577F4FCE0187569F4F0F94FD191F5F39
:100260001530F1F6BE01635B7F4F86E1FB01119211
:100270008A95E9F79E0129563F4F46E150E0CE01AD
:1002800087569F4F0F94FD198CE2EFEAF2E0DE01F2
:10029000119601900D928A95E1F79E0129563F4FE4
:1002A0004CE250E0BE016F5F7F4FCE0187569F4FFB
:1002B0000F94FD19BE0165587F4F86E0FB01119236
:1002C0008A95E9F79E0129563F4F46E050E0CE015E
:1002D00087569F4F0F94FD19CF57DF4F1882198211
:1002E0001A821B82C158D0409E0129563F4F44E0DC
:1002F00050E0BE016F577F4FCE0187569F4F0F943E
:10030000FD19BE0161597F4F8CE0FB0111928A9566
:10031000E9F79E0129563F4F4CE050E0CE01875649
:100320009F4F0F94FD19CF57DF4F188219821A8201
:100330001B82C158D0401CE1115071F09E0129561A
:100340003F4F44E050E0BE016F577F4FCE018756CC
:100350009F4F0F94FD19F0CFCF57DF4F18821982AE
:100360001A821B82C158D04014E0115071F09E01D6
:1003700029563F4F44E050E0BE016F577F4FCE01FA
:1003800087569F4F0F94FD19F0CF10E0111110C048
:100390008091320C9091330CA091340CB091350CBB
:1003A000CF57DF4F88839983AA83BB83C158D0403E
:1003B0009E0129563F4F44E050E0BE016F577F4FEA
:1003C000CE0187569F4F0F94FD191F5F1530F1F630
:1003D00010E0111110C080912E0C90912F0CA09163
:1003E000300CB091310CCF57DF4F88839983AA83AB
:1003F000BB83C158D0409E0129563F4F44E050E096
:10040000BE016F577F4FCE0187569F4F0F94FD1946
:100410001F5F1530F1F68091C604811167C0C75681
:10042000DF4FE880F980C959D040F4E6EF1AF108AF
:10043000C956DF4F88819981C759D040CB56DF4FCD
:1004400099838883C559D04084E690E0C756DF4F32
:1004500099838883C959D0409E0129563F4F44E073
:1004600050E06BED72E0CE0187569F4F0F94FD195F
:100470009E0129563F4F42E050E0BE016B567F4F30
:10048000CE0187569F4F0F94FD19E2E5FFE284915C
:100490008F010F5F1F4F882321F00E949C5BF801A2
:1004A000F6CFB70183EF9EE00E9485C3CB56DF4FA6
:1004B00048815981C559D04060E070E086EE9EE0E9
:1004C0000E944BC3E3EEFEE084918F010F5F1F4F4C
:1004D000882321F00E949C5BF801F6CFC7010E949F
:1004E0003C779091C604892B8093C6049091C604F2
:1004F00081E08927CA55DF4F0FB6F894DEBF0FBEE3
:10050000CDBFDF91CF911F910F91FF90EF90DF90C2
:10051000CF90BF90AF909F908F900895CF92DF9231
:10052000EF92FF920F931F93CF93DF9300D01F9210
:10053000CDB7DEB781E08093060280912D139091B4
:100540002E13A0912F13B0913013B7FF08C0109253
:100550002D1310922E1310922F131092301380919E
:10056000311390913213A0913313B0913413409111
:100570002D1350912E1360912F1370913013841707
:100580009507A607B70744F480932D1390932E1375
:10059000A0932F13B093301380914D02882379F1EB
:1005A00040912D1350912E1360912F1370913013A1
:1005B0008091351390913613A0913713B091381371
:1005C0006A017B01C80ED91EEA1EFB1EC701B601D7
:1005D0000F94D34420E030E048EC52E40F943445CB
:1005E00069837A838B839C83CE0101960F94F011EB
:1005F000BC0180913B1390913C130E9431C7109134
:100600001E1311110AC080913D13882309F442C0C2
:1006100080914D02882309F43DC040912D135091E3
:100620002E1360912F137091301380913513909198
:100630003613A0913713B09138136A017B01C80EAD
:10064000D91EEA1EFB1EC701B6010F94D34420E059
:1006500030E048EC52E40F9434450F94424AE09164
:100660003913F0913A13309721F0608371838283BC
:100670009383E0913E13F0913F13309731F08091D6
:100680003D13811101C01111199580911E13811123
:100690000E9454C610921E130F900F900F900F904F
:1006A000DF91CF911F910F91FF90EF90DF90CF904E
:1006B0000895CF92DF92EF92FF920F931F93CF9303
:1006C000DF9300D01F92CDB7DEB781E080930602A2
:1006D00080912D1390912E13A0912F13B091301370
:1006E000B7FF08C010922D1310922E1310922F13E3
:1006F000109230138091311390913213A0913313E3
:10070000B091341340912D1350912E1360912F13FB
:100710007091301384179507A607B70744F48093A8
:100720002D1390932E13A0932F13B0933013809119
:100730004D02882379F140912D1350912E13609131
:100740002F13709130138091351390913613A0912F
:100750003713B09138136A017B01C80ED91EEA1E07
:10076000FB1EC701B6010F94D54420E030E048ECF1
:1007700052E40F94344569837A838B839C83CE0142
:1007800001960F94F011BC0180913B1390913C13A2
:100790000E9431C710911E13111109C080913D13A1
:1007A000882309F43FC080914D028823D9F14091FC
:1007B0002D1350912E1360912F137091301380914F
:1007C000351390913613A0913713B09138136A0105
:1007D0007B01C80ED91EEA1EFB1EC701B6010F948D
:1007E000D54420E030E048EC52E40F943445E091E9
:1007F0003913F0913A13309721F06083718382832B
:100800009383E0913E13F0913F13309731F0809144
:100810003D13811101C01111199580911E13811191
:100820000E9454C610921E130F900F900F900F90BD
:10083000DF91CF911F910F91FF90EF90DF90CF90BC
:100840000895CF92DF92EF92FF920F931F93CF9371
:10085000DF9300D01F92CDB7DEB781E08093060210
:1008600080912D1390912E13A0912F13B0913013DE
:10087000B7FF08C010922D1310922E1310922F1351
:10088000109230138091311390913213A091331351
:10089000B091341340912D1350912E1360912F136A
:1008A0007091301384179507A607B70744F4809317
:1008B0002D1390932E13A0932F13B0933013809188
:1008C0004D02882379F140912D1350912E136091A0
:1008D0002F13709130138091351390913613A0919E
:1008E0003713B09138136A017B01C80ED91EEA1E76
:1008F000FB1EC701B6010F94D5442AE037ED43E251
:100900005CE30F94344569837A838B839C83CE01A7
:1009100001960F948E10BC0180913B1390913C1373
:100920000E9431C710911E13111109C080913D130F
:10093000882309F43FC080914D028823D9F140916A
:100940002D1350912E1360912F13709130138091BD
:10095000351390913613A0913713B09138136A0173
:100960007B01C80ED91EEA1EFB1EC701B6010F94FB
:10097000D5442AE037ED43E25CE30F943445E0913F
:100980003913F0913A13309721F060837183828399
:100990009383E0913E13F0913F13309731F08091B3
:1009A0003D13811101C01111199580911E13811100
:1009B0000E9454C610921E130F900F900F900F902C
:1009C000DF91CF911F910F91FF90EF90DF90CF902B
:1009D0000895CF92DF92EF92FF920F931F93CF93E0
:1009E000DF9300D01F92CDB7DEB781E0809306027F
:1009F00080912D1390912E13A0912F13B09130134D
:100A0000B7FF08C010922D1310922E1310922F13BF
:100A1000109230138091311390913213A0913313BF
:100A2000B091341340912D1350912E1360912F13D8
:100A30007091301384179507A607B70744F4809385
:100A40002D1390932E13A0932F13B09330138091F6
:100A50004D02882379F140912D1350912E1360910E
:100A60002F13709130138091351390913613A0910C
:100A70003713B09138136A017B01C80ED91EEA1EE4
:100A8000FB1EC701B6010F94D5442AE037ED43E2BF
:100A90005CE30F94344569837A838B839C83CE0116
:100AA00001960F944F11BC0180913B1390913C1320
:100AB0000E9431C710911E13111109C080913D137E
:100AC000882309F43FC080914D028823D9F14091D9
:100AD0002D1350912E1360912F137091301380912C
:100AE000351390913613A0913713B09138136A01E2
:100AF0007B01C80ED91EEA1EFB1EC701B6010F946A
:100B0000D5442AE037ED43E25CE30F943445E091AD
:100B10003913F0913A13309721F060837183828307
:100B20009383E0913E13F0913F13309731F0809121
:100B30003D13811101C01111199580911E1381116E
:100B40000E9454C610921E130F900F900F900F909A
:100B5000DF91CF911F910F91FF90EF90DF90CF9099
:100B60000895CF92DF92EF92FF920F931F93CF934E
:100B7000DF9300D01F92CDB7DEB781E080930602ED
:100B800080912D1390912E13A0912F13B0913013BB
:100B9000B7FF08C010922D1310922E1310922F132E
:100BA000109230138091311390913213A09133132E
:100BB000B091341340912D1350912E1360912F1347
:100BC0007091301384179507A607B70744F48093F4
:100BD0002D1390932E13A0932F13B0933013809165
:100BE0004D02882379F140912D1350912E1360917D
:100BF0002F13709130138091351390913613A0917B
:100C00003713B09138136A017B01C80ED91EEA1E52
:100C1000FB1EC701B6010F94D5442FE632E143E82D
:100C20005AE30F94344569837A838B839C83CE0186
:100C300001960F94C921BC0180913B1390913C1304
:100C40000E9431C710911E13111109C080913D13EC
:100C5000882309F43FC080914D028823D9F1409147
:100C60002D1350912E1360912F137091301380919A
:100C7000351390913613A0913713B09138136A0150
:100C80007B01C80ED91EEA1EFB1EC701B6010F94D8
:100C9000D5442FE632E143E85AE30F943445E0911E
:100CA0003913F0913A13309721F060837183828376
:100CB0009383E0913E13F0913F13309731F0809190
:100CC0003D13811101C01111199580911E138111DD
:100CD0000E9454C610921E130F900F900F900F9009
:100CE000DF91CF911F910F91FF90EF90DF90CF9008
:100CF0000895CF92DF92EF92FF920F931F93CF93BD
:100D0000DF9300D01F92CDB7DEB781E0809306025B
:100D100080912D1390912E13A0912F13B091301329
:100D2000B7FF08C010922D1310922E1310922F139C
:100D3000109230138091311390913213A09133139C
:100D4000B091341340912D1350912E1360912F13B5
:100D50007091301384179507A607B70744F4809362
:100D60002D1390932E13A0932F13B09330138091D3
:100D70004D02882379F140912D1350912E136091EB
:100D80002F13709130138091351390913613A091E9
:100D90003713B09138136A017B01C80ED91EEA1EC1
:100DA000FB1EC701B6010F94D5442AE037ED43E29C
:100DB0005CE30F94344569837A838B839C83CE01F3
:100DC00001960F942013BC0180913B1390913C132A
:100DD0000E9431C710911E13111109C080913D135B
:100DE000882309F43FC080914D028823D9F14091B6
:100DF0002D1350912E1360912F1370913013809109
:100E0000351390913613A0913713B09138136A01BE
:100E10007B01C80ED91EEA1EFB1EC701B6010F9446
:100E2000D5442AE037ED43E25CE30F943445E0918A
:100E30003913F0913A13309721F0608371838283E4
:100E40009383E0913E13F0913F13309731F08091FE
:100E50003D13811101C01111199580911E1381114B
:100E60000E9454C610921E130F900F900F900F9077
:100E7000DF91CF911F910F91FF90EF90DF90CF9076
:100E80000895CF92DF92EF92FF920F931F93CF932B
:100E900081E08093060280912D1390912E13A091F2
:100EA0002F13B0913013B7FF08C010922D1310927A
:100EB0002E1310922F1310923013809131139091B2
:100EC0003213A0913313B091341340912D135091EC
:100ED0002E1360912F137091301384179507A60776
:100EE000B70744F480932D1390932E13A0932F13E0
:100EF000B093301380914D028823E1F140912D137E
:100F000050912E1360912F137091301380913513EF
:100F100090913613A0913713B09138138A019B0139
:100F2000080F191F2A1F3B1FC901B8010F94D54490
:100F30006B017C0120E030E0A9010F94CF4487FDD4
:100F400005C020E030E040E05FE304C020E030E096
:100F500040E05FEBC701B6010F94F9480F943D4A9A
:100F6000CB010F946A14BC0180913B1390913C1308
:100F70000E9431C7C0911E13C11108C080913D135A
:100F80008823C9F180914D028823A9F140912D1346
:100F900050912E1360912F1370913013809135135F
:100FA00090913613A0913713B09138138A019B01A9
:100FB000080F191F2A1F3B1FC901B8010F94D54400
:100FC000E0913913F0913A13309721F060837183E7
:100FD00082839383E0913E13F0913F13309731F079
:100FE00080913D13811101C0C111199580911E138B
:100FF00081110E9454C610921E13CF911F910F9120
:10100000FF90EF90DF90CF900895CF92DF92EF9214
:10101000FF926B017C0183E3C816D104E104F10463
:1010200070F082E3C81AD108E108F10862E370E0C9
:1010300080E090E00F949A0E0E94BEE8ECCFC701CA
:10104000B6010F949A0EFF90EF90DF90CF900C9422
:10105000BEE82091190230911A022F5031098217EF
:1010600093070CF49C013093DC042093DB0480E0B4
:101070000C94CDE30F931F930F94D20E0091F104C3
:101080001091F2042091F3043091F404DC01CB01BF
:10109000801B910BA20BB30BB7FD0CC086B186FB76
:1010A000992790F981E08927349B8260329B846084
:1010B0008093F0048091F00481709091F00491FD90
:1010C00082609091EF04891751F18130A9F028F0E6
:1010D000823041F0833059F020C0913089F0923055
:1010E000A9F01BC0992361F0933081F016C09130B4
:1010F00069F0923091F404C0992341F0933069F47F
:101100009091EE0420910602921B05C02091EE04FE
:1011100090910602920F9093EE048093EF041F913A
:101120000F9108950F931F93CF93DF938C0167FF67
:1011300003C01092350D60E08091350D90E0262FB0
:10114000062E000C330B281739071CF16093350D60
:10115000C8010F941F44800F911FEC01C01BD10BDD
:10116000C334D1053CF00197FC012491207C203848
:10117000D1F3F3CFDD27AE01B80182EF9CE00F94ED
:101180004044CE50D34F188283E080934D0210929A
:10119000F10CDF91CF911F910F910895CF93DF93C1
:1011A0002091350D21111FC0FC0101900020E9F7AD
:1011B0003197EF01C81BD90BC334D1052CF0229114
:1011C000207C2038E1F3F5CFBC01DD27AE0182EFB2
:1011D0009CE00F94D54CCE50D34F188283E080937F
:1011E0004D021092F10CDF91CF9108954F925F92D2
:1011F0006F927F928F929F92AF92BF92CF92DF9227
:10120000EF92FF920F931F93CF93DF9300D01F9223
:10121000CDB7DEB78091CF0481111EC000910502C9
:101220000F3FD1F00F94D20EC090CB04D090CC04DD
:10123000E090CD04F090CE04DC01CB018C199D0927
:10124000AE09BF09B7FD08C08091A80F9091A90F02
:101250008F5F8F70891310C20DDF8091F00482FFC1
:1012600044C08091ED04811142C091E09093ED045F
:101270002091EE0C211103C08091DA04892780931C
:101280001E131092EE0C83E080934D021092F00436
:101290000F94D20EDC01CB018C509E4FAF4FBF4F4D
:1012A0008093F1049093F204A093F304B093F404B8
:1012B00088E893E19C838B8382E090E09A83898322
:1012C000BE016D5F7F4FCE0101960E9462F816E06D
:1012D000115069F082E090E10E945D5662E070E09A
:1012E00080E090E00F949A0EF3CF1092ED0480917D
:1012F0000901817091E098271091EC04191731F1E0
:101300009093EC04811110C264EF71E080E090E0F2
:101310007CDE0E941FF7123009F002C21092751095
:101320008BE1EAE7F0E1A9E9B0E101900D928A953D
:10133000E1F78091781090917910909398108093B4
:10134000971083E080934D020E946AC70F94D20EDB
:101350006B017C018091E8049091E904A091EA047A
:10136000B091EB04A7019601281B390B4A0B5B0BCC
:1013700057FD0EC2D701C6018C599F4FAF4FBF4FCB
:101380008093E8049093E904A093EA04B093EB04FB
:101390008091EE04082E000C990B97FF03C09195E5
:1013A0008195910984302CF480911E13811194C091
:1013B000A4C08091D904882309F467C08091EE0409
:1013C0008090D5049090D604A090D704B090D80413
:1013D00081149104A104B10409F44AC0082E000C40
:1013E000990B97FF03C0919581959109682F87FF0D
:1013F00002C063E0680F65956595062E000C770BBB
:10140000880B990B0F94D5442B013C01C701B60101
:10141000681979098A099B090F94D3449B01AC018F
:10142000C301B2010F94D54920E030E04AE754E40B
:101430000F9434454B015C0120E030E040E253E47E
:101440000F946D4B87FF0FC020E030E046E952E477
:10145000C501B4010F946D4B87FD0AC02AE030E04E
:1014600040E050E009C024E630E040E050E004C035
:1014700021E030E040E050E0C092D504D092D604A4
:10148000E092D704F092D80404C021E030E040E0BC
:1014900050E0A091EE040A2E000CBB0B0F94664C9A
:1014A00024E030E040E050E00F94424C80912D1356
:1014B00090912E13A0912F13B0913013820F931F90
:1014C000A41FB51F80932D1390932E13A0932F1359
:1014D000B09330131092EE04D701C601805A9541A3
:1014E000AF4FBF4F8093E4049093E504A093E604CC
:1014F000B093E70481E080934D0220915702309130
:10150000580247EC2237340741F480915602882371
:1015100009F416C18150809356022B5C394D71F449
:101520008091231390912413891740F490915602CF
:10153000992309F415C191509093560280916F0040
:10154000282F227081FF05C080916F008D7F8093CE
:101550006F008091D0049091D104A091D204B091F9
:10156000D304222329F020916F00226020936F0082
:1015700020914D02222309F449C04AE0B695A7956F
:10158000979587954A95D1F70097E1E0AE07B105A9
:1015900020F08FEF9FEFA0E0B0E096958795009741
:1015A00039F04091E2045091E3044817590770F56F
:1015B000223050F0243028F0243031F410924D02C3
:1015C00003C081E080934D02E0915702F0915802F0
:1015D000199510921E138090E2049090E304A12CC0
:1015E000B12C0F94D20EDC01CB018C199D09AE09F0
:1015F000BF0988169906AA06BB0640F40F94D20EBE
:101600006C197D097093E3046093E20480915702A2
:10161000909158028257974C21F08091D4048823EE
:1016200079F020E6C20E2AEED21EE11CF11CC09217
:10163000E404D092E504E092E604F092E7040FC0DF
:101640008091E4049091E504A091E604B091E70450
:10165000C81AD90AEA0AFB0AF7FE0E944EC6809110
:101660004D02813031F0833009F092C00F94BA01FD
:101670008FC010924D028CC0C0900102D090020227
:10168000E0900302F090040234E003028001112490
:10169000F801E152FD4F20E030E040E752E4608184
:1016A0007181828193810F94D54960930102709377
:1016B000020280930302909304020E94885B035B02
:1016C0001C4E2091C7043091C8044091C904509128
:1016D000CA04F80160817181828193810F94F94875
:1016E000F80160837183828393831092C704109200
:1016F000C8041092C9041092CA048FEF80930502A7
:1017000081E08093CF040E94C5671092CF04C092FD
:101710000102D0920202E0920302F09204029CCDF8
:1017200060E084EB9FE00AC0109222101092231018
:10173000123009F406CE60E087EA9FE0F3DC01CEC8
:1017400089E0809356028091E2049091E30401972E
:101750009093E3048093E20481E080934D02DDCE18
:1017600096E09093560291E090934D028F5F8093A4
:101770002313D701C601805A9541AF4FBF4F8093C5
:10178000E4049093E504A093E604B093E704D6CE76
:101790000F900F900F900F90DF91CF911F910F91AD
:1017A000FF90EF90DF90CF90BF90AF909F908F9081
:1017B0007F906F905F904F900895CF92DF92EF925D
:1017C000FF920F931F930F94D20E0091DE0410919D
:1017D000DF042091E0043091E1046B017C01C01A28
:1017E000D10AE20AF30AF7FC13C02091DD04209528
:1017F0002093DD04DC01CB018A549C4FAF4FBF4FD7
:101800008093DE049093DF04A093E004B093E1049E
:1018100081E09091DD04911101C080E01F910F9152
:10182000FF90EF90DF90CF900895FC0180E090E072
:101830002491222339F02491207C203809F001964C
:101840003196F6CF0895FC0120E030E09191992384
:1018500031F0907C9038D1F32F5F3F4FF7CFC90123
:1018600008950E946AC73E98469A3C98449A3A98CE
:10187000429AEAE0F1E080818E7F808380910B01C3
:10188000809581708093090182E08093EC04F2DB03
:101890001092EE040895CF93DF93EC010E940BC6E3
:1018A00040E050E0BA01CE01DF91CF910C942BC6FD
:1018B0002F923F924F925F926F927F928F929F9260
:1018C000AF92BF92CF92DF92EF92FF920F931F934E
:1018D000CF93DF93CDB7DEB7C256D6400FB6F8949C
:1018E000DEBF0FBECDBF41E061E081E00E94E14973
:1018F00081110C94E99A8091010C882371F08FE496
:101900000E94765B882319F00E94EB5A03C08FE493
:101910000E942D5B81110C94E99AFE01ED54FA4F5F
:101920008CE3DF011D928A95E9F71091010CC45CEC
:10193000D94F1883CC53D6408AE40E942D5B88236C
:1019400021F00E94B4490C94E99A86E50E94765BE6
:10195000882349F00E94CA5AC65CD94F79836883AC
:10196000CA53D64006C0C65CD94F19821882CA53E2
:10197000D640C65CD94F08811981CA53D64005307C
:10198000110570F0E6EAF1E184918F010F5F1F4FBE
:10199000882311F40C94E99A0E949C5BF801F4CF1F
:1019A00084E40E94765B882319F00E94EB5A03C0FE
:1019B00084E40E942D5BC45BD94F8883CC54D6400D
:1019C000C65CD94F28813981CA53D64023303105AE
:1019D0008CF484E50E94765B882319F00E94EB5A10
:1019E00003C084E50E942D5BC35CD94F8883CD532F
:1019F000D64006C011E0C35CD94F1883CD53D64002
:101A000088E50E94765B882321F00E94CA5A162F2F
:101A100001C019E089E50E94765B882321F00E94CD
:101A2000CA5A062F01C009E080E50E94765B811149
:101A300007C0C75CD94F1883C953D640202E08C0B1
:101A40000E94CA5AC75CD94F6883C953D640262E14
:101A5000C75CD94F8881C953D6408250883070F016
:101A6000EDE7F1E184918F010F5F1F4F882311F49F
:101A70000C94E99A0E949C5BF801F4CF8EEF820DE2
:101A8000883070F0E4E5F1E184918F010F5F1F4F22
:101A9000882311F40C94E99A0E949C5BF801F4CF1E
:101AA00083E50E94765B882319F00E94FA5A04C0ED
:101AB00060E070E08AE795E420E030E040E752E43F
:101AC0000F94D5496093070270930802809309022E
:101AD00090930A028CE40E94765B882381F00E9436
:101AE000FA5A2091D60C3091D70C4091D80C5091D5
:101AF000D90C0F94F8480F943D4A7B0104C006E9C5
:101B0000E02EFF24FA9482E50E94765B882381F020
:101B10000E94FA5A2091D60C3091D70C4091D80CE3
:101B20005091D90C0F94F8480F943D4A6B0103C0B3
:101B30001AE6C12ED12C86E40E94765B882381F0C0
:101B40000E94FA5A2091DA0C3091DB0C4091DC0CA7
:101B50005091DD0C0F94F8480F943D4A5B0104C08E
:101B6000B6E9AB2EBB24BA9482E40E94765B88234C
:101B700081F00E94FA5A2091DA0C3091DB0C4091EE
:101B8000DC0C5091DD0C0F94F8480F943D4A8B010A
:101B900002C00AE610E0B7010F2C000C880B990B6D
:101BA0000F94D544C75DD94F688379838A839B831B
:101BB000C952D6409B01AC010F94344520E030E07F
:101BC000A9010F94F9482B013C0120E030E442E5E3
:101BD00056E40F94CF44181654F020E030E94FE259
:101BE00056E4C301B2010F94CF44181674F4E8E32D
:101BF000F1E184918F010F5F1F4F882311F40C9442
:101C0000E99A0E949C5BF801F4CFB6010D2C000C00
